:020000040800F2
:1000000020580020F5340008510300085F8A0008DA
:1000100053030008550300085703000800000000C0
:10002000000000000000000000000000073500088C
:100030005903000800000000E7890008C902000811
:100040000F3500080F3500080F3500080F35000880
:100050000F3500080F3500089B060008AF060008A2
:10006000C3060008D7060008EB0600080F35000895
:100070000F3500080F3500080F3500080F35000850
:100080000F3500080F3500080F3500080F35000840
:100090000F3500080F3500080F350008FF0600086F
:1000A0000F3500080F3500080F3500080F35000820
:1000B0000F3500080F3500080F3500080F35000810
:1000C0000F3500080F3500080F3500080F35000800
:1000D0000F350008390900080F3500080F350008F2
:1000E0002F0700080F3500080F3500080F350008EE
:1000F0000F3500080F3500080F3500080F350008D0
:100100000F3500080F3500080F3500080F350008BF
:100110000F3500080F3500080F3500080F350008AF
:100120000F3500080F3500080F3500080F3500089F
:10013000DFF810D00BF08AFD004800472736000892
:10014000AFF3008020580020FEE71CB5C820032133
:10015000CDE900104FF400630022AFF2130118A0A4
:1001600007F034FF00201CBDEFF3098070470844FE
:10017000704770B5012502260021032008F040FDDC
:1001800000240121032008F050FD322008F09EF8E1
:100190000021032008F049FD322008F097F8641C84
:1001A000E4B20A2CEDD331462846FFF7E0FFFFF713
:1001B000DBFF046804A0214605F022FE204670BD46
:1001C0005468726561643300632076616C756520E4
:1001D0003A2025640D0A000008B5032001F0C2FC96
:1001E0004748816941F001018161806900F00100A7
:1001F0000090002211466FF00B0001F0C0FC0022BD
:1002000011466FF00A0001F0BAFC002211466FF0AF
:10021000090001F0B4FC00221146501F01F0AFFCB0
:1002200000221146101F01F0AAFC00220F21901E8F
:1002300001F0A5FC00220F21501E01F0A0FC314866
:10024000416821F0E0614160416841F00071416026
:1002500008BD30B58FB00121059108040690002437
:100260000794099102250C950D904FF4E0100E9023
:1002700005A801F090FD20B13F22234923A005F0FD
:100280007CFE0F200090019502944FF48060039053
:1002900004940221684601F064FF20B147221A4904
:1002A000264805F06AFE02F02DF86421B0FBF1F05B
:1002B00001F0A7FC042001F01EFD00220F21501EBA
:1002C00001F05DFC0FB030BD10B505F073FA03F01E
:1002D000A3F803F02FF9BDE8104005F07BBA10B584
:1002E00003F07CF8FFF7B5FF1549164805F023FF2A
:1002F00003F04EF9BDE8104013A005F0D0BD00009A
:100300000010024000000140E4BC000848414C5F7E
:100310005243435F4F7363436F6E6669672826528B
:1003200043435F4F7363496E6974537472756374AA
:1003300029203D3D2048414C5F4F4B00A0CF000895
:100340000000012020580020756172743100000007
:100350007047FEE7FEE7FEE77047000008B5FE487D
:10036000816941F004018161806900F0040000901E
:1003700008BD08B5F848816941F0080181618069CC
:1003800000F00800009008BD08B5F348816941F00D
:1003900010018161806900F01000009008BD08B56F
:1003A000ED48816941F020018161806900F0200001
:1003B000009008BD08B5E848816941F040018161BD
:1003C000806900F04000009008BD08B5E2488169EE
:1003D00041F080018161806900F08000009008BDDB
:1003E00008B5DD48816941F480718161806900F45C
:1003F0008070009008BD912807D2D84901EB001009
:100400000168491C00D1002070470020704710B5DA
:10041000C8B2FFF7F0FF002807D081898068BDE8E7
:100420001040D2B289B200F09ABD10BD10B50022C2
:10043000C8B2FFF7E0FF30B181898068BDE81040A5
:1004400089B200F085BD104610BD7FB51446C8B214
:10045000FFF7D1FF0546002D22D068688047E86885
:1004600000900121019100200290032203929CB18F
:10047000012C06D0022C06D0032C07D0042C09D066
:100480000AE0019008E00190029105E0019002204D
:10049000029001E0112001906946A86800F0F0FB8D
:1004A0007FBD2DE9F0470E46DDF8209017469846AF
:1004B000F0B2FFF7A0FF50B1C06800F069F9044640
:1004C000002C01DB102C04D30620BDE8F0870620A9
:1004D000FBE708F071FA0546A14B04EB440033F941
:1004E0002020B2420FD103EB80014C6844450AD171
:1004F0004C88BC4207D18968494504D1284608F098
:100500005FFA0020E1E7521C04D0284608F058FAB0
:100510000720DAE723F8206003EB8000C0F80480AE
:100520004780C0F80890284608F04AFA0020CCE737
:1005300070B54FF0FF35C8B2FFF75DFF48B1C06836
:1005400000F026F90446002C01DB102C03D3062012
:1005500070BD062070BD08F02FFA0146804B04EBF9
:10056000440033F92020521C0CD023F8205003EB18
:1005700080000022426042808260084608F020FA33
:10058000002070BD084608F01BFA002070BD2DE960
:10059000FF47C8B2FFF72FFF0446200008D000260F
:1005A000DFF8C091012A05D07AB3062004B08CE7A9
:1005B0000620FBE7E06800F0EBF80546002D01DBC4
:1005C000102D01D30620F1E708F0F6F98046DFF898
:1005D00090A105EB45073AF92700401C10D009EB24
:1005E000850560688047E0680090032003900AEB6F
:1005F0008700408850B101280DD0022813D10FE0A8
:10060000404608F0DDF90620D0E71EE0564801908C
:100610000220029007E0554801900120029002E07C
:100620005348019002966946A06800F029FB95F9AD
:1006300002000022052101F0A2FA95F9020001F062
:10064000BCFA404608F0BCF90DE0E06800F0A0F804
:10065000002803DB102801D209EB80062EB196F9A1
:10066000020001F0B5FA0020A0E706209EE73D4910
:10067000002240313FA008F05FBA10B500F088F8C2
:1006800000EB4001364800EB81004168002903D0AF
:100690008068BDE81040084710BD10B505F08AF825
:1006A000012000F07AFCBDE8104005F093B810B5C9
:1006B00005F080F8022000F070FCBDE8104005F065
:1006C00089B810B505F076F8042000F066FCBDE8A6
:1006D000104005F07FB810B505F06CF8082000F068
:1006E0005CFCBDE8104005F075B810B505F062F887
:1006F000102000F052FCBDE8104005F06BB810B5BA
:1007000005F058F8202000F048FC402000F045FC9F
:10071000802000F042FC4FF4807000F03EFC4FF46B
:10072000007000F03AFCBDE8104005F053B810B579
:1007300005F040F84FF4806000F02FFC4FF40060AB
:1007400000F02BFC4FF4805000F027FC4FF40050D9
:1007500000F023FC10E0000000100240F8BC00088C
:100760000000002008C60008000011100000211041
:100770000000311070696E004FF4804000F00DFCF5
:100780004FF4004000F009FCBDE8104005F022B82D
:1007900001460020012303FA00F28A4204D0401CE3
:1007A0002028F8DB4FF0FF307047000070B5054699
:1007B0000C46002D04D12422E049E1A005F0DDFB28
:1007C00024B92522DD49E3A005F0D7FBE86B2168B9
:1007D0004160002181610C224261C161227902F0F5
:1007E0000F02082A17D0092A17D081602279C2F394
:1007F0000112B2B1012A16D0C1602279C2F381126E
:10080000AAB1012A15D0022A17D0016101F0DDFE3C
:10081000B8B1012070BD8160E8E74FF4805282607A
:10082000E4E7C160E9E74FF40052C260E5E7016127
:10083000ECE74FF4C0610161E8E74FF480610161CA
:10084000E4E7002070BD70B505460C46002D05D1CB
:10085000BA495C221031BAA005F08FFBE86B012287
:10086000102C12D0112C20D190F9401001F01F0350
:100870009A404909890001F1E021C1F8802100680E
:10088000C16821F02001C1600FE090F9401001F033
:100890001F039A404909890001F1E021C1F80021B4
:1008A0000068C16841F02001C160002070BD70B5D2
:1008B00004460D46002C05D1A04975221E31A0A08A
:1008C00005F05BFBE06B00680268D2431206FBD4C4
:1008D0004560012070BD10B50446002C05D1974934
:1008E0008022293196A005F048FBE16B4FF0FF30E4
:1008F00009680A68D243920601D44868C0B210BDA4
:1009000070B50546EC6B002C05D18C499222343130
:1009100094A005F032FB21680868C04380060AD421
:10092000C868800607D50121284608F035FB2168F4
:100930006FF02000086070BD10B504F03BFF8D48DB
:10094000FFF7DEFFBDE8104004F044BF10B54FF4E0
:10095000E131416000218160C16001610C2242618E
:100960008161C16101F031FE002808D07349BDE802
:10097000104040F215123D317FA005F0FEBA10BDC7
:100980001CB56E481C3840680190844C4FF4E1302F
:100990006A4A7849143A0A64019AC1E91102204668
:1009A000FFF7D4FF234640F203127DA1714808F0FF
:1009B000CBFA00201CBDF0B585B002687A4F02204A
:1009C00000247A4903237A4D4602BA4228D18A6923
:1009D00042F480428A618A6902F4804200928A6904
:1009E00042F004028A61896901F004010091010268
:1009F00001910290049301A9284600F041F9019663
:100A00000294039401A9284600F03AF90022052136
:100A1000252001F0B4F8252001F0CFF805B0F0BD95
:100A2000644FBA4228D1CA6942F40032CA61CA6925
:100A300002F4003200928A6942F004028A618969F4
:100A400001F004010091042101910290049301A995
:100A5000284600F015F9082101910294039401A998
:100A6000284600F00DF900220521262001F087F824
:100A7000262001F0A2F8D1E74F4DAA42CED1CA6993
:100A800042F48022CA61CA6902F4802200928A6913
:100A900042F008028A61896901F00801009101961B
:100AA00002900493454D01A9284600F0E9F8E914A5
:100AB00001910294039401A9284600F0E1F8002274
:100AC0000521272001F05BF8272001F076F8A5E743
:100AD00010B5354B0168354A354899420CD19169BA
:100AE00021F4804191614FF4C06100F0BDF9BDE88F
:100AF0001040252001F06CB82E4B99420BD1D169E2
:100B000021F40031D1610C2100F0AEF9BDE81040B4
:100B1000262001F05DB8284881420DD1D06920F42B
:100B20008020D0614FF44061244800F09DF9BDE879
:100B30001040272001F04CB810BD00007CC6000812
:100B400073657269616C20213D2052545F4E554C93
:100B50004C00000063666720213D2052545F4E55D3
:100B60004C4C00007561727420213D2052545F4E40
:100B7000554C4C00EC02002048414C5F554152540A
:100B80005F496E6974287561727448616E646C6542
:100B900029203D3D2048414C5F4F4B00C0000020C4
:100BA000756172743100000000380140001002408D
:100BB000000801400044004000480040000C014093
:100BC0002748016841F0010101604168254A114050
:100BD00041600168244A11400160016821F48021CC
:100BE0000160416821F4FE0141604FF41F01816002
:100BF0001E49C0030860704710B5194A506800F0DC
:100C00000C011B4B1B4800290DD004290DD00829CD
:100C10000DD003605168184AC1F30311515C02689A
:100C2000CA40026010BD0360F4E70360F2E7516858
:100C300001F47011536803F48033022404EB9141F2
:100C400033B153689B0307D50C4B59430160E1E76F
:100C50000A4B59430160DDE7054B59430160D9E771
:100C6000001002400000FFF8FFFFF6FE08ED00E074
:100C700000127A0004010020CCC6000800093D00E3
:100C80002DE9F84F00230024DFF824934FF00F08DC
:100C900009F1040A0AF1040B0BF1040E0127A74025
:100CA0000A683A40BA4275D1DFF808C34D68A5EB2F
:100CB0000C0665452BD00DDC032D34D005DC35B397
:100CC000012D19D0022D2FD11BE0112D16D0122D80
:100CD0002AD119E0B6F5881F19D006DCB6F5803F99
:100CE00015D0B6F5801F1FD111E0B6F5001F0ED04C
:100CF000B6F5041F18D10AE0CB6815E0CB681B1DC0
:100D000012E0CB6808330FE0CB680C330CE08B6843
:100D100023B1012B04D00823476105E0042303E03D
:100D20000823076100E00023FF2A01D8054601E0FF
:100D300000F1040502D84FEA840603E0A4F1080696
:100D40004FEA86062F6808FA06FC27EA0C0703FA22
:100D500006F647EA06072F604D68ED007ED5964DF2
:100D6000AE6946F00106AE61AD6905F0010500957A
:100D7000924D24F003067719BE68A5072D0F08FAD7
:100D800005FC26EA0C06DFF838C2604503D14FF0B7
:100D9000000C25E062E0DFF82CC2604502D14FF084
:100DA000010C1DE0DFF820C2604502D14FF0020CBB
:100DB00016E0DFF818C2604502D14FF0030C0FE0D7
:100DC000DFF80CC2604502D14FF0040C08E0DFF8F8
:100DD00004C2604502D14FF0050C01E04FF0060C53
:100DE0000CFA05FC4CEA060CC7F808C04D68ED0388
:100DF00005D5D9F800501543C9F8005004E0D9F8DA
:100E000000509543C9F800504D68AD0305D5DAF898
:100E100000501543CAF8005004E0DAF8005095433A
:100E2000CAF800504D68ED0205D5DBF800501543B7
:100E3000CBF8005004E0DBF800509543CBF80050AD
:100E40004D68AD0205D5DEF800501543CEF80050D0
:100E500004E0DEF800509543CEF80050641C102CDE
:100E6000FFF41CAFBDE8F88F2DE9F04300224FF0EE
:100E70000F0CDFF8488166E0012393400B4083B3F9
:100E8000FF2B01D8044601E000F1040402D84FEA28
:100E9000820503E0A2F108054FEA850527680CFAF0
:100EA00005F927EA09074FF0040909FA05F947EAA5
:100EB000090766462760C46824EA0304C46022F078
:100EC000030404EB0805AC684FEA82774FEA177712
:100ED00006FA07F606EA0409394CA04202D10024BA
:100EE0001AE02FE0374CA04201D1012414E0364C27
:100EF000A04201D102240FE0344CA04201D10324CE
:100F00000AE0334CA04201D1042405E0314CA04258
:100F100001D1052400E00624BC404C4512D1AC6848
:100F2000B443AC60224C25689D432560241D256890
:100F30009D432560241D25689D432560241D25684B
:100F40009D432560521C31FA02F395D1BDE8F08330
:100F50008068084201D00120704700207047002AB5
:100F600001D001617047090401617047C2684A40BD
:100F7000C260704708B541F480320092009A8261E5
:100F8000816100998161816900918069C00301D507
:100F9000002008BD012008BD704710B50449143178
:100FA0000A68024202D00860FFF767FB10BD00002C
:100FB0000004014000001110001002400000014038
:100FC00000080140000C01400010014000140140E5
:100FD00000180140001C014030B500280DD0F74B2F
:100FE0000168142299420AD2F54B0B44B3FBF2F28A
:100FF00092000264F34AC2630BE0012030BDEF4B64
:101000005B420B44B3FBF2F292000264EB4A083AF3
:10101000C2630222001D42770B6843F6F0729343CD
:10102000D0E900242243D0E902452C43224304693D
:10103000224344692243846922431A430A600021FF
:1010400041628162C162016341630122427701779B
:10105000002030BD10B500281BD001680A6822F0BE
:1010600001020A60016800220A6001684A600168A2
:101070008A600168CA60D14C01681423A1420AD277
:10108000CF4C2144B1FBF3F189000164CD49C16328
:101090000BE0012010BDC94C64422144B1FBF3F1C7
:1010A00089000164C5490839C1632030012190F8E5
:1010B00020309940C36959608261427002700020FB
:1010C00010BD30B590F840500124AC40C56B6C6049
:1010D000046863604368102B04D00368996000685B
:1010E000C26030BD03689A600068C16030BD70B5F1
:1010F0000446002594F8200001280CD0012084F833
:10110000200094F821600020012E06D084F82000F1
:101110000225284670BD022070BD022684F8216099
:10112000A0632068066826F0010606602046FFF7E7
:10113000C8FF2068016841F001010160E9E770B56E
:101140000446002594F8200001280CD0012084F8E2
:10115000200094F821600020012E06D084F82000A1
:101160000225284670BD022070BD022684F8216049
:10117000A0632068066826F0010606602046FFF797
:10118000A0FFE06A28B12068016841F00E0101600B
:1011900009E02068016821F004010160206801680D
:1011A00041F00A0101602068016841F0010101601D
:1011B000D7E701680A6822F00E020A6001680A682F
:1011C00022F001020A6090F84020012303FA02F1A4
:1011D000C26B516080F82130002180F82010084651
:1011E00070472DE9F05F002590F82110022903D007
:1011F00004218163012595E001680A6822F00E024E
:101200000A6001680A6822F001020A606D4E6D4FA3
:101210008036B215DFF8ACC1DFF8A881DFF8A49101
:10122000DFF8A0A1DFF89CB10168083713011402B0
:101230000CF11C0C08F1300809F144090AF1580AB4
:101240000BF16C0B4FF4801EB1422FD9B94201D182
:10125000012227E0614501D1102223E0414521D040
:10126000494501D11A461DE0514501D1224619E0F8
:10127000594501D1724615E0504EB14201D10122CB
:1012800010E04E4E1436B14201D110220AE04B4E0E
:101290002836B14206D0494A3C32914201D11A4621
:1012A00000E022464549091F0A6032E0B94201D1F7
:1012B00001222CE0614501D1102228E0414526D0D1
:1012C000494501D11A4622E0514501D122461EE08E
:1012D000594501D172461AE0B14202D14FF08072F5
:1012E00015E0364EB14201D1012210E0334E1436E2
:1012F000B14201D110220AE0304E2836B14206D068
:101300002E4A3C32914201D11A4600E022462D4934
:101310004A60012180F82110002180F82010416BE3
:1013200001B188472846BDE8F09F2DE9F74F82B00C
:101330000446154694F82100022808D00420A06332
:10134000002084F82000012005B0BDE8F08F20685F
:101350000168890604D54FF48070A0630120F3E78B
:10136000184FDFF86080DFF85C90DFF858A0DFF8F6
:1013700054B003991C3708F1300809F144090AF107
:10138000580A0BF16C0B29B10E490831884245D13E
:1013900004267AE00B490831884201D1022674E024
:1013A000B84201D1202670E0404502D14FF40076CA
:1013B0006BE0484508D14FF4005666E0080402404F
:1013C000F8FFFDBF00000240504502D14FF4003647
:1013D0005BE0584502D14FF4001656E0F7498842C9
:1013E00001D1860451E0F649884201D102264CE041
:1013F000F3491431884201D1202646E0F0492831D2
:10140000884201D1461540E0ED493C31884202D185
:101410004FF4005639E04FF4003636E0B84201D1BF
:10142000402632E0404502D14FF480662DE0484529
:1014300002D14FF4804628E0504502D14FF4802677
:1014400023E0584502D14FF480061EE0DB49884274
:1014500001D1C60419E0DA49884201D1042614E01A
:10146000D7491431884201D140260EE0D4492831B1
:10147000884201D1061508E0D1493C31884202D1A9
:101480004FF4804601E04FF4802601F0CAFF01903E
:10149000A5E090423CD9CA4908390968C74A783A58
:1014A000904201D1082031E0B84201D180202DE0E6
:1014B000404502D14FF4006028E0484502D14FF486
:1014C000004023E0504502D14FF400201EE0584573
:1014D00002D14FF4000019E0B94A904201D108202E
:1014E00014E0B74A1432904201D180200EE0B44A91
:1014F0002832904201D1C01408E0B14A3C329042F7
:1015000002D14FF4004001E04FF40020014040E0E0
:10151000AA4980390968A94B783B984201D1082033
:1015200036E0B84201D1802032E0404502D14FF48C
:1015300000602DE0484502D14FF4004028E05045BE
:1015400002D14FF4002023E0584502D14FF40000AF
:101550001EE0904202D14FF0006019E0984A90429C
:1015600001D1082014E0964A1432904201D1802023
:101570000EE0934A2832904201D1C01408E0904A0C
:101580003C32904202D14FF4004001E04FF4002081
:10159000014081B12034012294F8201002FA01F0B8
:1015A000E1694860A16941F00101A1616270002018
:1015B00020700120C8E6681C11D02DB101F031FF68
:1015C0000199401AA8420AD92034A06940F02000AD
:1015D000A06101206070002020700120B4E6774AED
:1015E0002068904204D9764908390968314003E0FF
:1015F000724980390968314000293FF44AAF704B85
:1016000003991B1F49B16D4A2168914271D96B49F9
:10161000783988426ED10420B5E0684922688A4250
:1016200039D966497839884201D1022031E0B8427F
:1016300001D120202DE0404502D14FF4007028E078
:10164000484502D14FF4005023E0504502D14FF4F9
:1016500000301EE0584502D14FF4001019E05849FF
:10166000884201D1022014E055491431884201D149
:1016700020200EE052492831884201D1401508E06F
:101680004F493C31884202D14FF4005001E04FF401
:101690000030186041E0494A783A904201D1022076
:1016A00038E0B84201D1202034E0404502D14FF467
:1016B00000702FE0484502D14FF400502AE0504519
:1016C00002D14FF4003025E0584502D14FF400100C
:1016D00020E0884202D14FF000701BE03849884278
:1016E00001D1022016E036491431884203D120206E
:1016F00010E04AE015E032492831884201D1401516
:1017000008E02F493C31884202D14FF4005001E0FB
:101710004FF40030294980394860012084F82100C5
:1017200076E0B84201D140202DE0404502D14FF48F
:10173000806028E0484502D14FF4804023E05045C6
:1017400002D14FF480201EE0584502D14FF48000B2
:1017500019E01B49884201D1042014E018491431D2
:10176000884201D140200EE015492831884201D13C
:10177000001508E012493C31884202D14FF4804004
:1017800001E04FF48020186042E00C49783988422B
:1017900001D104203AE0B84201D1402036E0404572
:1017A00002D14FF4806031E0484502D14FF48040CF
:1017B0002CE0504506D14FF4802027E08000024005
:1017C00008040240584502D14FF480001EE09042C8
:1017D00002D14FF0806019E0D949884201D104203C
:1017E00014E0D7491431884201D140200EE0D44999
:1017F0002831884201D1001508E0D1493C318842A6
:1018000002D14FF4804001E04FF48020CD49486080
:10181000002084F8200097E52DE9F05FC16B0A688D
:1018200001680B68046C4FF0040E0EFA04FEC64DFE
:10183000C64EC74FDFF81CC3DFF81C83DFF81C93CC
:10184000DFF8FCA2DFF818B31EEA020F7AD05FEAD5
:10185000437E77D50A68920603D40A6822F0040210
:101860000A60DFF8F8E24FF4806201680EF1140EAE
:101870001301140271452DD9A94201D1042225E09A
:10188000B14201D1402221E0B9421FD0614501D1CE
:101890001A461BE0414501D1224617E0494502D1D5
:1018A0004FF4800212E0514501D104220EE0594567
:1018B00001D140220AE0AA4D1435A94206D0A84A17
:1018C0002832914201D11A4600E022469C49091F64
:1018D0000A6031E0A94201D104222BE0B14201D1DA
:1018E000402227E0B94225D0614501D11A4621E0C6
:1018F000414501D122461DE0494502D14FF4800205
:1019000018E0714502D14FF0806213E0514501D1DA
:1019100004220FE0594501D140220BE0904D1435CF
:10192000A94207D08E4A2832914202D11A4601E0DC
:1019300008E0224683494A60C16A00296FD0BDE8A9
:10194000F05F08474FF0020E0EFA04FE1EEA020F87
:1019500074D05FEA837E7ED50A68920606D40A6850
:1019600022F00A020A60012180F82110DFF8ECE180
:101970004FF4007201680EF1140E13011402714548
:101980002DD9A94201D1022225E0B14201D1202264
:1019900021E0B9421FD0614501D11A461BE0414503
:1019A00001D1224617E0494502D14FF4001212E05E
:1019B000514501D102220EE0594501D120220AE011
:1019C000674D1435A94206D0654A2832914201D1AB
:1019D0001A4600E022465A49091F0A6032E0A9422D
:1019E00001D102222CE0B14201D1202228E0B942EB
:1019F00026D0614501D11A4622E0414501D1224657
:101A00001EE0494502D14FF4001219E0714502D1A0
:101A10004FF0007214E0514502D1022210E037E08D
:101A2000594501D120220BE04D4D1435A94207D074
:101A30004B4A2832914202D11A4601E00BE022467D
:101A400040494A60002180F82010816A00291FD097
:101A5000BDE8F05F08470825A540154218D01A07D1
:101A600016D50A6822F00E020A6090F84020C36B77
:101A7000012101FA02F25A60816380F821100021ED
:101A800080F82010016B002902D0BDE8F05F084704
:101A900049E410B5002390F82040012C0CD001241B
:101AA00080F8204090F82140012C07D0012300212C
:101AB00080F82010184610BD022010BD39B1012950
:101AC00007D0022907D0032907D00123EFE782625C
:101AD000EDE7C262EBE70263E9E74263E7E710B5CF
:101AE000002290F82030012B0CD0012380F8203008
:101AF00090F821400023012C06D0012280F82030EC
:101B0000104610BD022010BD052911D2DFE801F0FA
:101B1000030507090B008362F0E7C362EEE7036386
:101B2000ECE74363EAE78362C36203634363E5E789
:101B30000122E3E790F821007047806B70470000B6
:101B40000804024000000240080002401C0002405D
:101B50003000024044000240580002406C00024045
:101B60001C04024000F00701744A10684FF6FF039E
:101B7000184040EA01207249084310607047F0B4F1
:101B80000D466E4B1B68C3F30223C3F10704042CFC
:101B900000D90424191D072901D2002300E0DB1E0F
:101BA000012606FA04F1491E294099409E40761EFE
:101BB00016403143F0BC00F0B1B800F01F02012123
:101BC00091404009800000F1E020C0F8001170470A
:101BD00000F01F02012191404009800000F1E02047
:101BE000C0F880117047BFF34F8F54480168544AC2
:101BF00001F4E061121D11430160BFF34F8F00BF7C
:101C0000FDE710B5401EB0F1807F01D3012010BD6B
:101C10004FF0E02460610F21601700F07FF8002092
:101C2000A06107202061002010BD44480068C0F377
:101C300002207047F0B5002807DA00F00F0000F12D
:101C4000E02090F8140D040904E000F1E02090F881
:101C50000004040901F00700C0F10701042900D9BC
:101C60000421051D072D01D2002000E0C01E012720
:101C700024FA00F607FA01F56D1E2E40166007FAE9
:101C800000F56D1E25401D60F0BD00F01F02012112
:101C900091404009800000F1E020C0F80012704738
:101CA0004109890001F1E021D1F8001200F01F0282
:101CB00001209040014201D0012070470020704770
:101CC00000F01F02012191404009800000F1E02056
:101CD000C0F8801270474109890001F1E021D1F874
:101CE000001300F01F0201209040014201D00120AA
:101CF0007047002070474FF0E021042804D00869A5
:101D000020F0040008617047086940F00400086191
:101D10007047704710B5FFF7FCFF10BD0907090EAB
:101D2000002806DA00F00F0000F1E02080F8141D12
:101D3000704700F1E02080F8001470470CED00E0DF
:101D40000000FA05F948416821F00301416001688B
:101D5000F74A11400160016821F4802101600021EF
:101D60004160026822F0F80242F080020260816065
:101D7000F149F0480860704708B5EF494FF4FA524E
:101D80000968B1FBF2F14143009100BF0098411E88
:101D90000091FAD208BD2DE9F84F0446E34D2078B2
:101DA000C0075BD06868C0F38100012807D068686D
:101DB000C0F3810002280AD16868C00307D52868EB
:101DC00080034BD5606878BB0120BDE8F88F606860
:101DD000B0F5803F11D0A8B1B0F5A02F1BD0286876
:101DE00020F480302860286820F480202860606813
:101DF00030B301F016FB06461EE0286840F4803040
:101E00002860F4E7286820F480302860286820F4EF
:101E100080202860EBE7286840F48020286028684C
:101E200040F480302860E2E718E001F0FAFA801B05
:101E3000642801D90320C8E728688003F5D50DE0A0
:101E400001F0EFFA064606E001F0EBFA801B642889
:101E500001D90320B9E728688003F5D42078DFF89A
:101E6000DC8280074FF0010A4FF0000945D5686811
:101E700010F00C0F07D06868C0F38100022812D15F
:101E80006868C0030FD42868800704D5206901283A
:101E900001D0012099E72868616920F0F80040EA44
:101EA000C100286029E02069B8B1C8F800A001F09D
:101EB000B8FA064606E001F0B4FA801B022801D900
:101EC000032082E728688007F5D52868616920F03B
:101ED000F80040EAC10028600FE0C8F8009001F067
:101EE000A0FA064606E001F09CFA801B022801D900
:101EF00003206AE728688007F5D42078000726D5F4
:101F00008F48A16999B1C0F800A001F08AFA06468D
:101F100006E001F086FA801B022801D9032054E76D
:101F2000686A8007F5D50120FFF726FF0FE0C0F8AB
:101F3000009001F076FA064606E001F072FA801B86
:101F4000022801D9032040E7686A8007F5D4207889
:101F5000400773D50026E869C00008D4E86940F05E
:101F60008050E861E86900F0805000900126DFF8B9
:101F7000D4B1DBF80000C00514D4DBF8000040F455
:101F80008070CBF8000001F04CFA074606E001F043
:101F900048FAC01B642801D9032016E7DBF80000CB
:101FA000C005F4D5E068012812D0B0B105281DD0D5
:101FB000286A20F001002862286A20F004002862C4
:101FC000E06841F2883B28B301F02BFA07461DE098
:101FD000286A40F001002862F2E7286A20F0010038
:101FE0002862286A20F004002862E9E7286A40F0A5
:101FF00004002862286A40F001002862E0E701F04E
:1020000010FAC01B584501D90320DEE6286A800774
:10201000F5D50DE001F005FA074606E001F001FAFA
:10202000C01B584501D90320CFE6286A8007F5D4A4
:10203000012E03D1E86920F08050E861E069A0B387
:102040006968C1F38101022947D0022805D0C8F888
:10205000609001F0E6F904463AE0C8F8609001F0BB
:10206000E0F9064606E001F0DCF9801B022801D900
:102070000320AAE628688001F5D4206AB0F5803FE5
:1020800005D16868A16820F4003008436860D4E98D
:1020900008010843696821F4741108436860C8F8AE
:1020A00060A001F0BEF9044607E014E001F0B9F9C0
:1020B000001B022801D9032087E628688001F5D596
:1020C00009E001F0AEF9001B022801D903207CE6EB
:1020D00028688001F5D4002077E6012075E610B568
:1020E00085B019A0D0E901130268C068CDE90213D8
:1020F0000192049018A0006800900C4B59680D489C
:1021000001F00C02042A0FD0082A0DD101AAC1F354
:102110008344125DC90321D55968C1F340411DF8BC
:102120000110B0FBF1F0504305B010BD00100240AB
:10213000FFFFF6FE00127A00040100200000424278
:1021400080044242007000400203040506070809AB
:102150000A0B0C0D0E0F101001020000AC4850438A
:10216000E2E72DE9F04704460E46DFF8A882D8F8EA
:10217000000000F00700B0420FD2D8F8000020F0B5
:1021800007003043C8F80000D8F8000000F007004E
:10219000B04202D00120BDE8F08720789E4F800732
:1021A00005D57868A16820F0F000084378602078B1
:1021B000C00748D06068012806D0022809D03968D5
:1021C00089070BD40120E6E73968890306D401208A
:1021D000E1E73968890101D40120DCE7796821F061
:1021E00003010143796001F01CF90546606841F282
:1021F0008839012809D0022814D020E001F011F913
:10220000401B484501D90320C5E77868C0F3810029
:102210000128F3D117E001F004F9401B484501D92A
:102220000320B8E77868C0F381000228F3D10AE000
:1022300001F0F7F8401B484501D90320ABE7786867
:1022400010F00C0FF4D1D8F8000000F00700B042F5
:102250000ED9D8F8000020F007003043C8F800007D
:10226000D8F8000000F00700B04201D0012092E74A
:102270002078400705D57868E16820F4E0600843DD
:1022800078602078000706D57868216920F46050CE
:1022900040EAC1007860FFF722FF79685F4AC1F326
:1022A0000311515CC8405E4908600F2001F085F8B9
:1022B000002070E730B585B00D4600200390022065
:1022C0000290032004904FF480700190524CA0695A
:1022D00040F00400A061A06900F00400009001A992
:1022E0005048FEF7CDFC606820F0E0602843606055
:1022F00005B030BD4C490120C86470474A490020F0
:10230000C864704746480068704700B5FFF7FAFF99
:1023100041494968454AC1F30221515CC84000BDAA
:1023200000B5FFF7EFFF3C494968404AC1F3C221BD
:10233000515CC84000BD10B50F210160364B1968D3
:102340004A034FF0000103D54FF4A022426007E09A
:102350001A68D20303D54FF48032426000E0416036
:102360005A6802F4003282601A68D4074FF0010202
:1023700001D0026100E001611C68C4F3C40444613F
:102380001C6A640702D50524C46005E01C6AE407E2
:1023900001D0C26000E0C1605C6AE40701D08261E4
:1023A00000E081611968C90102D50221C16100E024
:1023B000C261596801F480310162596801F47011F9
:1023C0004162B2E60F220260134A536803F003032E
:1023D0004360536803F0F0038360536803F4E063E1
:1023E000C360526802F46052D20802610948006872
:1023F00000F0070008607047704710B5064CA068F1
:10240000000603D5FFF7F8FF8020A0728DE60000DC
:1024100000093D000020024000100240CCC6000828
:10242000040100200008014000004242DCC6000810
:102430002DE9F041044620680169E26821F4405129
:1024400011430161A168206901436069014320686B
:10245000C26841F20C639A430A43C2602068416932
:10246000A26921F4407111434161FE49206864254D
:102470003226884254D1FFF753FF00EBC00101EB35
:10248000001061688900B0FBF1F7FFF749FF00EB2E
:10249000C00101EB001061688900B0FBF1F0B0FBF6
:1024A000F5F06FF01801484307EB800006EB0010D1
:1024B000B0FBF5F000F0F007FFF732FF00EBC001D2
:1024C00001EB001061688900B0FBF1F0B0FBF5F0A2
:1024D00007EB0017FFF724FF00EBC00101EB001032
:1024E00061688900B0FBF1F8FFF71AFF00EBC0014B
:1024F00001EB001061688900B0FBF1F0B0FBF5F072
:102500006FF01801484308EB800006EB0010B0FBA9
:10251000F5F0216800F00F0038448860BDE8F081D4
:10252000FFF7F3FE00EBC00101EB001061688900CA
:10253000B0FBF1F7FFF7E9FE00EBC00101EB001083
:1025400061688900B0FBF1F0B0FBF5F06FF01801A5
:10255000484307EB800006EB0010B0FBF5F000F0FD
:10256000F007FFF7D2FE00EBC00101EB001061683D
:102570008900B0FBF1F0B0FBF5F007EB0017FFF7B7
:10258000C4FE00EBC00101EB001061688900B0FBE4
:10259000F1F8FFF7BAFE00EBC00101EB0010616833
:1025A0008900B0FBF1F0B0FBF5F06FF01801484383
:1025B00008EB800006EB0010B0FBF5F0216800F09E
:1025C0000F0038448860A9E7704770B50446002CB6
:1025D00004D094F83900002510B106E0012070BD48
:1025E00084F838502046FEF7E6F9242084F83900B4
:1025F0002068C16821F40051C1602046FFF718FF30
:102600002068016921F4904101612068416921F04D
:102610002A0141612068C16841F40051C160E5634D
:10262000202084F8390084F83A00002070BD70B58D
:102630000446002C04D094F83900002510B106E0BF
:10264000012070BD84F838502046FEF7B4F92420EC
:1026500084F839002068C16821F40051C160204627
:10266000FFF7E6FE2068016921F4904101612068CE
:10267000416921F0220141612068416941F008016E
:1026800041612068C16841F40051C160E5632020C8
:1026900084F8390084F83A00002070BD70B5044613
:1026A0000E46002C04D094F83900002510B106E045
:1026B000012070BD84F838502046FEF77CF92420B4
:1026C00084F839002068C16821F40051C1602046B7
:1026D000FFF7AEFE2068016921F400610161206806
:1026E000416921F02A0141612068016941F480417A
:1026F00001612068016921F02001314301612068F6
:10270000C16841F40051C160E563202084F83900BC
:1027100084F83A00002070BD2DE9F04104460F46D0
:102720001646002C04D094F83900002510B106E0BC
:102730000120F3E684F838502046FEF73CF92420C7
:1027400084F839002068C16821F40051C160204636
:10275000FFF76EFE2068016921F490410161206855
:10276000416921F02A0141612068016921F00F01CE
:10277000394301612068C16821F400613143C160BF
:102780002068C16841F40051C160E563202084F8ED
:10279000390084F83A000020C0E6704710B50446BE
:1027A000002C0CD0242084F839002046FEF790F944
:1027B0000020383460606070A070207010BD01206F
:1027C00010BD2DE9F04104460E4617469846069D79
:1027D0001CE0681C1AD02DB100F023FEA0EB08000D
:1027E000A84213D92068C16821F4D071C160206863
:1027F000416921F001014161202084F8390084F809
:102800003A00002084F83800032087E6206800683A
:1028100036EA000004D00020B842DAD000207DE67D
:102820000120F9E72DE9F84304460D4691461E467E
:1028300094F83900202802D00220BDE8F883CDB1F9
:10284000B9F1000F16D094F83800012814D00120F7
:1028500084F838000027E763212084F8390000F06D
:10286000E0FD01E0003801408046A4F82490A4F87F
:1028700026902DE00120E0E70220DEE7E08C401EFC
:10288000E084A068B0F5805F09D043460022802133
:1028900020460096FFF795FFB0B10320CDE74346F1
:1028A0000022802120460096FFF78BFF08B103200D
:1028B000C3E728882168C0F308004860206908B190
:1028C0006D1C05E0AD1C03E0216815F8010B4860A4
:1028D000E08C0028D2D143460022402120460096B9
:1028E000FFF76FFF08B10320A7E72020383460709E
:1028F00027700020A1E72DE9F84304460D469146D4
:102900001E4694F83A00202801D0022095E7B5B180
:10291000B9F1000F13D094F83800012811D001202C
:1029200084F838000027E763222084F83A0000F09A
:1029300078FD8046A4F82C90A4F82E9035E0012074
:102940007BE7022079E7E08D401EE085A068B0F5C6
:10295000805F09D043460022202120460096FFF7E1
:1029600030FFD0B1032068E74346002220212046F3
:102970000096FFF726FF08B103205EE7206928B123
:1029800020684068C1B229806D1C0EE02068406854
:10299000C0F308012980AD1C07E0206970B12068F0
:1029A000406800F07F0005F8010BE08D0028CAD1D7
:1029B00020203834A070277000203EE7206840684F
:1029C00005F8010BF1E790F83930202B01D00220F7
:1029D0007047A9B1A2B190F83830012B12D0016232
:1029E0008284C2840021C163212280F8392080F8CA
:1029F00038100068C16841F08001C1600020704754
:102A0000012070470220704790F83A30202B01D007
:102A100002207047F9B1F2B190F83830012B1CD088
:102A200081628285C2850021C163222280F83A201A
:102A300080F838100168CA6842F48072CA60016880
:102A40004A6942F001024A610068C16841F0200110
:102A5000C160002070470120704702207047704716
:102A60000168CA6822F49072CA6001684A6922F05B
:102A700001024A61202180F83A1070470168CA6853
:102A800022F0C002CA60202180F83910704770B56A
:102A9000446A20684069C0F3C01094F839100025DA
:102AA000212904D118B1E5842046FFF7E7FF20680B
:102AB0004069C0F3801094F83A10222904D118B16B
:102AC000E5852046FFF7CCFFE06B40F01000E063A7
:102AD0002046FFF7C4FF70BD704710B5406AFFF78E
:102AE000FBFF10BD704710B50146486A09680968C8
:102AF00089060CD40021C18401684A6922F0800251
:102B00004A610068C16841F04001C16010BDFFF733
:102B1000E9FF10BDF7B5044694F83900202801D02C
:102B20000220FEBD019979B372B394F838000128F0
:102B30002DD0012084F838002162A284E28400258F
:102B4000E563212084F83900236BF8489862236BF1
:102B5000F748D862236BF7481863206B45632068F9
:102B60001346001D266B02463046FEF7E8FA216840
:102B70006FF04000086084F838502068416941F0E7
:102B8000800141610020FEBDFFE70120FBE702203C
:102B9000F9E7704710B5406AFFF7FBFF10BD7047BB
:102BA00010B50146486A09680968890613D40021EE
:102BB000C1850168CA6822F48072CA6001684A69E6
:102BC00022F001024A6101684A6922F040024A612A
:102BD000202180F83A10FFF7E2FF10BD37B582B030
:102BE0000446134694F83A00202802D0022005B08B
:102BF00030BD039AA2B39BB394F83800012832D0B9
:102C0000012084F83800A262A3850025E563222014
:102C100084F83A00616BC8488862616BC748C86233
:102C2000616BC4480863606B45632168606B091D74
:102C3000FEF785FA206801684168019184F83850F0
:102C4000C16841F48071C1602068416941F00101AF
:102C500041612068416941F0400141610020C6E7BF
:102C6000FFE70120C3E70220C1E790F838100129EF
:102C70000BD0012180F8381001684A69C2F3C012F4
:102C800090F83930212B02D006E0022070471AB1AB
:102C90004A6922F080024A6101684A69C2F38012DF
:102CA00090F83A30222B0ED16AB1CA6822F48072B1
:102CB000CA6001684A6922F001024A6101684A69F2
:102CC00022F040024A61002180F83810002070474D
:102CD00008B590F83810012907D0012180F8381084
:102CE00090F83910212902D006E0022008BD0168C1
:102CF0004A6942F080024A6190F83A100022222983
:102D000011D101680B684B680093CB6843F4807362
:102D1000CB6001684B6943F001034B6101684B696B
:102D200043F040034B6180F83820002008BD10B507
:102D3000044620684169C1F3C01194F83920212A62
:102D40000BD151B1416921F080014161206B08B183
:102D5000FEF72FFA2046FFF791FE20684169C1F384
:102D6000801194F83A20222A0BD151B1416921F007
:102D700040014161606B08B1FEF71BFA2046FFF786
:102D80006FFE002010BD70B504462068C16821F4B4
:102D9000F071C1602068416921F001014161206842
:102DA00041694FF00005090609D5416921F080010C
:102DB0004161206B18B14563206BFEF7FAF920687A
:102DC0004169490609D5416921F040014161606BC3
:102DD00018B14563606BFEF7ECF9E584E585E563C2
:102DE000202084F83A0084F83900002070BD70B5C6
:102DF00004462068C16821F0C001C16020684169B3
:102E00004FF00005090609D5416921F080014161B3
:102E1000206B18B14563206BFEF7CBF9E5842020C9
:102E200084F83900002070BD70B504462068C16880
:102E300021F49071C1602068416921F00101416174
:102E4000206841694FF00005490609D5416921F024
:102E500040014161606B18B14563606BFEF7A9F9F1
:102E6000E585202084F83A00002070BD704710B539
:102E7000406A0022416B4A63016B002902D0496B12
:102E8000002909D1C284C285C263202180F839108B
:102E900080F83A10FFF7EAFF10BD10B5406A002233
:102EA000016B4A63416B002902D0496B002909D1AB
:102EB000C284C285C263202180F8391080F83A109C
:102EC000FFF7D4FF10BD70B5044601252068C16826
:102ED00021F4F071C1602068416921F00101416174
:102EE000206B0026002807D021684969090602D511
:102EF0001349416300E04663606B38B1216849695A
:102F0000490602D50F49416300E0466320684169E4
:102F100009061AD5416921F080014161206BA0B1F9
:102F2000FEF75FF980B1206B46630EE0E72A0008E8
:102F3000DB2A00088F2A0008A12B0008952B000827
:102F40009B2E00086F2E0008002520684169490665
:102F50000DD5416921F040014161606B38B1FEF748
:102F600040F918B1606B4663012500E00025012D92
:102F70000AD1E684E685E663202084F8390084F8E7
:102F80003A002046FFF772FF002070BD704710B571
:102F9000406A0021C184202180F83910FFF7F6FF34
:102FA00010BD10B504462068C16821F0C001C160A1
:102FB000206841694FF020020B064FF0000116D542
:102FC000436923F080034361206B48B1F7494163B3
:102FD000206BFEF706F980B1206B416B88470CE04F
:102FE000E18484F839202046FFF7D0FF05E0E18432
:102FF00084F839202046FFF7C9FF002010BD704734
:1030000010B5406A0021C185202180F83A10FFF7F1
:10301000F6FF10BD10B504462068C16821F4907118
:10302000C1602068416921F0010141612068416966
:103030004FF000024B064FF0200116D5436923F0F4
:1030400040034361606B48B1D9494163606BFEF74F
:10305000C8F880B1606B416B88470CE0E28584F86A
:103060003A102046FFF7CBFF05E0E28584F83A10DE
:103070002046FFF7C4FF002010BD10B50168CA68E4
:1030800022F04002CA60202180F83910FFF72AFDA3
:10309000002010BD90F83910212901D0022070477E
:1030A0008168B1F5805F0CD0016A4A1C0262026837
:1030B00009785160C18C491E0904090CC18410D0E3
:1030C00019E0016A02680988C1F3080151600169C9
:1030D00019B1016A491C0162ECE7016A891C0162AD
:1030E000E8E70168CA6822F08002CA600068C16827
:1030F00041F04001C1600020704710B5406A0021D6
:10310000C185C184FFF7ABFC10BD10B590F83A1033
:10311000222901D0022010BD8168B1F5805F11D055
:10312000016919B30168496801F07F03816A4A1C8B
:1031300082620B70C18D491E0904090CC1851CD027
:10314000002010BD816A02693AB102685268D2B2A9
:103150000A80816A491C8162ECE702685268C2F306
:1031600008020A80816A891C8162E3E701684A6873
:10317000816A4B1C83620A70DCE70168CA6822F02E
:103180002002CA600168CA6822F48072CA600168BD
:103190004A6922F001024A61202180F83A10FFF7C3
:1031A000FEFC002010BD70B5044622681068D1688E
:1031B000526900F00F03002B07D1850605D58D0657
:1031C00003D52046BDE870409FE7002B5ED002F09B
:1031D000010301F490752B4358D0C30705D0CB05EC
:1031E00003D5E36B43F00103E363430705D5D3073E
:1031F00003D0E36B43F00203E363830705D5D307F2
:1032000003D0E36B43F00403E363030705D5D20760
:1032100003D0E26B42F00802E263E26B002A2AD09C
:10322000800604D5880602D52046FFF76EFF206889
:103230004069C0F38010E16B090700D400B3204659
:10324000FFF70EFC20684169490615D5416921F058
:1032500040014161606B58B156494163606BFDF7B5
:10326000C0FF002807D0606B416BBDE87040084785
:103270002046FFF7F4FB70BD2046FFF7F0FB70BD62
:103280002046FFF7ECFB0020E06370BD020605D589
:103290000A0603D52046BDE87040FBE64006F4D59B
:1032A0004806F2D52046BDE87040E6E690F83810B2
:1032B000012910D0012100F8381F2421417050F855
:1032C000381CCA6842F00102CA6020214170002106
:1032D0000170002070470220704790F838100129D3
:1032E00010D0012100F8381F2421417050F8381CFB
:1032F000CA6842F00202CA602021417000210170B8
:10330000002070470220704790F83810012910D033
:10331000012100F8381F2421417050F8381CCA6878
:1033200022F00202CA6020214170002101700020B9
:1033300070470220704790F83810012912D00121FF
:1033400000F8381F2421417050F8381CCA6822F058
:103350000C0242F00802CA60202141700021017075
:10336000002070470220704790F83810012912D0D1
:10337000012100F8381F2421417050F8381CCA6818
:1033800022F00C0242F00402CA60202141700021A8
:1033900001700020704702207047014611F8390F74
:1033A000497808437047C06B704700008F2F0008B2
:1033B00001300008FB300008704710B5044646484D
:1033C0004FF47A720068B0FBF2F0FEF71AFC0022AC
:1033D0002146501EFEF7D3FB002010BD10B53F481C
:1033E000016841F0100101600320FEF7BBFB0F20D4
:1033F000FFF7E3FFFCF7F0FE002010BD704710B5AB
:1034000037484FF0FF31C16000220261C160C260E5
:10341000FFF7F4FF002010BD32480168491C01602D
:10342000704730480068704731B5FFF7FAFF05462E
:10343000009C601C00D0641CFFF7F3FF401BA042FF
:10344000FAD338BD4FF0E020016921F0020101619B
:1034500070474FF0E020016941F0020101617047BF
:103460002148704721480068000C70471F480068D9
:10347000C0F30B0070471D48416841F001014160F5
:1034800070471A48416821F00101416070471748B0
:10349000416841F00201416070471448416821F0E1
:1034A0000201416070471148416841F004014160E8
:1034B00070470E48416821F00401416070470C4993
:1034C000096801600A49091D096841600849083115
:1034D000096881607047000004010020002002405C
:1034E000001002400801002000010101002004E05A
:1034F000E8F7FF1F0648804706480047FEE7FEE75B
:10350000FEE7FEE7FEE7FEE7FEE7FEE7FEE7FEE793
:10351000C10B000831010008704718480068704767
:1035200010B5044605F048FA14490C60BDE8104097
:1035300005F046BA10B511490868401C086004F04F
:1035400095FCC16D491EC16519B9816DC16504F055
:1035500025FEBDE8104004F0D8BA002802DA4FF08A
:10356000FF30704700EBC00101EB001040F2E73183
:1035700001EB8000491C90FBF1F070470C0100202A
:1035800000207047002070470020704700207047DF
:1035900070B5284C284D02E020688047241DAC42BD
:1035A000FAD370BD70B5244C244D02E020688047EA
:1035B000241DAC42FAD370BD10B5FFF7F3FFBDE890
:1035C0001040FCF7C2BD1CB514200A21CDE9001043
:1035D0004FF400630022AFF21F0119A004F0F6FCC3
:1035E000044624B9D422184918A002F0C6FC20468B
:1035F000BDE81C4004F074BC10B505F0DDF9FCF723
:103600006EFE02F01EFC04F0BEFA03F01EFD04F094
:1036100077F8FFF7D8FF04F0C1FA00F04BFB03F096
:103620002AFD002010BD10B505F0C6F9FFF7E4FF34
:10363000002010BDFCDA000808DB000810DB0008E1
:103640006D61696E00000000E4C6000874696420C2
:10365000213D2052545F4E554C4C00002DE9F04165
:10366000074604F003FC08B103F0B1FD082003F0A5
:1036700037FB054625B98A22FD49FEA002F07DFCF4
:103680006C682D1D08E0A4F10C060822394630466E
:1036900002F0A2F950B12468AC42F4D104F0E6FB88
:1036A00008B103F09FFD0020BDE8F08104F0DEFBCF
:1036B00008B103F097FD3046F6E72DE9F0410446E6
:1036C0000F4615464FF0FF36002C05D03846FFF761
:1036D000C5FF18B13046E7E73046E5E73A4608212E
:1036E000204603F00DFBE5820020A0762083DBE777
:1036F00010B50446002C05D1DD4960221539E3A040
:1037000002F03BFC204603F0CDFB082805D0D84949
:1037100061221539E1A002F030FC204603F0B0FB35
:1037200028B9D34962221539EBA002F026FC2046C5
:1037300003F010FB002010BD0020704770B5054657
:10374000C91C21F00300403002F03DFD04462CB1BD
:1037500040220021204602F07FF82575204670BDEA
:1037600010B50446002C05D1C149C8220F31C7A0AD
:1037700002F003FC204603F095FB082805D0BC4965
:10378000C9220F31C5A002F0F8FB204603F078FBF8
:1037900028B1B749CA220F31D9A002F0EEFB20466A
:1037A00003F0D8FA2046BDE8104002F0D2BD70B553
:1037B00004460025002C05D1AD49DF222131B3A0FC
:1037C00002F0DBFB616A81B1A07DC0060DD420460A
:1037D000884705462DB12A462146D6A002F010FBA7
:1037E00003E0E08A40F01000E082284670BD70B52A
:1037F00004460E460025002C06D19D494FF48172E7
:103800003031A2A002F0B9FB204603F04BFB0828A0
:1038100006D0974940F203123031A0A002F0ADFB70
:10382000A07DC00611D4616A59B12046884705467B
:10383000280006D02A462146BEA002F0E1FA28461A
:1038400070BDE08A40F01000E082A07D000705D541
:10385000207E000702D56FF0060070BDA26A22B17B
:10386000314620469047054603E040F60F7006407B
:1038700026830DB1A81D0FD1208B40F008002083B6
:10388000A07E401CC0B2A07630B9794940F2311216
:103890003031B6A002F071FB284670BD70B5044609
:1038A0000025002C06D1724940F243123F3177A027
:1038B00002F063FB204603F0F5FA082806D06C49B5
:1038C0004FF4A2723F3175A002F057FBA07E28B1E1
:1038D000401EC0B2A07620B1002070BD4FF0FF3076
:1038E00070BDE16A11B12046884705460DB1A81D9B
:1038F00001D100202083284670BD2DE9F041044607
:103900000E4617469846002C06D1594940F26D12D2
:103910004F315EA002F031FB204603F0C3FA0828C5
:1039200006D053494FF4B7724F315CA002F025FB2B
:10393000A07E48B1256B6DB143463A4631462046DC
:10394000AC46BDE8F04160474FF0FF3001F066FF44
:103950000020A9E66FF0050001F060FF0020A3E65B
:103960002DE9F04104460E4617469846002C06D134
:103970003F494FF4CA725E3144A002F0FEFA20467D
:1039800003F090FA082806D0394940F295125E31CA
:1039900042A002F0F2FAA07E48B1656B6DB14346D9
:1039A0003A4631462046AC46BDE8F04160474FF00C
:1039B000FF3001F033FF002076E66FF0050001F0E4
:1039C0002DFF002070E670B504460D461646002C0B
:1039D00006D1274940F2B5126E312CA002F0CDFA83
:1039E000204603F05FFA082806D021494FF4DB7225
:1039F0006E312AA002F0C1FAA36B2BB132462946E0
:103A00002046BDE8704018476FF0050070BD70B5E6
:103A100004460D46002C06D1154940F2CF128031E4
:103A20001AA002F0AAFA204603F03CFA082806D0B1
:103A30000F494FF4E872803118A002F09EFAE56158
:103A4000002070BD70B504460D46002C06D1084913
:103A500040F2E5129A310DA002F08FFA204603F0F1
:103A600021FA082802D04FF4F37289E08DE00000BB
:103A70000DC70008696E666F726D6174696F6E20A4
:103A8000213D2052545F4E554C4C00006465762019
:103A9000213D2052545F4E554C4C000072745F6FB4
:103AA000626A6563745F6765745F74797065282600
:103AB0006465762D3E706172656E7429203D3D20EF
:103AC00052545F4F626A6563745F436C6173735FE6
:103AD000446576696365000072745F6F626A65634E
:103AE000745F69735F73797374656D6F626A656320
:103AF0007428266465762D3E706172656E742900A7
:103B000072745F6F626A6563745F69735F73797300
:103B100074656D6F626A65637428266465762D3EF0
:103B2000706172656E7429203D3D2052545F46419C
:103B30004C534500546F20696E697469616C697AF1
:103B400065206465766963653A2573206661696CF2
:103B500065642E20546865206572726F7220636FF1
:103B600064652069732025640A0000006465762D71
:103B70003E7265665F636F756E7420213D20300074
:103B80000349AFF2E80002F0F8F92562002070BDA9
:103B9000A7C7000870B505466FF0020404F00CFFDB
:103BA00003460021544A52F8210038B1491C042927
:103BB000F9D3184604F004FF204670BD42F82150A6
:103BC0000024F6E770B504466FF0050504F0F4FE36
:103BD00003460021484850F82120A24204D1002287
:103BE00040F82120002502E0491C0429F3D318469F
:103BF00004F0E6FE284670BD70B53DE004F0DCFE42
:103C0000044601F0F7FD40B13C493DA002F0F8F850
:103C1000A7223A4944A002F0B0F9204604F0D0FEB1
:103C200004F0CAFE064600F05FF888B33F48046817
:103C3000A4F11405D4E900104860D4E9000108603B
:103C40006460246003F0C3FAD5F88C1009B12846EB
:103C50008847284603F0D5FC284603F011F90128CF
:103C60000FD003F0BFFA304604F0AAFEA86A02F0B3
:103C700070FB284603F0D9F800F036F80028BDD1D3
:103C800070BD03F0AFFA3046BDE8704004F098BE56
:103C90003046BDE8704004F093BE174D08E055F87B
:103CA000240000B18047641C042CF8D3FFF7A4FF64
:103CB0000024F4E71FB52020C2001F211C4BCDE9D2
:103CC0000210CDE900321A4800231A4A1AA194388A
:103CD00004F0A1F804B01648BDE81040943804F090
:103CE000FFB813489438704710480168814201D0EA
:103CF0000120704700207047D4040020C1C700088D
:103D000046756E6374696F6E5B25735D20736861C1
:103D10006C6C206E6F742062652075736564206919
:103D20006E204953520A00003000000014020020A7
:103D3000D40300209B3C00087469646C650000009B
:103D40002DE9F04105460E461446304604F052FA7D
:103D500006F1140714B1012C1DD104E039462846A0
:103D600001F005FD17E02C680DE0A4F1140096F8B1
:103D7000351090F83520914204D23946143001F0C4
:103D8000F6FC02E02468AC42EFD1AC4203D13946E4
:103D9000284601F0ECFC0020BDE8F08170B5054636
:103DA0004FF0FF340AE004F007FE06462868143896
:103DB000046304F05EF8304604F002FE284601F089
:103DC000DDFC0028EFD0002070BD2DE9F041044655
:103DD0000F4615461E46002C04D1D822FD49FEA0F0
:103DE00002F0CBF83A460121204602F089FF204636
:103DF000143040600060A58366720020CCE710B5E7
:103E00000446002C05D1F349F6220C31F2A002F051
:103E1000B4F8204603F046F8012805D0ED49F72212
:103E20000C31F14802F0A9F8204603F029F828B92E
:103E3000E849F8220C31EDA002F09FF804F11400DB
:103E4000FFF7ACFF204602F085FF002010BD2DE9F2
:103E5000F04106460C46154604F0AEFD074601F05B
:103E6000C9FC58B1DB49EDA01A3101F0C9FFD949AD
:103E70004FF48A721A31F3A002F07FF8384604F04A
:103E80009FFD3146012002F083FF002884D000F11D
:103E9000140149600960848345727DE770B504466A
:103EA00004F08AFD054601F0A5FC58B1C949DBA024
:103EB000283101F0A5FFC74940F233122831E1A0B3
:103EC00002F05BF8284604F07BFD34B9C1494FF499
:103ED0009B722831C0A002F050F8204602F0E2FFA9
:103EE000012806D0BB4940F237122831BE4802F003
:103EF00044F8204602F0C4FF30B1B6494FF49C723A
:103F00002831D1A002F039F804F11400FFF746FF80
:103F1000204602F08AFF002070BD2DE9F3410446DF
:103F2000002C06D1AB494FF4AA723631AAA002F098
:103F300024F8204602F0B6FF012806D0A54940F239
:103F400055123631A84802F018F8CE48016809B178
:103F50002046884704F030FD0646A08B28B1401E5D
:103F6000A083304604F02CFD53E0019840B104F0EA
:103F700023FD074603F07AFF40F2751538B111E0D2
:103F8000304604F01DFD6FF00100BDE8FC81914951
:103F9000BDA0363101F034FF8E492A463631A9A042
:103FA00001F0EBFF04F008FD804601F023FC50B166
:103FB00088499AA0363101F023FF86492A463631D6
:103FC000A0A001F0DAFF404604F0FAFC384604F005
:103FD000F7FC03F04BFF054600202863627A294670
:103FE00004F11400FFF7ACFE0198002809DD05F18B
:103FF000600001AA0021074603F055FD384603F092
:1040000094FC304604F0DCFC03F045F8286B0028F3
:10401000BBD1AB48016809B1204688470020B4E70E
:1040200000217AE72DE9F0410446002C06D16949C8
:1040300040F2C112423168A001F09FFF204602F019
:1040400031FF012806D063494FF4E17242316648DE
:1040500001F093FF9B48016809B12046884700257D
:1040600004F0AAFC064604F11400074601F086FBA2
:1040700040B1A08B401CA083304604F0A1FC012D70
:1040800005D006E0384601F080FB0125F4E703F097
:1040900002F8002080E670B504460E461546002C56
:1040A00006D14C494FF4F97251314BA001F065FF34
:1040B000204602F0F7FE012806D0464940F2F312EE
:1040C0005131494801F059FF012E02D04FF0FF3025
:1040D00070BD04F071FC064604F11400FFF75EFEAB
:1040E000A583304604F06CFC02F0D5FF002070BDC3
:1040F00070B504460E461546002C06D1354940F2EF
:104100001F22603170A001F038FF324602212046A4
:1041100002F0F6FD20461430406000600120A083CC
:1041200000202062FF21A177E077657270BD10B595
:104130000446002C06D1274940F23F226E3162A08E
:1041400001F01BFF204602F0ADFE022806D02149F7
:104150004FF410726E31614801F00FFF204602F0FB
:104160008FFE30B91B4940F241226E315CA001F054
:1041700004FF04F11400FFF711FE204602F0EAFDEF
:10418000002010BD70B505460C4604F015FC06462F
:1041900001F030FB58B10F4920A07E3101F030FE14
:1041A0000C494FF417727E3126A001F0E6FE30462E
:1041B00004F006FC2946022002F0EAFD002807D0A0
:1041C00000F1140149600960012181830021A1E00F
:1041D000A5E00000D7C7000873656D20213D20527F
:1041E000545F4E554C4C0000E4CF000872745F6F72
:1041F000626A6563745F69735F73797374656D6F09
:10420000626A656374282673656D2D3E7061726500
:104210006E742E706172656E7429000046756E634F
:1042200074696F6E5B25735D207368616C6C206EC2
:104230006F74206265207573656420696E20495330
:10424000520A00003000000072745F6F626A65639A
:10425000745F69735F73797374656D6F626A6563A8
:1042600074282673656D2D3E706172656E742E70B4
:104270006172656E7429203D3D2052545F46414C69
:10428000534500005801002046756E6374696F6ED7
:104290005B25735D207368616C6C206E6F742062A7
:1042A000652075736564206265666F72652073634F
:1042B000686564756C65722073746172740A0000BD
:1042C0005C010020600100206D7574657820213D3F
:1042D0002052545F4E554C4C00000000B8D00008EE
:1042E00072745F6F626A6563745F69735F73797319
:1042F00074656D6F626A65637428266D7574657880
:104300002D3E706172656E742E706172656E7429D7
:10431000000000000162FF228277C177447270BD05
:1043200070B5044604F048FB054601F063FA58B145
:10433000FB49AFF2181001F063FDF94940F27D220C
:10434000AFF2001001F019FE284604F039FB34B931
:10435000F3494FF42072AFF2900001F00EFE2046B8
:1043600002F0A0FD022805D040F28122EC49ED4880
:1043700001F003FE204602F083FD28B140F28222C4
:10438000E749E9A001F0F9FD04F11400FFF706FD8B
:10439000204602F04AFD002070BD2DE9F34104469D
:1043A00004F00AFB064603F061FD40F29E2560B969
:1043B000DB491031AFF2301001F022FDD8492A4616
:1043C0001031AFF2801001F0D8FD04F0F5FA074685
:1043D00001F010FA60B1D2491031AFF2C01001F013
:1043E0000FFDCF492A461031AFF2A81001F0C5FDEC
:1043F000384604F0E5FA304604F0E2FA3CB9C84920
:1044000040F2A1221031AFF2401001F0B6FD20467B
:1044100002F048FD022806D0C14940F2A222103124
:10442000C04801F0AAFD03F021FD054604F0C4FADE
:104430000646CD48016809B1204688470020286318
:10444000206AA84203D1E07F401CE07743E0A08BC4
:1044500050B1A08B401EA083256295F83500A0774F
:10446000E07F401CE07736E0019848B3206A95F879
:10447000351090F83520914204D205F13502022121
:1044800003F02AFF627A294604F11400FFF758FC72
:104490000198002809DD05F1600001AA0021074606
:1044A00003F001FB384603F040FA304604F088FA86
:1044B00002F0F1FD286B58B10930C8D0286B64E5D3
:1044C0006FF001042C63304604F07AFA20465CE574
:1044D00004F072FA0646304604F072FAA348016806
:1044E00009B12046884700204FE52DE9F0410446F8
:1044F000002C07D18A4940F227321E31AFF2382012
:1045000001F03BFD204602F0CDFC022806D0844994
:104510004FF44A721E31834801F02FFD002504F04C
:104520004BFA074603F0A2FC40F22D3660B97C49F5
:104530001E31AFF2AC2001F063FC794932461E31E6
:10454000AFF2003001F019FD04F036FA804601F0B8
:1045500051F960B172491E31AFF2403001F050FCA8
:104560006F4932461E31AFF2243001F006FD40465D
:1045700004F026FA384604F023FA03F077FC0746E5
:1045800004F01AFA06467A48016809B120468847BD
:10459000206AB84207D04FF0FF343C63304604F045
:1045A0000FFA20462AE4E17F491EC9B2E177B1B98A
:1045B000A17F90F83520914204D004F11E0202211F
:1045C00003F08AFE04F11400074601F0D7F860B149
:1045D000A08B401CA08300202062FF20A0773046E3
:1045E00004F0EEF9012D0ED00FE06069143820625E
:1045F00090F83500A077E07F401CE077384601F066
:10460000C4F80125EBE702F046FD002045E410B5B3
:104610000446002C07D1424940F28A322F31AFF2D2
:10462000583001F0AAFC204602F03CFC022806D0DB
:104630003B4940F28B322F313A4801F09EFC4FF05B
:10464000FF3010BD70B504460E461546002C06D14D
:1046500033494FF46872403146A001F08EFC324677
:104660000321204602F04CFB657220461430406066
:1046700000600020E06170BD10B50446002C06D13A
:1046800027494FF46F724E313AA001F076FC204674
:1046900002F008FC032806D0214940F2BD324E3119
:1046A000394801F06AFC204602F0EAFB30B91C49A7
:1046B00040F2BE324E3135A001F05FFC04F114002F
:1046C000FFF76CFB204602F045FB002010BD70B5E3
:1046D00005460C4604F070F9064601F08BF868B107
:1046E0000F495E31AFF2CC4001F08AFB0C4940F239
:1046F000D7325E31AFF2B44001F03FFC304604F0F7
:104700005FF92946032002F043FB002806D04472DB
:1047100000F11401496009600021C16170BD000011
:1047200065C80008B8D0000872745F6F626A65637C
:10473000745F69735F73797374656D6F626A6563C3
:104740007428266D757465782D3E706172656E747F
:104750002E706172656E7429203D3D2052545F4673
:10476000414C534500000000580100205C0100202E
:10477000600100206576656E7420213D2052545FF3
:104780004E554C4C0000000074D0000872745F6FEE
:10479000626A6563745F69735F73797374656D6F63
:1047A000626A65637428266576656E742D3E706155
:1047B00072656E742E706172656E7429000000005F
:1047C00070B50446002C06D1FF4940F2F532AFF235
:1047D0005C0001F0D2FB204602F064FB032805D008
:1047E00040F2F632F849F94801F0C7FB204602F0E2
:1047F00047FB28B140F2F732F349F5A001F0BDFBC9
:1048000004F0DAF8054600F0F5FF58B1EE49AFF2D2
:10481000F45001F0F5FAEC4940F2F932AFF2DC5015
:1048200001F0ABFB284604F0CBF804F11400FFF7CD
:10483000B5FA204602F0F9FA00206FE72DE9F047BB
:1048400004460D46002C07D1DF494FF48362103136
:10485000AFF2E00001F091FB204602F023FB0328B9
:1048600006D0D94940F219421031D84801F085FBF1
:104870004FF0FF3895B1002704F09EF88246E069BA
:104880002843E061E248016809B12046884704F105
:104890001400814600F072FF18B128E04046BDE8E0
:1048A000F087656921E0A5F11400464690F84010B4
:1048B000CA0705D0C16BE269914309D1002607E020
:1048C000890705D5C16BE269114001D0C16300269B
:1048D0002D6856B990F84010490703D5E169C26BBD
:1048E0009143E16103F0C5FA01274D45DBD1504604
:1048F00004F066F8012F01D102F0CDFB0020CEE7D5
:104900002DE9FF4705460E469046DDF8309004F04D
:1049100053F8074603F0AAFA40F27B4460B9AA496B
:104920001E31AFF29C6001F06BFAA74922461E319E
:10493000AFF2F06001F021FB04F03EF8824600F097
:1049400059FF60B1A0491E31AFF2307001F058FA42
:104950009D4922461E31AFF2147001F00EFB504605
:1049600004F02EF8384604F02BF83DB9964940F291
:104970007E421E31AFF2042001F0FFFA284602F019
:1049800091FA032806D0904940F27F421E318F48A9
:1049900001F0F3FA4FF0FF30002E59D0074603F034
:1049A00065FA0446002121639A48016809B1284646
:1049B000884704F001F882465FEAC87005D0E869CC
:1049C00036EA000011D100270FE05FEA887004D5B5
:1049D000E869304209D0002707E07B4940F29E4257
:1049E0001E31AFF2A07001F0C8FA9FB3039890B3E4
:1049F000E66384F840806A7A214605F11400FFF7E7
:104A00009FF90398002809DD04F1600003AA002142
:104A1000064603F048F8304602F087FF504603F0A0
:104A2000CFFF02F038FB206B002811D103F0C4FF48
:104A30008246B9F1000F02D0E06BC9F80000504681
:104A400003F0BEFF7448016809B128468847206B0F
:104A500004B024E700E00DE0B9F1000F03D0E869ED
:104A60003040C9F800005FEA4870E8D5E869B04313
:104A7000E861E4E76FF001002063E0E770B5044609
:104A80000D46002C07D150494FF49E622C31AFF2F5
:104A90001C3001F072FA204602F004FA032806D016
:104AA000494940F2F1422C31484801F066FA012DA3
:104AB00002D04FF0FF3031E603F07EFF054604F1EF
:104AC0001400FFF76BF90020E061284603F078FF3F
:104AD00002F0E1FA002021E62DE9F0410446069FAC
:104AE000884616461D46002C06D1374940F21E5214
:104AF0003D314AA001F041FA42460421204602F02D
:104B0000FFF867722046143040600060E66125843B
:104B100000206084A084E08428346460246041E53F
:104B200010B50446002C06D1274940F241524831C5
:104B30003AA001F022FA204602F0B4F9042806D087
:104B4000214940F242524831384801F016FA2046D5
:104B500002F096F930B91C4940F24352483134A072
:104B600001F00BFA04F11400FFF718F904F1280022
:104B7000FFF714F9204602F0EDF8002010BD2DE9F2
:104B8000F04104460D46164603F016FF074600F0B6
:104B900031FE68B10C495531AFF6801001F030F9A3
:104BA000094940F25F525531AFF6681001F0E5F95E
:104BB000384603F005FF2146042002F0E9F80446D8
:104BC00004B14DE062E00000D3C8000874D00008D2
:104BD00072745F6F626A6563745F69735F73797320
:104BE00074656D6F626A65637428266576656E7498
:104BF0002D3E706172656E742E706172656E7429DF
:104C0000203D3D2052545F46414C5345000000007A
:104C100060010020580100205C0100206D6220210D
:104C20003D2052545F4E554C4C000000FCD0000813
:104C300072745F6F626A6563745F69735F737973BF
:104C400074656D6F626A65637428266D622D3E70AF
:104C50006172656E742E706172656E742900000059
:104C600066722046143040600060A8B22084800044
:104C700001F0A9FAE06158B100206084A084E084CA
:104C800004F128004060006020468BE4204689E45F
:104C9000204602F0CAF8002084E470B5044603F010
:104CA0008BFE054600F0A6FD58B1F749AFF69420FB
:104CB00001F0A6F8F44940F28A52AFF6782001F0EC
:104CC0005CF9284603F07CFE34B9EF4940F28D527E
:104CD000AFF2B80001F051F9204602F0E3F80428E1
:104CE00005D040F28E52E849E84801F046F92046E6
:104CF00002F0C6F828B140F28F52E349E4A001F077
:104D00003CF904F11400FFF749F804F12800FFF71B
:104D100045F8E06901F01DFB204602F086F800200E
:104D2000FCE42DE9F74F82B004468B46002C07D1F6
:104D3000D54940F2B5520D31AFF2201001F01DF906
:104D4000204602F0AFF8042806D0CF4940F2B65210
:104D50000D31CE4801F011F9002603F087F8054621
:104D6000DA48016809B12046884703F025FE8046ED
:104D7000608C218C6FF0020A884201D1049808B13E
:104D800000276BE0404603F01BFE504605B0BDE82F
:104D9000F08F2F63049830B103F00EFE019003F002
:104DA00065F828B112E0404603F00AFE5046EDE7F0
:104DB000B5490D31AFF6303001F022F8B24940F27A
:104DC000D9520D31AFF6843001F0D7F803F0F4FD7D
:104DD000814600F00FFD68B1AB490D31AFF6C4302C
:104DE00001F00EF8A84940F2D9520D31AFF6AC30BF
:104DF00001F0C3F8484603F0E3FD019803F0E0FD3D
:104E0000627A294604F12800FEF79AFF04980028E8
:104E10000CDDFEF782FB064605F1600004AA0021C6
:104E2000814602F040FE484602F07FFD404603F016
:104E3000C7FD02F030F9286B08B1286BA6E703F034
:104E4000BBFD80460498002808DDFEF766FB861B44
:104E50000498801B0490002800DA0497608C218C51
:104E6000884296D0A18CE06940F821B0A08C401C0B
:104E700080B2A084218C884200D3A784608C401C1F
:104E8000608404F11400044600F078FC20B1404630
:104E900003F096FD002079E7204600F076FC4046BE
:104EA00003F08EFD02F0F7F800206FE7002238E7EC
:104EB0002DE9F74F82B004468B46002C07D172498A
:104EC00040F247621D31AFF2AC2001F056F82046A7
:104ED00001F0E8FF042806D06B494FF4C9621D3188
:104EE0006A4801F04AF8002602F0C0FF05467848FB
:104EF000016809B12046884703F05EFD8046608C5A
:104F00006FF0010A08B9049808B100276BE0404629
:104F100003F056FD504639E72F63049830B103F093
:104F20004BFD019002F0A2FF38B114E0404603F0BF
:104F300047FD5046C5F830A028E753491D31AFF66C
:104F4000B84000F05DFF504940F26D621D31AFF690
:104F50000C5001F012F803F02FFD814600F04AFCDE
:104F600068B149491D31AFF64C5000F049FF464940
:104F700040F26D621D31AFF6345000F0FEFF48463E
:104F800003F01EFD019803F01BFD627A294604F12F
:104F90001400FEF7D5FE049800280CDDFEF7BDFADC
:104FA000064605F1600004AA0021814602F07BFD5F
:104FB000484602F0BAFC404603F002FD02F06BF8EE
:104FC000286B08B1286BE1E603F0F6FC80460498F4
:104FD000002808DDFEF7A1FA861B0498801B0490C8
:104FE000002800DA0497608C002895D0E18CE069F5
:104FF00050F82100CBF80000E08C401C80B2E08427
:10500000218C884200D3E784608C401E608404F1C8
:105010002800064600F0B2FB2E4D40B1404603F09A
:10502000CFFC296809B1204688470020AEE630460B
:1050300000F0ABFB404603F0C3FC296809B12046F1
:10504000884702F028F80020A0E670B504460D4617
:10505000002C07D10C4940F2CD622831AFF2444018
:1050600000F08BFF204601F01DFF042806D0064902
:1050700040F2CE622831054800F07FFF012D2BD091
:105080004FF0FF3017E5000035C90008FCD00008DC
:1050900072745F6F626A6563745F69735F7379735B
:1050A00074656D6F626A65637428266D622D3E704B
:1050B0006172656E742E706172656E7429203D3D5B
:1050C0002052545F46414C534500000060010020CF
:1050D000580100205C01002003F06EFC054604F13D
:1050E0001400FEF75BFE04F12800FEF757FE0020D7
:1050F0006084A084E084284603F062FC01F0CBFFCA
:105100000020D8E42DE9F0470446DDE90868894627
:1051100017461D46002C05D140F20A72FD49FEA03B
:1051200000F02BFF4A460521204601F0E9FD84F8F6
:1051300009802046143040600060E761ED1C4FF6A6
:10514000FC70054025842D1DB6FBF5F0608400221F
:10515000A262E2622263002008E0218CE369091D5B
:1051600000FB0131236B0B602163401C618C814289
:10517000F3DCA2840020BDE8F08710B50446002CC3
:1051800006D1E44940F23B720B31E3A000F0F5FE9A
:10519000204601F087FE052806D0DE4940F23C7229
:1051A0000B31E14800F0E9FE204601F069FE30B91C
:1051B000D84940F23D720B31DCA000F0DEFE04F174
:1051C0001400FEF7EBFD204601F0C4FD002010BDE9
:1051D00070B5044603F0F0FB054600F00BFB68B128
:1051E000CC492531AFF6CC7000F00AFEC94940F237
:1051F00097722531AFF6B47000F0BFFE284603F079
:10520000DFFB34B9C34940F29A722531C2A000F0E5
:10521000B4FE204601F046FE052806D0BD4940F206
:105220009B722531C04800F0A8FE204601F028FE00
:1052300030B1B84940F29C722531C8A000F09DFE03
:1052400004F11400FEF7AAFDE06901F082F820469F
:1052500001F0EBFD00202EE42DE9F04104460D465F
:1052600016461F4603F0A8FB804600F0C3FA58B16B
:10527000A849C948183100F0C3FDA64940F25D7243
:105280001831C6A000F079FE404603F099FB214694
:10529000052001F07DFD0446BCB167722046143044
:1052A00040600060ED1C4FF6FC7005402584B0B2F4
:1052B00060842D1D684300F086FFE06138B1002254
:1052C000A262E262226300200FE0204627E420462B
:1052D000FFF77EFF002022E4218CE369091D00FB1B
:1052E0000131236B0B602163401C618C8142F3DC34
:1052F000A284204613E42DE9F04104460F461646E9
:10530000002C06D1834940F2BC72323182A000F0F9
:1053100034FE204601F0C6FD052806D07D4940F246
:10532000BD723231804800F028FE37B9794940F229
:10533000BE7232319AA000F020FE36B9754940F2B3
:10534000BF7232319BA000F018FE208CB04202D216
:105350004FF0FF3099E49A4803680BB12046984714
:1053600003F02AFB256BA5B12968216303F028FB14
:105370000020286032463946281D00F090FA03F0DC
:105380001BFB0646E06A00B10560E562A06A28B131
:1053900005E003F015FB6FF0020076E4A562A08C37
:1053A000401CA08404F11400044600F0E7F920B189
:1053B000304603F005FB002067E4204600F0E5F9E5
:1053C000304603F0FDFA01F066FE00205DE42DE9B1
:1053D000F04104460F461646002C06D14D4940F6D2
:1053E00016023D314CA000F0C8FD204601F05AFDE8
:1053F000052806D0474940F617023D314A4800F0DB
:10540000BCFD37B9434940F618023D3164A000F0B5
:10541000B4FD36B93F4940F619023D3165A000F0B0
:10542000ACFD208CB04202D24FF0FF302DE4644836
:1054300003680BB12046984703F0BEFA256B8DB187
:105440002968216303F0BCFA32463946281D00F072
:1054500026FA03F0B1FA0646A06A2860A562E06A5F
:1054600028B105E003F0ACFA6FF002000DE4E5624C
:10547000A08C401CA08404F11400044600F07EF9C6
:1054800020B1304603F09CFA002005E4204600F0ED
:105490007CF9304603F094FA01F0FDFD002015E799
:1054A0002DE9FF4F81B004461746002C06D119495B
:1054B0004FF407624A3118A000F05FFD204601F06A
:1054C000F1FC052806D0134940F671024A3116480E
:1054D00000F053FD029830B90E4940F672024A318D
:1054E0002FA000F04AFD37B90A4940F673024A314D
:1054F00030A000F042FD002602F0B8FC054631481D
:10550000016809B12046884703F056FA8146A08C0D
:105510005AE000006BC900086D7120213D205254F3
:105520005F4E554C4C0000002CD0000872745F6F29
:10553000626A6563745F69735F73797374656D6FB5
:10554000626A65637428266D712D3E706172656EA6
:10555000742E706172656E742900000072745F6F42
:10556000626A6563745F69735F73797374656D6F85
:10557000626A65637428266D712D3E706172656E76
:10558000742E706172656E7429203D3D2052545F07
:1055900046414C53450000001C420008300000000A
:1055A00062756666657220213D2052545F4E554CEF
:1055B0004C00000073697A6520213D203000000016
:1055C00060010020580100206FF0010B08B9049819
:1055D00010B14FF0000867E0484603F0F1F9584673
:1055E0002CE403F0E9F9009002F040FC50B96A495C
:1055F0006A4800F005FC684940F68902AFF2640091
:1056000000F0BBFC03F0D8F9824600F0F3F858B183
:10561000624861496C3800F0F3FB5F4940F689024B
:10562000AFF2880000F0A9FC504603F0C9F90098D9
:1056300003F0C6F9C5F830800498F0B1627A2946C3
:1056400004F11400FEF77CFB049800280CDDFDF744
:1056500064FF064605F1600004AA0021824602F0BC
:1056600022FA504602F061F9484603F0A9F901F028
:1056700012FD286B40B1286B0DE4484603F0A0F9F9
:105680005846C5F830B006E403F096F98146049810
:10569000002809DDFDF741FF861B0498801B04905C
:1056A000002801DACDF81080A08C002899D0A56AD6
:1056B0002868A062E06AA84201D1C4F82C80A08CBE
:1056C000401EA084484603F07BF9208CB84200D2EB
:1056D00007463A46291D029800F0E1F803F06CF9FC
:1056E000216B2960256303F06BF92D48016809B12E
:1056F0002046884700200EE470B504460D46002C75
:1057000007D1254940F6F8020B31AFF2F41000F052
:1057100034FC204601F0C6FB052806D01E4940F6A1
:10572000F9020B311F4800F028FC012D02D04FF088
:10573000FF30A7E403F040F9054604F11400FEF73A
:105740002DFB002108E00268A262E26A824200D1D9
:10575000E162226B02602063A06A0028F3D1A18479
:10576000284603F02DF901F096FC00208AE44268F7
:10577000116042684A604160086070470168814278
:1057800001D1012070470020704710B5006814381F
:1057900002F06FFB002010BDB5C900088842000868
:1057A0005C0100202CD00008144948607047134960
:1057B0008860704710B503F0FFF804460F490A7877
:1057C000521C0A70496801B188472046BDE8104064
:1057D00003F0F6B810B503F0EFF8044607490A786D
:1057E000521E0A70896801B188472046BDE8104002
:1057F00003F0E6B80148007870470000100100206F
:1058000010B5FFF7F7FFF84C08B1606810BD02F063
:105810002DFB08B1006B10BD606810BD70B504466B
:10582000FFF7E8FFF04D08B16C6070BD02F01EFBA1
:1058300008B1046370BD6C6070BD10B5FFF7DAFF8E
:1058400010B1E948001D10BD02F010FB08B1303066
:1058500010BDE548001D10BD10B50346CCB2042AAA
:1058600015D3810713D1014644EA042343EA0343D5
:1058700005E00B604B608B60CB601031103A102A52
:10588000F7D201E008C1121F042AFBD20B46E1B295
:1058900001E003F8011B521E541CFAD110BD30B5B3
:1058A0000346102A1ED301F0030403F003052C4322
:1058B0000BD017E00C681C604C685C608C689C60C6
:1058C000CC681031DC601033103A102AF2D202E0BA
:1058D00010C910C3121F042AFAD203E011F8014BB9
:1058E00003F8014B521E541CF8D130BD10B50346CD
:1058F0001846814210D28C189C420DD9991803E0A9
:1059000014F8013D01F8013D521E531CF8D110BDA1
:1059100011F8014B03F8014B521E541CF8D110BD75
:1059200010B5002306E003780C781B1B04D1401C43
:10593000491C521E002AF6D1184610BD014600E04F
:10594000491C0A78002AFBD1081A7047F0B50646B0
:105950000F463846FFF7F2FF0546280004D03046D0
:10596000FFF7ECFF044609E03046F0BD641E2A460E
:1059700039463046FFF7D4FF20B1761CAC42F5DA49
:105980000020F0BD3046F0BD10B510F8012B11F825
:10599000013BA2F14104192C00D82032A3F14104AB
:1059A000192C00D820339A4201D1002AEDD1D01A07
:1059B00010BD10B5002A07D0034611F8014B03F8BB
:1059C000014B14B1521EF8D110BD002101E003F8C3
:1059D000011B521EFBD110BD10B5002308E011F8C9
:1059E000013B0478E31A5BB223B9401C14B1521E88
:1059F000002AF4D1184610BD01E0401C491C027871
:105A000012B10B789A42F8D000780978401A7047A2
:105A1000024600E0521C137813B1131A8B42F9D3DB
:105A2000101A704770B506463046FFF787FF451CD1
:105A3000284600F0C8FB044634B12A4631462046C9
:105A4000FFF72DFF204670BD002070BD70472DE987
:105A5000FF4FDDE90DB60F9D6C0602D5DFF88CA176
:105A600003E0DFF888A1AAF1110AEC0601D525F0C0
:105A70000105EC0702D04FF0300901E04FF020099A
:105A80000027AC070BD5002A02DA2D27524206E088
:105A90006C0701D52B2702E02C0700D52027002416
:105AA000EE467AB9302201248DF800200CE00A2B52
:105AB00015D002F00F081209A4461AF80880641CD9
:105AC0000EF80C80002AF2D1B44200DD2646ABEB82
:105AD000060215F0110F4FF0200309D016E04FF029
:105AE0000A0CB2FBFCF80CFB1828B2FBFCF2E3E753
:105AF0003FB1002A05DD521E03E0884200D8037042
:105B0000401CB2F1000CA2F10102F6DC27B1884280
:105B100001D80770521E401CED0605D508E08842EA
:105B200001D880F80090401C151EA2F10102F6DC9D
:105B3000302703E0884200D80770401C3546761EA7
:105B4000A542F7DC05E0884202D81EF80450057033
:105B5000401C251EA4F10104F5DC03E0884200D8B6
:105B60000370401C141EA2F10102F7DC04B0BDE872
:105B7000F08F2DE9FF4F83B082460AEB01077F1EAD
:105B80005446A74201D24FF0FF374FF020094FF0A3
:105B9000250B17E1252804D0BC4200D82070641CD6
:105BA0000DE100250599491C059108782D2814D090
:105BB0002B2815D020281BD023281CD030281DD0FE
:105BC0004FF0FF384646059A1278303A0A2A18D222
:105BD00005A800F0EBF906461FE045F01005E1E7E7
:105BE00045F00405DEE700001C010020DFCA0008C4
:105BF00045F00805D6E745F02005D3E745F0010557
:105C0000D0E72A2809D1491C0591069840C806907A
:105C1000002E02DA764245F01005059801782E290B
:105C200018D1401C05900178A1F130020A2A04D253
:105C300005A800F0BBF9804607E02A2905D1401CE1
:105C40000590069850F8048B0690B8F1000F01DA21
:105C50004FF000080021059A1078682801D06C28C0
:105C600002D10146521C05920A23059800786F283C
:105C700071D00CDC632820D004DC25286CD0582897
:105C80000DD187E0642801D0692808D186E070280A
:105C900063D073282FD0752871D078287CD0BC426F
:105CA00001D884F800B0641C05990878002868D0F1
:105CB000BC4200D82070641C81E0E80605D507E0EE
:105CC000BC4201D884F80090641C761E002EF7DCDC
:105CD000069810F8041B0690C8B2BC4200D8207089
:105CE000641C04E0BC4201D884F80090641C761E59
:105CF000002EF7DC63E0069808C8069003B9B5A348
:105D00001846FFF71BFEB8F1000F02DD404500DD2D
:105D10004046E90605D508E0BC4201D884F8009069
:105D2000641C3146761E8142F6DC002106E0BC424E
:105D300001D81A782270641C5B1C491C8142F6DB76
:105D400004E0BC4201D884F80090641C3146761E01
:105D50008142F6DC33E01BE014E0701C02D108261F
:105D600045F00105CDE9006806980295102304C8A6
:105D7000069039462046FFF76AFE04461FE00FE012
:105D80000AE028E0BC4201D884F800B0641C16E0A8
:105D9000082305E045F04005102301E045F0020529
:105DA0006C291BD068291DD0069804C80690CDE93F
:105DB0000068394620460295FFF749FE04460598DB
:105DC000401C05900598007800287FF4E3AEBC42A3
:105DD00011D8207010E0491E0591F0E7069804C81C
:105DE0000690E4E7069830F8041B06908AB2A807EC
:105DF000DDD512B2DBE73870A4EB0A0007B0B6E6D7
:105E00000FB438B505AB00937F217448049AFFF7AF
:105E1000B0FE03467F2B00D97F23714D286860B107
:105E2000048B44F0400101836C4A0021FDF798FD8A
:105E30002868048338BC5DF814FB6848FFF706FE49
:105E4000F8E708B567A0FFF7DBFF69A0FFF7D8FF09
:105E500070A0009000230122032171A0FFF7D0FF62
:105E6000BDE8084076A0CBE70FB410B505AB049AA7
:105E7000FFF77FFE10BC5DF814FB17B40A46029BC7
:105E800003B04FF0FF3110BC73E60FB410B504AA95
:105E90000399FFF7F2FFEDE751480068704770B5CE
:105EA0004F4D2E68FDF7DAFB044644B1286808B16F
:105EB000FDF7F4FC43212046FDF799FC2C603046A9
:105EC00070BD70B50446002C11D0454E306878B1D5
:105ED000058B45F0400101832046FFF72FFD034667
:105EE000224600213068FDF73BFD3068058370BD18
:105EF0002046FFF7ABFD70BD10B5C91C21F00304AF
:105F0000C01C20F00300204400F05DF900280BD0F5
:105F1000611E084201D1011903E00219521E22EA52
:105F2000010141F8040C084610BD50F8040C00F0C3
:105F300010BA002807D04D4910F0FF0F05D0C0B2AD
:105F4000085C401C70470020704710F47F4F04D05D
:105F5000C0F30720085C0930704710F47F0F04D0AD
:105F6000C0F30740085C1130704701EB1060007807
:105F7000193070471A498860704738B50D460021BE
:105F8000009117498C68002C05D001B02946A44621
:105F9000BDE830406047134601462A4634A0FFF76B
:105FA0002FFF9DF800000028FBD038BD10B5024639
:105FB00000206FF02F0407E04B1C1360097800EB02
:105FC000800004EB4000084411680B78303B0A2B3A
:105FD000F2D310BD284E554C4C290000E40400209B
:105FE0001C0100200A205C207C202F0A00000000F9
:105FF0002D205254202D20202020205468726561CD
:1060000064204F7065726174696E67205379737490
:10601000656D0A004D617920313020323032330015
:10602000202F207C205C202020202025642E256429
:106030002E2564206275696C642025730A000000B7
:106040002032303036202D203230313820436F70EE
:106050007972696768742062792072742D7468722D
:10606000656164207465616D0A000000CEC9000896
:106070002825732920617373657274696F6E2066B9
:1060800061696C65642061742066756E6374696F04
:106090006E3A25732C206C696E65206E756D626595
:1060A000723A2564200A0000F74908607047F649F3
:1060B0004860704770B50446F34DA868844204D226
:1060C000A222F249F2A0FFF758FFE868844204D305
:1060D000A322EE49F6A0FFF750FF608820B1A4226A
:1060E000EA49FEA0FFF749FF6068A96808448442B6
:1060F0000FD042886AB9EA6890420AD02A6982427F
:1061000000D12C6142686260436801F10800621AA4
:106110001A50A0680844A0420CD04288002A09D135
:106120002A69A24200D1286162684260401A62680E
:106130000831505070BD2DE9F04106460F46F01C65
:1061400020F0030427F0030502F036FC8046FFF739
:1061500051FB50B1CD49E5A00B31FFF751FECB49C2
:10616000D3220B31EBA0FFF708FF404602F028FCDA
:10617000182D21D9A5F11800A0421DD3291BC24D0D
:1061800018396961AC604FF4F55222800C316160BE
:106190000020A060608060682044E86002800122E6
:1061A0004280416081600023DBA1DD48FDF70DFEE8
:1061B000A8682861BDE8F0813A463146BDE8F04163
:1061C000D8A0FFF71DBE2DE9F047044602F0F4FB0E
:1061D0000546FFF70FFB58B1AC49C4A01F31FFF7CC
:1061E0000FFEAA494FF48B721F31CAA0FFF7C5FEFC
:1061F000284602F0E5FB4CB1E41C24F00305A24E56
:106200007069854204D90020BDE8F0870020FBE7D3
:106210000C2D00D20C254FF0FF31C148FDF77DFE5B
:106220003769B168781AD6F814C0ACEB050388E07A
:106230000C186288002A78D16268121A0C3AAA42B5
:106240007ED362684FF00109131A0C3B05F1180266
:106250004FF4F558934221D343190C33CA18A2F8CE
:1062600000804FF0000AA2F802A0D4F804A0C2F8FF
:1062700004A090606360A4F8029050680CF10C0CCC
:10628000604502D001F108028350B06928440C3007
:10629000B061F26982420DD2F0610BE0A4F8029085
:1062A0006068621A801AB2691044B061F269824271
:1062B00000D2F061A4F80080BC4215D1F26802E07F
:1062C000406808443061306943880BB19042F7D18F
:1062D0003169914208D0408830B16C4940F2831254
:1062E0001F319FA0FFF749FE8D48FDF79BFE601907
:1062F000F1680C30884206D9644940F287121F3198
:10630000A148FFF73AFE04F10C07B80706D05F4931
:106310004FF4C4721F319D48FFF72FFEA00708D02D
:106320005A4940F289121F3100E009E098A0FFF7B6
:1063300024FE326812B1294638469047384663E752
:10634000606883423FF674AF7548FDF76BFE00202E
:106350005AE770B5044602F02FFB0546FFF74AFAEC
:1063600058B14A4961A00839FFF74AFD474940F250
:106370002922083967A0FFF700FE284602F020FB1B
:10638000002C5FD0A00706D0404940F22D220839EA
:106390008BA0FFF7F2FD3C4DA868844202D3E86869
:1063A000844206D3394940F22E2208399148FFF73A
:1063B000E4FD696809B120468847A868844241D352
:1063C000E86884423ED20C3C4FF0FF315448FDF760
:1063D000A4FD60884FF4F55610B12088B04208D073
:1063E00085A0FFF70DFD23886288214689A0FFF76D
:1063F00007FD608830B9254940F24D22083991A047
:10640000FFF7BBFD2088B04206D0204940F24E2263
:1064100008398FA0FFF7B1FD002060802680286931
:10642000844200D22C61A9686068611A401AA96987
:10643000081AA8612046FFF73DFEBDE870403848C5
:10644000FDF7F0BD70BD2DE9F04107460C4602F0A6
:10645000B3FA0546FFF7CEF958B10C4923A029310C
:10646000FFF7CEFC094940F2AD12293129A0FFF710
:1064700084FD284602F0A4FAE41C24F00304DFF8AB
:106480000880D8F81400F1E028010020F8CA0008BC
:106490002872745F75696E74385F74202A296D657F
:1064A0006D203E3D20686561705F70747200000071
:1064B0002872745F75696E74385F74202A296D655F
:1064C0006D203C202872745F75696E74385F74208B
:1064D0002A29686561705F656E6400006D656D2DC9
:1064E0003E75736564203D3D2030000046756E6347
:1064F00074696F6E5B25735D207368616C6C206ED0
:106500006F74206265207573656420696E2049533D
:10651000520A000030000000686561700000000051
:10652000640500206D656D20696E69742C206572AC
:10653000726F7220626567696E2061646472657350
:106540007320307825782C20616E6420656E64207D
:106550006164647265737320307825780A000000E6
:1065600028286C66726565203D3D20686561705F16
:10657000656E6429207C7C2028216C667265652DFF
:106580003E75736564292900E8D1000840D10008F0
:1065900028282872745F75696E7433325F74296DB0
:1065A000656D292026202852545F414C49474E5F93
:1065B00053495A45202D20312929203D3D203000C6
:1065C00028282872745F75696E7433325F7429727B
:1065D0006D656D292026202852545F414C49474E55
:1065E0005F53495A45202D20312929203D3D203037
:1065F000000000008CD10008746F20667265652071
:106600006120626164206461746120626C6F636BFD
:106610003A0A00006D656D3A203078253038782CC4
:10662000207573656420666C61673A2025642C20B0
:106630006D6167696320636F64653A203078253047
:1066400034780A006D656D2D3E7573656400000039
:106650006D656D2D3E6D61676963203D3D20484548
:1066600041505F4D4147494300000000844201D939
:1066700000209FE594B1B7B14FF0FF315148FDF7CD
:106680004CFCD8F808108F4203D3D8F80C0087428E
:106690000DD34C48FDF7C6FC38468BE53846FFF76E
:1066A00058FE002086E52046BDE8F0418BE5A7F1C5
:1066B0000C06731A7068C51A0C3DA54204D14148F6
:1066C000FDF7B0FC384675E504F11800A84220D269
:1066D000D8F81820281B101AC8F818001A190C32FC
:1066E00088184FF4F5540480002444807468446092
:1066F00083607260D8F8144043680C34A34201D020
:1067000008315A50FFF7D6FC2E48FDF78BFC38466F
:1067100050E52C48FDF786FC2046FFF754FD064661
:1067200056B1A54200D22C46224639463046FFF7E4
:10673000B6F83846FFF70DFE30463BE570B5044627
:106740000D4602F039F90646FFF754F858B11E49D4
:10675000AFF26820FFF754FB1B4940F21222AFF260
:106760004C20FFF70AFC304602F02AF96C43204621
:10677000FFF729FD054625B1224600212846FFF7EF
:106780006BF8284670BD10B5104B002801D05C692D
:10679000046009B198690860002A01D0D8691060C6
:1067A00010BD10B5094C0AA06169FFF729FB0DA0C7
:1067B000A169FFF725FBE169BDE810400EA0FFF7D6
:1067C0001FBB0000640500202CCB0008280100201E
:1067D000746F74616C206D656D6F72793A202564F9
:1067E0000A00000075736564206D656D6F72792015
:1067F0003A2025640A0000006D6178696D756D208E
:10680000616C6C6F6361746564206D656D6F727926
:106810003A2025640A000000EC4908607047EB4903
:10682000486070472DE9F0410446069E88461546AB
:106830001F46002C04D16522E549E6A0FFF79DFB29
:1068400042460721204600F05BFA656127F003000D
:10685000A061F61C26F00302E261121DB0FBF2F00B
:106860006062A06204F12C00406000600025656356
:106870006169002006E0431C03FB021600FB02F3E3
:10688000CE50401C636A8342F5D8401E50430D50E1
:1068900021620020BDE8F0812DE9F0410446002C82
:1068A00005D1CB4998220B31CAA0FFF766FB2046E1
:1068B00000F0F8FA072805D0C54999220B31C9A084
:1068C000FFF75BFB204600F0DBFA28B9C0499A22AB
:1068D0000B31D3A0FFF751FB4FF0FF3504F12C072C
:1068E0000DE002F069F80646E06A1438056301F02D
:1068F000C0FA606B401E6063304602F061F83846B3
:1069000000F05CF90028ECD0204600F023FA0020CB
:10691000C0E72DE9F04104460E46154602F04CF85A
:106920000746FEF767FF50B1A949C7A01831FFF726
:1069300067FAA749CF221831CDA0FFF71EFB3846D2
:1069400002F03EF82146072000F022FA044620001B
:1069500016D0ED1C25F00300E061001D05467043D4
:10696000A061FFF730FC606160B16662A66204F16D
:106970002C004060006000236363616900200DE02B
:10698000002087E7204600F050FA002082E7421CF2
:1069900002FB051600FB05F28E50401C626A824223
:1069A000F5D8401E68430B502162204672E72DE95E
:1069B000F041044602F000F80546FEF71BFF58B10F
:1069C0008349A1A02531FFF71BFA814940F20B1240
:1069D0002531A7A0FFF7D1FA284601F0F1FF34B91D
:1069E0007B494FF4877225317AA0FFF7C6FA20461B
:1069F00000F058FA072806D0754940F20F122531E9
:106A000078A0FFF7BAFA204600F03AFA30B17049A0
:106A10004FF48872253197A0FFF7AFFA4FF0FF359A
:106A200004F12C070DE001F0C7FF0646E06A1438B8
:106A3000056301F01EFA606B401E6063304601F092
:106A4000BFFF384600F0BAF80028ECD06069FFF7C5
:106A500080FC204600F0E9F900201BE72DE9F34710
:106A600004464FF0000801F001FA064601F0A4FFC9
:106A7000814600275BE0019800283FD001F09CFF91
:106A80000546FEF7B7FE58B151496FA03231FFF706
:106A9000B7F94F494FF4AC72323175A0FFF76DFA78
:106AA000284601F08DFF3763304601F0A3FB04F167
:106AB0002C0006F1140501684D600168296005602D
:106AC0006860606B401C6063019800280CDDFCF777
:106AD00024FD804606F1600001AA0021054600F071
:106AE000E2FF284600F021FF484601F069FF00F070
:106AF000D2FA306B58B10020BDE8FC87484601F05F
:106B00005FFF6FF00100FEF789FE0020F4E70198B7
:106B1000002809DDFCF701FD0199A0EB0800081A27
:106B20000190002800DA019701F046FF8146A06A33
:106B30000028A0D0A06A401EA062256A35B9244969
:106B400040F28512323158A0FFF717FA2868206208
:106B50002C60484601F034FF1C48026812B1291D20
:106B600020469047281DC7E770B5051F2C681749B8
:106B70004A68002A02D001462046904701F01CFFD7
:106B80000646A06A401CA062206A28602562606BED
:106B900078B1E06A14380021016301F06AF9606B92
:106BA000401E6063304601F00BFFBDE8704000F00E
:106BB00072BA3046BDE8704001F002BF0168814200
:106BC00001D10120704700207047000048010020DB
:106BD00036CB00086D7020213D2052545F4E554C3D
:106BE0004C00000072745F6F626A6563745F676572
:106BF000745F7479706528266D702D3E70617265C2
:106C00006E7429203D3D2052545F4F626A65637463
:106C10005F436C6173735F4D656D506F6F6C000007
:106C200072745F6F626A6563745F69735F737973AF
:106C300074656D6F626A65637428266D702D3E7091
:106C40006172656E7429000046756E6374696F6EBB
:106C50005B25735D207368616C6C206E6F742062BD
:106C600065207573656420696E204953520A0000DF
:106C70003000000072745F6F626A6563745F6973ED
:106C80005F73797374656D6F626A65637428266DCE
:106C9000702D3E706172656E7429203D3D20525406
:106CA0005F46414C53450000626C6F636B5F7074CC
:106CB0007220213D2052545F4E554C4C0000000084
:106CC000A94908607047A84948607047A64988608C
:106CD0007047A549C8607047A3490861704770476D
:106CE0000021A14A143202EB01131B78834202D126
:106CF00002EB01107047491C0A29F4DB00207047A1
:106D00002DE9F04105460E4617463046FFF7E8FFED
:106D100004462CB94FF48472944995A0FFF72DF9DD
:106D200046F080002872082239462846FEF741FEC8
:106D30008D48016809B12846884701F03DFE0646A6
:106D400005F10C01201D00F0FFF83046BDE8F041D0
:106D500001F036BE70B50446002C06D1834940F2DE
:106D600033120F3188A0FFF708F97F48416809B155
:106D7000204688470020207201F01EFE054604F1DF
:106D80000C0000F0E8F82846BDE8704001F018BE9D
:106D90002DE9F04106460F4601F00EFE0446FEF7CF
:106DA00029FD58B171497DA02031FFF729F86F49BD
:106DB0004FF4AB72203183A0FFF7DFF8204601F0DB
:106DC000FFFD3046FFF78CFF0546280006D16749D6
:106DD0004FF4AD72203166A0FFF7CFF8E868FFF7F7
:106DE000F2F90446FCB100212046EA68FEF734FDC2
:106DF000267200206072082239462046FEF7D9FD2F
:106E00005948016809B12046884701F0D5FD06467A
:106E100004F10C01281D00F097F8304601F0D0FD78
:106E20002046BDE8F0810020FBE770B50446002C49
:106E300006D14E494FF4CA72333153A0FFF79DF883
:106E4000207A000606D5494940F2951233315EA0FA
:106E5000FFF793F84448416809B12046884700206D
:106E6000207201F0A9FD054604F10C0000F073F852
:106E7000284601F0A5FD2046BDE87040FFF769BA3D
:106E800010B50446002C06D138494FF4DB7244316A
:106E90003DA0FFF772F8207A000601D5012010BD51
:106EA000002010BD10B50446002C06D12F4940F239
:106EB000C9125E3134A0FFF760F8207A20F080001C
:106EC00010BD2DE9F04107460C46002F01D00B2CD8
:106ED00001D90020A5E701F06FFD0546FEF78AFC09
:106EE00058B122492DA07131FEF78AFF1F4940F2A7
:106EF000E512713133A0FFF740F8284601F060FD3C
:106F000000F065F92046FFF7EBFE054635B9174955
:106F10004FF4F772713116A0FFF72FF86C682D1D32
:106F200008E0A4F10C06082239463046FEF754FD6D
:106F300030B12468AC42F4D100F054F9002070E77D
:106F400000F050F930466CE70268516002680A6050
:106F5000016048607047D0E900215160D0E900121B
:106F600011604060006070475001002074CB000841
:106F7000696E666F726D6174696F6E20213D20527B
:106F8000545F4E554C4C00006F626A65637420215B
:106F90003D2052545F4E554C4C00000046756E63C8
:106FA00074696F6E5B25735D207368616C6C206E15
:106FB0006F74206265207573656420696E20495383
:106FC000520A00003000000021286F626A65637475
:106FD0002D3E7479706520262052545F4F626A6599
:106FE00063745F436C6173735F5374617469632985
:106FF000000000008849C860704710B50446002CA6
:1070000004D15922854986A0FEF7B7FFA06A01780E
:10701000232906D1E169814203D9E26A02448A4206
:107020000AD2214683A0FEF7EBFE02F062FC01F0DB
:10703000C3FC0028FDD110BD20308142FBD8214681
:10704000BDE8104082A0FEF7DBBE10B5724B0024F5
:107050005C8000208C4A02EBC00149600960401C42
:107060002028F8DB1F2018705C609C606A48103094
:107070004060006010BD10B5674CA068FEF759FF76
:10708000401E814951F8300014386060BDE810405E
:107090001C3001F0C6BC2DE9F04101F08DFC074623
:1070A0005D4E708820B13846BDE8F04101F088BCE3
:1070B000B068FEF73EFF401E734951F83040143C63
:1070C0007568AC4225D030707460F26812B1214608
:1070D000284690472046FFF790FF6C48007850B153
:1070E00004F11C0105F11C0001F06DFC3846BDE8FF
:1070F000F04101F065BC04F11C0105F11C0001F038
:1071000062FC384601F05CFCBDE8F041012000F073
:10711000C0B83846BDE8F04101F052BC10B5044695
:10712000002C06D13D494FF491721A313CA0FEF774
:1071300024FF01F041FC024614F8340F20F00F0048
:10714000401C207060785049343C01EBC00104F1D0
:1071500014004B6818604B684360486001602E481B
:10716000A16B836819438160BDE81040104601F0AF
:1071700027BC70B50546002D06D128494FF4A872EA
:10718000343127A0FEF7F9FE01F016FC014605F1A7
:107190001404D4E900205060D4E900021060646057
:1071A000246095F83500384A02EBC000026882423C
:1071B00001D1012000E0002020B11748AB6B8268AC
:1071C0009A438260BDE87040084601F0F9BB10B5F3
:1071D00001F0F2FB104A5188491C5180BDE8104073
:1071E00001F0EEBB10B501F0E7FB0B4A5188491ED8
:1071F00009B25180002906DC0021518001F0E0FB3A
:10720000BDE8104047E7BDE8104001F0D9BB024897
:10721000408880B27047000004020020F4CB0008D0
:1072200074687265616420213D2052545F4E554C54
:107230004C0000007468726561643A2573207374B1
:1072400061636B206F766572666C6F770A00000071
:107250007761726E696E673A20257320737461637B
:107260006B20697320636C6F736520746F20656E8B
:1072700064206F6620737461636B2061646472655F
:1072800073732E0A00000000840500201001002006
:1072900070472DE9F047814600F0E8FD044601F013
:1072A0008BFB8046D4E91101084232D094F83400B7
:1072B00080061ED52DE0656DFDB1A86808B30838BD
:1072C00060652E88206D50F82670404601F078FBEE
:1072D0000FB13046B84701F06FFB80460121606C6A
:1072E000B140884360646FF008062846FFF73CFC15
:1072F0002663D4E911010842DDD1B9F1010F03D0B1
:1073000007E000206065DCE714F8340F20F010007F
:1073100020704046BDE8F04701F052BB10B500F0C8
:10732000A5FD04460020FFF7B4FF01F045FBE06C2B
:10733000E0610020E06494F8340020F0100084F84C
:10734000340004F11C00BDE8104001F06ABB70B5C8
:107350000446D4E9110108423CD001F02DFB05465A
:1073600094F8340000F00F0002280FD000F07EFDEA
:10737000A0421AD114F8340F40F0100020702846B3
:1073800001F01EFBBDE87040012082E7204600F0BE
:1073900070FD14F8340F40F010002070284601F002
:1073A0000FFBBDE87040FFF776BE1C34207E40F036
:1073B00010002076226822630023203A1946D9481B
:1073C00001F048F82060284601F0FAFABDE8704064
:1073D000FFF761BE70BD70B505468020FEF7F3FE75
:1073E0000446200005D14FF4B672CF49CFA0FEF776
:1073F000C4FD0021D24844F82100491C2029FADBB1
:1074000001F0DAFA2C65BDE8704001F0D9BA2DE937
:10741000F04104460D46002700F028FD0646202CCA
:1074200002D3B81EBDE8F081FFF7D1FE306D10B970
:107430003046FFF7D0FF306D38B150F82470E91CAA
:1074400007D0691C09D040F82450FFF7CBFE38461E
:10745000E8E7002140F82410F7E7B94940F8241084
:10746000F3E770B5054600F001FD044601F0A4FA0B
:107470000122A16CAA409143A164BDE8704001F0D3
:107480009FBA70B5054600F0F1FC044601F094FA8D
:107490000122A16CAA401143A164626C114205D083
:1074A00001F08EFA2046BDE8704050E7BDE870401C
:1074B00001F086BA2DE9F74F82B0064688460027CC
:1074C00000F0D4FC0446002501F076FA814600F075
:1074D000CDFC50B994499BA00F39FEF791FC92491D
:1074E000D7220F39A5A0FEF748FD01F065FA8246C4
:1074F000FEF780F950B18C49A1A00F39FEF780FC4E
:107500008949D7220F399DA0FEF737FD504601F07B
:1075100057FA484601F054FAF6B33068E0B3B8F1D0
:10752000000F3DD04FF0000AC8F800A0C8F804A032
:1075300001F042FA8146606C316808422AD1049811
:107540006FF0010B48B3204600F054FE94F834006D
:1075500040F0200084F834000498401C09D004F165
:10756000600004AA0021019000F09DFA019800F04B
:10757000DCF9484601F024FAFFF78DFD01F01CFA12
:10758000814694F8340020F0200084F83400206B09
:10759000801C0AD0606D01E002E004E0012327E0D6
:1075A0006FF0090729E05F4624E0C4F830A04846A0
:1075B00001F006FA5F4620E00288D6F800C003FA20
:1075C00002F111EA0C0F10D0D0E90016C8E900163C
:1075D00015B18168A96001E081686165616C9340C3
:1075E00099436164FFF7C0FA04E0054680680838F3
:1075F0000028E1D1484601F0E3F905B03846BDE87E
:10760000F08F70B5054601F0D7F96C6D0021696502
:107610002E6D296501F0D4F93CB10834A4F10800BD
:10762000FFF7A2FA2468002CF8D1002E04D03046CF
:10763000BDE87040FEF78DBE70BD2DE9FC410546EA
:107640000E46002D06D138494FF4D172143156A0A0
:10765000FEF793FC202E03D36FF00900BDE8FC81F8
:10766000ADF800600124ADF802400027019701F059
:10767000A3F9696CB440214219D06C6D01F0A0F9F6
:10768000FFF7A5FD0CE0A4F108000188B14206D186
:10769000DDE9001206C0FFF7A5FD0020DEE7246843
:1076A000002CF0D1FFF79EFD01F086F901E02143A7
:1076B000696401F085F9404800210068FFF7CEF9C0
:1076C0000446200017D0A760DDE90001C4E90001ED
:1076D00001F072F90246696D11B10831083402E017
:1076E0006C6505E0014608680028FBD10C60276046
:1076F000104601F065F92846FFF729FE0020ADE7A6
:1077000010B50C2220212DA0FFF703F92A490860AB
:1077100030B905494FF4F772233118A0FEF72DFC5C
:10772000002010BD1D73000851CC000876656374FD
:107730006F727320213D2052545F4E554C4C000017
:107740009172000846756E6374696F6E5B25735D98
:10775000207368616C6C206E6F7420626520757395
:107760006564206265666F72652073636865647521
:107770006C65722073746172740A0000300000003E
:1077800046756E6374696F6E5B25735D2073686107
:107790006C6C206E6F74206265207573656420695F
:1077A0006E204953520A000074696420213D205222
:1077B000545F4E554C4C00001C0200207369676EEC
:1077C000616C0000F9494860704710B5029C24F0D4
:1077D00001044472C161026200218162436200EBD4
:1077E000C102143252601260491C0129F7DB10BD3E
:1077F00010B50446204600F04DFA10B14FF0FF30AE
:1078000010BD2068406910BD2DE9F8430546DDE94B
:107810000894884616461F46002D04D1BC22E44930
:10782000E4A0FEF7AAFB424609212846FFF768FAC2
:107830004B463A46314628460094FFF7C6FFBDE85E
:10784000F88370B50446002C05D1D949D1220E31F8
:10785000D8A0FEF792FB2046FFF724FB092805D0AD
:10786000D349D2220E31D8A0FEF787FB2046FFF77E
:1078700007FB28B9CE49D3220E31E2A0FEF77DFBEB
:1078800001F09AF80546204600F00BFA284601F070
:1078900097F82046FFF75EFA002070BD2DE9F84307
:1078A0000E46089D1746984601460920FFF770FAD4
:1078B000044644B143463A46314620460095FFF718
:1078C00084FF2046BBE70020B9E770B50446002CD2
:1078D00006D1B7494FF488721E31B6A0FEF74DFBB2
:1078E0002046FFF7DFFA092806D0B14940F211120D
:1078F0001E31B5A0FEF741FB2046FFF7C1FA30B1BB
:10790000AB494FF489721E31C9A0FEF736FB01F076
:1079100053F80546204600F0C4F9284601F050F817
:107920002046FFF782FA002070BD2DE9F843044697
:10793000002C06D19E494FF49A722E319DA0FEF77D
:107940001CFB2046FFF7AEFA092806D0984940F202
:1079500035122E319CA0FEF710FB01F02DF80546E4
:10796000204600F09EF9607A20F0010060722846FF
:1079700001F026F8BC48016809B120468847606AD2
:107980006FF00045A84206D3894940F245122E31D6
:10799000B6A0FEF7F2FAFBF7C0FD616A0844A062E8
:1079A00001F00AF80746DFF8048208F10808CDF86C
:1079B000008000226E4608EBC200D0F804C00BE045
:1079C0000068A0EBC201A36A4969994202D0C91AB2
:1079D000A94205D346F8220056F822006045EFD1AF
:1079E0002AB156F822100831531C46F82310521CB5
:1079F000002AE0D06D48D0F8008008F10108C0F8F6
:107A0000008004F11401009800F0C9F802250EE08E
:107A10005FEA88700DD1C5F1010004EBC00114319B
:107A200056F8200000F0BBF84FEA98086D1C012DB5
:107A3000EED9607A40F001006072384600F0C0FF75
:107A40000020FCE670B50446002C06D1584940F2EF
:107A5000AD123D3157A0FEF790FA2046FFF722FA0B
:107A6000092806D052494FF4D7723D3156A0FEF78F
:107A700084FA607AC00713D08548016809B12046AE
:107A8000884700F099FF0546204600F00AF928468D
:107A900000F096FF607A20F001006072002070BD57
:107AA0004FF0FF3070BD70B504460D461646002CF1
:107AB00006D13F494FF4E8724B313EA0FEF75DFA24
:107AC0002046FFF7EFF9092806D0394940F2D112D4
:107AD0004B313DA0FEF751FA4DB1012D04D0022DDE
:107AE00008D0032D0FD10AE0606A30600BE03068E7
:107AF000606208E0607A20F00200607203E0607A61
:107B000040F002006072002070BD2DE9F041FBF7EB
:107B100004FD074600F050FF0646244D25E02348AB
:107B200008300468143C6FF00041A06A381A88429B
:107B300021D2696809B120468847204600F0B1F893
:107B4000D4E907108847FBF7E8FC0746607A81070D
:107B500008D5C10706D020F0010060722046FFF76B
:107B6000E4FE02E020F0010060721048083000F0EE
:107B700091F80028D3D03046BDE8F04100F020BF96
:107B80000A48083034E60020084A083202EBC001F7
:107B900049600960401C0028F8D0704770470268AF
:107BA000516002680A60016048607047200200204E
:107BB0008ACC000874696D657220213D2052545FA3
:107BC0004E554C4C0000000072745F6F626A656332
:107BD000745F6765745F74797065282674696D6574
:107BE000722D3E706172656E7429203D3D205254A5
:107BF0005F4F626A6563745F436C6173735F54695E
:107C00006D65720072745F6F626A6563745F697339
:107C10005F73797374656D6F626A65637428267427
:107C2000696D65722D3E706172656E742900000089
:107C300072745F6F626A6563745F69735F7379738F
:107C400074656D6F626A656374282674696D657208
:107C50002D3E706172656E7429203D3D2052545F47
:107C600046414C53450000005C01002074696D657D
:107C7000722D3E696E69745F7469636B203C20529B
:107C8000545F5449434B5F4D4158202F2032000030
:107C9000600100200168814201D1012085E70020B8
:107CA00083E710B5002200EBC2011431D1E9004393
:107CB0006360D1E90034236049600960521C012AE5
:107CC000F1DB10BDE44908607047E3494860704744
:107CD000E1498860704770B5E048046800F06CFEC8
:107CE00005462046FFF745FA042084F8340004F1E5
:107CF0006000FFF7A6FD2046FFF7C2F8012802D179
:107D0000D4F88C0058B104F11401D54800F05CFBA4
:107D1000284600F055FEBDE87040FFF7BCB920468C
:107D2000FFF718F8F4E710B50446002C05D140F22F
:107D3000EB22CC49CCA0FEF720F994F8340000F0F7
:107D40000F00022805D04FF43B72C649CBA0FEF7C6
:107D500014F92046FFF7A6F828B140F2ED22C149F8
:107D6000D548FEF70AF96FF00100206304F1140012
:107D700000F031FB2046FFF7D1F9BDE81040FFF7D6
:107D80008AB92DE9FC4109A91F4662C9089B04462E
:107D900004F114004060006022626762A362E16245
:107DA0000A4623211846FDF757FDD4E90A01421877
:107DB000121FAFF2DD03D4E9080100F04BFBE061D4
:107DC000202D05D3A7499E229839BCA0FEF7D5F8EF
:107DD0003034A57165710025A560A662E662256054
:107DE0002571E5652566303C00952346AFF2C90252
:107DF000214604F160000195FFF706FDA564656466
:107E0000E564256565659448816809B12046884721
:107E10000020BDE8FC812DE9FF5F0746DDE90F8604
:107E2000119D0E9C894692469B46002F05D18D4997
:107E3000EE2288398CA0FEF7A0F82CB98949EF22F0
:107E40008839A7A0FEF799F84A4600213846FEF780
:107E500057FFCDE901865B465246494638460395B1
:107E60000094FFF78EFF04B0BDE8F09F7B480068E8
:107E7000704770B50446002C06D17A4940F2BE2204
:107E8000113979A0FEF779F82046FFF70BF830B1E9
:107E9000744940F2BF2211398748FEF76EF894F812
:107EA000340000F00F00022802D04FF0FF3070BD08
:107EB00000F082FD054604F1140000F08CFA04F194
:107EC0006000FFF7BFFD284600F07AFD2046FFF76F
:107ED00025F96148416809B120468847002070BDF6
:107EE00010B50446002C06D15E494FF48A727939E8
:107EF0005DA0FEF742F894F83400000706D0594917
:107F000040F2151279397CA0FEF737F82046FEF7CB
:107F1000C9FF30B153494FF48B7279396648FEF787
:107F20002CF83434A0786070012181406160022017
:107F300004F834092046FFF79CFFFFF797FF08B1CC
:107F4000FFF7A9F8002010BD70B50446002C06D13B
:107F5000444940F24112673943A0FEF70EF820462B
:107F6000FEF7A0FF30B13F494FF4A1726739524884
:107F7000FEF703F82046FEF783FF30B9394940F297
:107F8000431267396AA0FDF7F8FF94F83400000740
:107F900002D02046FFF7EDF804F16000FFF751FC36
:107FA000042084F834002046FEF7D4FED4F88C0078
:107FB00050B100F001FD054604F11401284800F01D
:107FC00003FA284600F0FCFC002070BD2DE9FF47B5
:107FD0008046DDE90C67894692461D4641460020F1
:107FE000FEF7D6FE044620000FD02846FEF7EBF839
:107FF00068B18DE8E10053464A4641462046FFF706
:10800000C0FE204604B0BDE8F0870020FAE7204615
:10801000FEF70BFF0020F5E770B50446002C06D1F3
:10802000104940F2A51256390FA0FDF7A6FF2046D1
:10803000FEF738FF30B10B494FF4D37256391E4862
:10804000FDF79BFF2046FEF71BFF20B1054940F2DC
:10805000A712563984E086E0300200200802002092
:10806000140200207ECD00087468726561642021CE
:108070003D2052545F4E554C4C00000028746872ED
:108080006561642D3E7374617420262052545F54E0
:1080900048524541445F535441545F4D41534B292D
:1080A000203D3D2052545F5448524541445F535552
:1080B0005350454E4400000030D200087072696F82
:1080C00072697479203C2052545F544852454144AF
:1080D0005F5052494F524954595F4D41580000007A
:1080E000737461636B5F737461727420213D2052FD
:1080F000545F4E554C4C0000287468726561642DC5
:108100003E7374617420262052545F544852454196
:10811000445F535441545F4D41534B29203D3D2012
:1081200052545F5448524541445F494E49540000FF
:1081300072745F6F626A6563745F69735F7379738A
:1081400074656D6F626A656374282872745F6F620C
:108150006A6563745F7429746872656164290000DC
:10816000A1A0FDF70AFF94F83400000702D02046D2
:10817000FEF7FFFF04F16000FFF763FB042084F8C3
:10818000340000F019FC054604F11401A54800F084
:108190001BF9284600F014FC002070BD70B500F0FB
:1081A0000BFC0646A048046894F8340000F00F0069
:1081B00001281AD1D4E90501884216D004F114002F
:1081C000054600F008F994F83500984901EBC00025
:1081D00041680D604168696045602860304600F084
:1081E000EFFBFEF758FF002070BD304600F0E8FBC3
:1081F000002070BD70B50446002C06D18C4940F2B9
:108200009322AFF29C10FDF7B8FE2046FEF74AFE1F
:1082100028B14FF4257286498648FDF7AEFE94F8E2
:10822000340000F00F00012802D04FF0FF3070BD85
:1082300000F0C2FB054694F8340020F00F00801CCB
:1082400084F834002046FEF794FF04F16000FFF745
:10825000F9FB284600F0B4FB7748016809B12046D5
:108260008847002070BDF1B500F0A6FB05466E48BA
:1082700004683CB96E4940F2FF122239AFF218206F
:10828000FDF77BFE2046FEF70DFE30B168494FF446
:10829000007222396748FDF770FE2046FFF7AAFFFB
:1082A00004F160006A4600210646FFF7FCFB3046F9
:1082B000FFF73BFB284600F083FBFEF7ECFE206B4C
:1082C000801C00D120630020F8BDCCE710B5FBF77F
:1082D00044F9BDE81040C6E72DE9F04104460D46DB
:1082E0001646002C07D152494FF411721239AFF2E1
:1082F0008820FDF742FE2046FEF7D4FD30B14C4900
:1083000040F2452212394B48FDF737FE25B3012DC7
:1083100026D0022D11D100F04FFB074694F834000F
:10832000012500F00F0001280AD0307884F83500CC
:108330008540A563384600F043FB0020BDE8F0818E
:108340002046FEF716FF307884F835008540A56397
:108350002046FEF7E3FEEDE72046BDE8F041BFE52D
:108360002046BDE8F04157E62DE9F0410746FFF70A
:108370007DFD08B1FEF72BFF0020FEF7B1FC05469E
:1083800035B92B4940F2123235312CA0FDF7F5FDFD
:108390006C682D1D08E0A4F10C0608223946304611
:1083A000FDF71AFB48B12468AC42F4D1FFF75EFD3B
:1083B00008B1FEF717FF0020C0E7FFF757FD08B12F
:1083C000FEF710FF3046B9E70268516002680A60A4
:1083D000016048607047D0E900215160D0E9001287
:1083E000116040600060704772745F6F626A65631D
:1083F000745F69735F73797374656D6F626A6563C7
:1084000074282872745F6F626A6563745F7429747C
:10841000687265616429203D3D2052545F46414C9D
:1084200053450000140200200802002084050020AB
:108430005BCD000830D2000830020020696E666F04
:10844000726D6174696F6E20213D2052545F4E55EC
:108450004C4C000070B50646121D22F00700A0F13A
:10846000400528460022A14C40F82240521C102A08
:10847000FAD30162002141628162C16201634363F8
:1084800086634FF08071C163284670BD98490860CB
:10849000704710B597A0FDF7B3FC9A4C21889AA0BD
:1084A000FDF7AEFC2088C00702D09DA0FDF7A8FC18
:1084B0002088800702D59DA0FDF7A2FC20884007F8
:1084C00002D59DA0FDF79CFC2088000702D59CA04A
:1084D000FDF796FC2088C00502D59BA0FDF790FC17
:1084E0002088800502D59BA0FDF78AFCBDE81040DE
:1084F00083A0FDF785BC10B599A0FDF781FC814CE8
:10850000641E217899A0FDF77BFC2078C00702D07B
:108510009CA0FDF775FC2078800702D59CA0FDF794
:108520006FFC2078400702D59CA0FDF769FC2078FD
:10853000000702D59DA0FDF763FC2078C00602D598
:108540009DA0FDF75DFC2078000607D56D480E3034
:108550000168BDE810409AA0FDF752BCBDE810408C
:1085600067A0FDF74DBC10B599A0FDF749FC654C1F
:10857000A41E21789BA0FDF743FC2078C00702D001
:108580009EA0FDF73DFC2078800702D59EA0FDF758
:1085900037FC2078000702D59EA0FDF731FC20783B
:1085A000C00602D59EA0FDF72BFC2078000607D55B
:1085B00054480A300168BDE810409CA0FDF720BC7B
:1085C000BDE810404EA0FDF71BBC10B54D4CA41CDF
:1085D0002068800702D599A0FDF712FC20684000B2
:1085E00010D54848401E007808B1FFF784FF454881
:1085F000801E007808B1FFF7B6FF4248008808B136
:10860000FFF747FF2068002804DABDE8104091A07A
:10861000FDF7F6BB10BD70B505462C1D344801684A
:10862000002903D028468847002851D08DA0E16B4F
:10863000FDF7E6FB8FA0216AFDF7E2FB91A0616ADE
:10864000FDF7DEFB93A0A16AFDF7DAFB95A0E16AD6
:10865000FDF7D6FB97A02168FDF7D2FB99A06168D2
:10866000FDF7CEFB9BA0A168FDF7CAFB9DA0E168CA
:10867000FDF7C6FB9FA02169FDF7C2FBA1A06169C0
:10868000FDF7BEFBA3A0A169FDF7BAFBA5A0E169B8
:10869000FDF7B6FBA7A0216BFDF7B2FBA9A0616BAC
:1086A000FDF7AEFBABA0A16BFDF7AAFB2878400756
:1086B00008D5FFF7DBFB0146AAA0FDF7A1FB01F0FF
:1086C00018F902E0AFA0FDF79BFBFFF77EFFFEE786
:1086D00070BD10B5B2A0FDF793FBBDE810404FF49C
:1086E000B072B349B3A0FDF748BC0000EFBEADDEE9
:1086F0003C0200207573616765206661756C743A91
:108700000A0000002AED00E05343425F4346535203
:108710005F554653523A30782530325820000000D9
:10872000554E444546494E5354522000494E5653E7
:108730005441544520000000494E5650432000004B
:108740004E4F435020000000554E414C49474E4586
:108750004420000044495642595A45524F200000D7
:10876000627573206661756C743A0A005343425F08
:10877000434653525F424653523A3078253032587E
:10878000200000004942555345525220000000008D
:10879000505245434953455252200000494D5052D2
:1087A000454349534552522000000000554E535452
:1087B0004B4552522000000053544B45525220006A
:1087C0005343422D3E424641523A253038580A0022
:1087D0006D656D206D616E616765206661756C7495
:1087E0003A0A00005343425F434653525F4D46539B
:1087F000523A307825303258200000004941434336
:1088000056494F4C200000004441434356494F4CC9
:10881000200000004D554E53544B4552522000004D
:108820004D53544B45525220000000005343422DFB
:108830003E4D4D41523A253038580A006661696C08
:10884000656420766563746F722066657463680A78
:10885000000000006465627567206576656E740AC5
:10886000000000007073723A203078253038780AA2
:10887000000000007230303A203078253038780A15
:10888000000000007230313A203078253038780A04
:10889000000000007230323A203078253038780AF3
:1088A000000000007230333A203078253038780AE2
:1088B000000000007230343A203078253038780AD1
:1088C000000000007230353A203078253038780AC0
:1088D000000000007230363A203078253038780AAF
:1088E000000000007230373A203078253038780A9E
:1088F000000000007230383A203078253038780A8D
:10890000000000007230393A203078253038780A7B
:10891000000000007231303A203078253038780A73
:10892000000000007231313A203078253038780A62
:10893000000000007231323A203078253038780A51
:1089400000000000206C723A203078253038780A18
:10895000000000002070633A203078253038780A13
:108960000000000068617264206661756C74206F9D
:108970006E207468726561643A2025730D0A0D0AD1
:108980000000000068617264206661756C74206F7D
:108990006E2068616E646C65720D0A0D0A0000003D
:1089A00073687574646F776E2E2E2E0A00000000B7
:1089B0009FCD000830000000EFF3108072B67047C2
:1089C00080F310887047324A1368012B04D04FF0AF
:1089D000010313602F4A10602F4A11602F484FF097
:1089E000805101607047EFF3108272B62848016829
:1089F00091B14FF0000101602648016829B1EFF301
:108A0000098121E9F00F00680160234909680968BC
:108A1000B1E8F00F81F3098882F310884EF0040E5C
:108A200070471D4908601B494FF000000860184955
:108A30004FF0010008601A484FF47F01D0F8002081
:108A400041EA0201016015484FF08051016015486C
:108A50000068006880F3088861B662B670471EF04F
:108A6000040F14BFEFF30880EFF3098020E9F00F43
:108A700040F804ED14BF80F3088880F3098800B53E
:108A8000FFF7C9FD5DF804EB4EF0040E70470000DF
:108A900048020020400200204402002004ED00E0D3
:108AA00020ED00E008ED00E070B5054614461E46D6
:108AB000002D04D12622714971A0FDF75EFA0CB198
:108AC000042E01D0002070BD286C218882682846C1
:108AD00090476080304670BD70B5054614461E460E
:108AE000002D05D1654935220A3165A0FDF745FA0B
:108AF0000CB1042E01D0002070BD286C6288218842
:108B000044682846A047304670BD70B505461446F7
:108B1000002D05D159494522153159A0FDF72DFAEF
:108B20003CB1286C62882188036828469847002059
:108B300070BD4FF0FF3070BD10B5554B12241C7541
:108B40000024DC611C625C629C62DC62514C1C6330
:108B5000514C5C63514C9C631964DA6301460322F7
:108B60001846FAF7AAFD002010BD2DE9F843064685
:108B70000F4690461D46464C206C002805D13F49C3
:108B80006822223146A0FDF7F8F9206CC4683CB198
:108B900043463A4631463E480095A047BDE8F88333
:108BA0000620FBE770B50546394C226C002A05D13A
:108BB0003249712234313AA0FDF7DFF9226C126993
:108BC00022B12946BDE8704031481047062070BDEB
:108BD00070B505460E462E4C216C002905D127495B
:108BE0007A2247312EA0FDF7C8F9216C4B692BB1D1
:108BF00032462946BDE8704025481847062070BD1A
:108C000070B505460E46224C216C002905D11B4942
:108C10008422593122A0FDF7B0F9216C32461C485C
:108C20000B682946BDE87040184770B505460E46EA
:108C3000174C216C002905D110498B22653118A0F1
:108C4000FDF79BF9216C324611484B682946BDE877
:108C50007040184770B505460D4C226C002A05D1AE
:108C60000649922272310EA0FDF787F9226C29463F
:108C700007489268BDE8704010470000B2CD000878
:108C800070696E20213D2052545F4E554C4C0000BF
:108C900084060020A98A0008D98A00080B8B0008E6
:108CA0005F68775F70696E2E6F707320213D205270
:108CB000545F4E554C4C000070B504460025002C06
:108CC00004D1A122F949FAA0FDF757F92046002165
:108CD000C1640165016C0A681AB100F14401904752
:108CE0000546284670BD2DE9F04104460D46002694
:108CF000002C05D1ED49B4220F31EDA0FDF73DF96F
:108D0000E8056FF0070105D5E08AC00502D40846E2
:108D1000BDE8F081680504D5E08A400501D4084625
:108D2000F6E7680602D4207E400600D54026E8B269
:108D30002083E16C002749B1E90502D540F4807138
:108D40002183208B304320830020E1E7E805F8D51C
:108D5000A06CC0F38F200C30FDF735FA05462800D3
:108D600005D1D249CF220F31D5A0FDF706F905F183
:108D70000C002860A16CC1F38F220021FCF76CFD70
:108D8000AF80EF80AF60E564208B40F48071218379
:108D9000206C4FF480721021436820469847D0E73A
:108DA00070B50446002C05D1C049F6221E31C0A082
:108DB000FDF7E3F8A07E012801D9002070BD208BCB
:108DC000C00518D5E56C35B9B84940F201121E311D
:108DD000BBA0FDF7D2F82846FDF7BBFA0021E164FD
:108DE000208B20F480712183206C4FF4807211213C
:108DF000436820469847002070BD2DE9F0410646A3
:108E000015461C46002E06D1A8494FF48A722E3111
:108E1000A7A0FDF7B2F84CB13046318BC90507D594
:108E200022462946BDE8F04100F00CB900206FE76A
:108E30000646300005D19D493A222F39A5A0FDF7FD
:108E40009CF827460AE0306CC16830468847411CD0
:108E500006D005F8010B641E0A2801D0002CF2D1BF
:108E6000381B55E72DE9F041064614461D46002EF5
:108E700006D18E494FF494723D318DA0FDF77DF8F7
:108E80000DB116B107E0002042E788494E221F3994
:108E900090A0FDF772F82F4611E020780A2807D13C
:108EA000307E400604D5306C0D21826830469047F4
:108EB000306C2178826830469047641C6D1E002D0E
:108EC000EBD1384624E72DE9F04104460D4616461D
:108ED0000027002C06D1754940F237124D3174A09D
:108EE000FDF74BF82046012D10D0022D09D0032D9F
:108EF00011D0016C32464B682946984707463846E0
:108F000006E7E08A40F02000E082F8E7E08A20F0FF
:108F10002000E082F3E7002EF1D07168836CC1F38A
:108F20008F22C3F38F239A4203D0827E0AB1072097
:108F3000EEE63268C0E91121817E0029DFD0016CA4
:108F40000A6831469047DAE72DE9F04105460F46B9
:108F500016469846002D06D1544940F26D125F31F5
:108F60005CA0FDF70AF8284600240475C461046279
:108F70005D4941625D4981625D49C1625D4901634C
:108F80005D4941635D498163C0F83C80B2B23946B6
:108F9000BDE8F041FAF791BB2DE9F0410546C8B2B2
:108FA00001284ED1EC6C34B940494FF4C872753188
:108FB00043A0FCF7E2FF00272DE0E869002840D03D
:108FC000FFF7FAFC0246A088E18888422BD3441AB6
:108FD0002EE0FFF7F1FC0146A28820688654A088A5
:108FE000401C80B2A080AA6CC2F38F22904200D3B2
:108FF000A780A288E08882420AD1401C80B2E0802B
:109000000122A260AA6CC2F38F22904200D3E780B3
:109010000846FFF7D5FC286CC168284688470646F5
:10902000701CD6D1C9E7081AA96CC1F38F210C1A9C
:109030001046FFF7C5FC21462846EA69BDE8F04125
:10904000104765E62DE9F04707460E461546002F06
:1090500005D116496D220F391EA0FCF78EFFAA46D6
:10906000FC6C2CB9114971220F3925A0FCF785FF42
:109070004FF000095BE0FFF79FFC0246E188A08803
:10908000814201D1A06880B1206810F80180491C9C
:1090900088B2E080B96CC1F38F21884201D3A4F873
:1090A0000690A068012839D03AE033E05FCE00088E
:1090B00064657620213D2052545F4E554C4C000093
:1090C00072785F6669666F20213D2052545F4E556D
:1090D0004C4C000073657269616C20213D20525434
:1090E0005F4E554C4C000000B98C0008E78C00081E
:1090F000A18D0008FB8D0008658E0008C78E000852
:1091000072785F6669666F20213D2052545F4E552C
:109110004C4C00001046FFF753FC0AE0C4F80890DE
:109120001046FFF74DFC86F80080761C6D1E002D62
:10913000A1D1AAEB0500BDE8F087000010B501F051
:1091400015F920B1F7A1F94802F068FD03E0F8A194
:10915000F64802F063FDF8A1F44802F03FFDF34841
:1091600010BD38B5F54C2068002804D15E22F449C2
:10917000F4A0FCF702FF4FF0FF3503E0294620681A
:10918000FAF7CBFE206801236A46D0F80802294688
:10919000FAF7B3FB0128F1D19DF8000038BD10B5F6
:1091A000E64C2068002805D1E54969220E31E5A08A
:1091B000FCF7E3FE2068FAF735FF002010BD70B51C
:1091C0000646DE4D2868002805D1DD497C221B318A
:1091D000DCA0FCF7D2FE3046FAF740FA0446200045
:1091E0002BD02868D0F80802A0422CD040F24311BE
:1091F0002046FAF7FCFA002825D12868D0F80802A2
:1092000038B1FAF74BFB28680021D0F80802FAF7CA
:10921000FEFB2868502100F5DB7002F0D4FC2868C2
:10922000002180F8061280F80712C0F80842204694
:10923000BDE87040C849FAF7EABB3146BDE8704066
:10924000C6A0FCF7DDBD70BD10B5BC4C2068002881
:1092500005D1BB49A3222C31BAA0FCF78EFE2068B1
:10926000D0F8080210BD70B50446B44D2968002935
:1092700005D1B349B3223D31B2A0FCF77EFE286888
:1092800080F8214070BD10B5AC4C2068002805D195
:10929000AB49C0224C31ABA0FCF76FFE206890F8C0
:1092A000210000F0010010BD10B50446B3A0FCF78A
:1092B000A7FD01F05BF8012802D1204601F05FF91B
:1092C000FFF73CFF22460146BDE81040ACA0FCF78A
:1092D00097BD10B50446ACA0FCF792FDFFF72EFF3A
:1092E000014604F5DB72A6A0FCF78AFD002010BD44
:1092F00070B5044694F80602002853D0A08C04F5FB
:10930000DB7605282AD35022314604F5B37002F0EB
:1093100078FC10B30025681C00EB800004EB001102
:1093200005EB850004EB001026312630502202F0B8
:1093300031FC6D1C042DEEDB05EB850004EB001009
:1093400026300546502102F03EFC94F806222846BD
:10935000314602F01FFC0520A08423E050B1401EDE
:1093600000EB800004EB001026305022314602F062
:1093700048FCB8B1A08C608400EB800004EB0010C6
:109380002630502102F01FFCA08C94F8062200EB3E
:10939000800004EB00102630314602F0FBFBA08C6D
:1093A000401CA084A08C608470BD644E012730688E
:1093B00080F82170D0F80802002804D1FCF76CFD79
:1093C00008B1FFF7FCFEFFF7B9FEFCF719FD002519
:1093D000FFF7C7FE04461B2C07D0306890F820101A
:1093E000012906D002290DD016E0306880F82070DF
:1093F000EEE75B2C02D080F820500DE0022180F8CF
:109400002010E5E780F82050412C40D0422C5DD060
:10941000442C7CD0432C7BD0002CD9D0FF2CD7D02F
:10942000092C76D07F2C75D0082C73D00D2C72D0DF
:109430000A2CFCD090F80612502901D380F806526D
:1094400090F8071290F80622914265D200F5DB737E
:1094500000F2B710521A0B4408441946FCF746FABA
:10946000306890F8071200F5DB700C54306890F803
:109470002110C90707D090F8071200F5DB700144EE
:1094800043A0FCF7BDFC306890F8074228E1418C0E
:10949000D1B1491E89B2418401EB810100EB011178
:1094A0002631502200F5DB7002F074FB306800F5C5
:1094B000DB7002F09FFB0146306880F8061280F8EE
:1094C0000712FFF706FF83E7458481E7818C428C12
:1094D0000B46491E8A4202DA521C428402E0002BEB
:1094E00086D04184418C502201EB810100EB0111B7
:1094F000263100F5DB7002F04DFB306800F5DB70C3
:1095000002F078FB0146306880F8061205E041E081
:109510004EE060E07AE0B9E0E8E080F80712FFF79B
:10952000D8FE55E76D73682000000000C8060020D3
:1095300066696E73682000003E0000004C02002047
:10954000E5CE00087368656C6C20213D2052545FA5
:109550004E554C4C000000009F91000866696E73E8
:10956000683A2063616E206E6F742066696E6420B5
:109570006465766963653A2025730A000A00000075
:1095800025732573000000001B5B324B0D000000AB
:109590002573000090F80702002894D07EA0FCF705
:1095A0002FFC306890F80712491E80F807120FE769
:1095B00090F8071290F80622914284D200F5DB70F1
:1095C000095C76A0FCF71CFC306890F80712491C77
:1095D00080F80712FCE6002403E06FA0FCF710FC03
:1095E000641C306890F80702A042F6DC306800F591
:1095F000DB70FFF759FE306800F5DB7002F0FAFA15
:10960000316881F8060281F80702E1E690F8072246
:10961000002A86D090F80612491EC9B280F80612B8
:10962000521ED3B280F80732994225D9CA1A00F2E5
:10963000B71100F5DB7019441844FCF757F930688E
:1096400090F8061200F5DB700D54306890F80712A0
:1096500000F5DB70014452A0FCF7D2FB306890F8B3
:10966000074203E04CA0FCF7CBFB641C306890F889
:109670000602A0429BDBF5E74BA0FCF7C1FB30687C
:1096800090F8061200F5DB700D54A1E6FFF730FEEE
:1096900000F06CFE01280FD1306890F82100C0075F
:1096A00003D0AFF22810FCF7ABFB306890F806123D
:1096B00000F5DB7000F031FFFFF740FDFCF7A0FB89
:1096C0003068502100F5DB7002F07DFA306880F8D8
:1096D000065280F807527BE62FA0FCF791FB641C32
:1096E000306890F80602A042F6DC0BE000F5DB7073
:1096F0001454306890F82100C00703D0214627A0F9
:10970000FCF77EFB306890F80612491CC9B280F85D
:10971000061290F80722521C80F807225029B4D371
:1097200080F8065280F8075252E6204A106020481E
:10973000016070471F4A10601F48016070477CB588
:109740001E491F48FFF7F1FF4FF403710120FCF79A
:10975000F5FF1C4D2860C0B10A201421CDE900108E
:109760004FF480530022AFF2BD3117A0FEF72EFC5C
:10977000044600231A4616A12868FAF726FB14B1FE
:109780002046FEF7ADFB00207CBD13A0FCF738FBA4
:109790004FF0FF307CBD0000080000002563000092
:1097A000082573202008000008200800500200202F
:1097B00054020020580200205C02002060DD0008F6
:1097C00014DB00084C020020747368656C6C0000A8
:1097D00073687278000000006E6F206D656D6F72A7
:1097E0007920666F72207368656C6C0A0000000057
:1097F00010B5FAA0FCF704FB002010BD10B5FCF773
:1098000020FB002010BD70B50E46FCF797F805460A
:10981000FDF7DDFC346807E0A4F10C00FCF78EF8DE
:10982000A84200DD05462468B442F5D1FDF7DAFC14
:10983000082D00DC05B90825284670BD2DE9FC413E
:109840000646EBA431462046FFF7DDFF07462246D9
:109850003946E948FCF7D4FA384600F056FCE7A050
:10986000FCF7CEFA35683FE0A5F10C04234694F8E6
:109870003500009008223946F0A0FCF7C1FA94F8B0
:10988000340000F00F00012805D0022807D050B1A5
:1098900004280CD00EE0ECA0FCF7B2FA0AE0EDA030
:1098A000FCF7AEFA06E0EEA0FCF7AAFA02E0EFA0A1
:1098B000FCF7A6FAA06A014600E0401C0278232AC1
:1098C000FBD0E26A401A101A64235843B0FBF2F34B
:1098D000D4F830C0E06DCDE9000CE069081A8118B9
:1098E000E5A0FCF78DFA2D68B542BDD10020BDE89A
:1098F000FC8110B50020FDF7F3F9BDE81040001D14
:109900009CE770B505462C680BE0A4F11401E4A0B7
:10991000FCF776FA2068A84202D0E2A0FCF770FAC1
:109920002468AC42F1D170BD2DE9FC410646DEA4AD
:1099300031462046FFF767FF074622463946DDA03D
:10994000FCF75EFA384600F0E0FBE1A0FCF758FABD
:10995000346814E0A4F10C0505F11400804600F011
:10996000C4FB80B1404600F0C7FBA98BCDE90010D5
:109970002B4608223946DCA0FCF742FA2468B442A0
:10998000E8D10020B3E7404600F0B6FBA98BCDE953
:1099900000102B4608223946D7A0FCF731FA404682
:1099A000FFF7AFFF91A0FCF72BFAE7E710B5012016
:1099B000FDF796F9BDE81040001DB5E72DE9FC4123
:1099C0000646D1A431462046FFF71DFF0746224632
:1099D0003946CFA0FCF714FA384600F096FBD5A024
:1099E000FCF70EFA346810E0A4F10C0505F1140040
:1099F000804600F07AFB60B1E86900902B460822AF
:109A00003946D4A0FCF7FCF92468B442ECD100201C
:109A10006DE7404600F070FBE969CDE900102B4688
:109A200008223946D0A0FCF7EBF94046FFF769FF62
:109A30006EA0FCF7E5F9E7E710B50320FDF750F954
:109A4000BDE81040001DB9E72DE9FF410646CCA452
:109A500031462046FFF7D7FE804622464146CAA03F
:109A6000FCF7CEF9404600F050FBD0A0FCF7C8F957
:109A70003568082712E0A5F10C0404F1140000F089
:109A80003BFBE17F226ACDE90210CDE9007223465B
:109A900008224146CDA0FCF7B3F92D68B542EAD1C2
:109AA000002004B0BDE8F08110B50220FDF718F9E0
:109AB000BDE81040001DC7E72DE9FE430646C9A4D6
:109AC00031462046FFF79FFE074622463946C7A08B
:109AD000FCF796F9384600F018FBCDA0FCF790F99A
:109AE000356816E0A5F10C0404F11400804600F07E
:109AF000FCFA98B1404600F0FFFA218C628CCDE967
:109B000000210290234608223946C8A0FCF778F9C4
:109B10002D68B542E6D10020BDE8FE83404600F046
:109B2000EBFA218C628CCDE90021029023460822B9
:109B30003946C4A0FCF764F94046FFF7E2FE2BA0CB
:109B4000FCF75EF9E4E710B50420FDF7C9F8BDE8BD
:109B50001040001DB0E72DE9FC410646BFA4314688
:109B60002046FFF750FE074622463946BEA0FCF7C6
:109B700047F9384600F0C9FAC2A0FCF741F9346849
:109B800014E0A4F10C0505F11400804600F0ADFAD4
:109B900080B1404600F0B0FAA98CCDE900102B4608
:109BA00008223946BDA0FCF72BF92468B442E8D15D
:109BB00000209CE6404600F09FFAA98CCDE90010F9
:109BC0002B4608223946BAA0FCF71AF94046FFF79F
:109BD00098FE06A0FCF714F9E7E7000048656C6CF6
:109BE0006F2052542D546872656164210A00000090
:109BF000746872656164000074D20008202D2D2DF8
:109C000020202D2D2D2D2D2D2D202D2D2D2D2D2DAB
:109C10002D2D2D2D202D2D2D2D2D2D2D2D2D2D208E
:109C2000202D2D2D2D2D2D20202D2D2D2D2D2D2D8B
:109C30002D2D2D202D2D2D0A00000000252D2A2E42
:109C40002A73202533642000207265616479202006
:109C5000000000002073757370656E6400000000E2
:109C600020696E69742020200000000020636C6F62
:109C700073652020000000002030782530387820DF
:109C80003078253038782020202025303264252572
:109C900020202030782530387820253033640A00A1
:109CA000257300002F00000073656D6170686F728E
:109CB00065000000252D2A2E732076202020737544
:109CC0007370656E64207468726561640A000000D8
:109CD000202D2D2D202D2D2D2D2D2D2D2D2D2D2DCE
:109CE0002D2D2D0A00000000252D2A2E2A73202557
:109CF0003033642025640A00252D2A2E2A7320255E
:109D00003033642025643A006576656E7400000087
:109D1000252D2A2E732020202020207365742020DA
:109D2000202073757370656E642074687265616459
:109D30000A00000020202D2D2D2D2D2D2D2D2D2D17
:109D4000202D2D2D2D2D2D2D2D2D2D2D2D2D2D0A73
:109D500000000000252D2A2E2A732020307825307F
:109D6000387820300A000000252D2A2E2A73202062
:109D700030782530387820253033643A00000000F0
:109D80006D75746578000000252D2A2E7320202023
:109D90006F776E65722020686F6C642073757370C6
:109DA000656E64207468726561640A00202D2D2D33
:109DB0002D2D2D2D2D202D2D2D2D202D2D2D2D2DED
:109DC0002D2D2D2D2D2D2D2D2D0A0000252D2A2E4A
:109DD0002A7320252D382E2A73202530346420251F
:109DE000640A00006D61696C626F7800252D2A2E6F
:109DF0007320656E7472792073697A652073757348
:109E000070656E64207468726561640A0000000009
:109E1000202D2D2D2D20202D2D2D2D202D2D2D2DA6
:109E20002D2D2D2D2D2D2D2D2D2D0A00252D2A2EBC
:109E30002A732025303464202025303464202564A2
:109E40000A000000252D2A2E2A7320253034642094
:109E500020253034642025643A0000006D7367715A
:109E60007565756500000000252D2A2E7320656E2E
:109E70007472792073757370656E6420746872658E
:109E800061640A00202D2D2D2D20202D2D2D2D2D0E
:109E90002D2D2D2D2D2D2D2D2D0A0000252D2A2E79
:109EA0002A732025303464202025640A0000000035
:109EB000252D2A2E2A732025303464202025643A4B
:109EC0000000000010B50520FCF70AFFBDE81040B7
:109ED000001D40E6FEB5054691A429462046FFF741
:109EE00092FC0646224631468FA0FBF789FF30469A
:109EF00000F00BF998A0FBF783FF2C680DE0A4F1AC
:109F00000C03D3E907029969CDE9001202900822F7
:109F100031469CA0FBF774FF2468AC42EFD10020CF
:109F2000FEBD10B50620FCF7DBFEBDE81040001DAD
:109F3000D0E72DE9FF41064699A431462046FFF7B8
:109F400062FC07462246394697A0FBF759FF384680
:109F500000F0DBF89EA0FBF753FF356826E0A5F183
:109F60000C04606BA0B1D4E90931E269CDE90210BB
:109F7000CDE900232346082239469EA0FBF740FF87
:109F800004F12C00FFF7BDFC7DA0FBF739FF0CE0CE
:109F9000D4E90931E269CDE90210CDE90023234675
:109FA000082239469AA0FBF72BFF2D68B542D6D17F
:109FB000002076E510B50720FCF792FEBDE81040C2
:109FC000001DB6E72DE9FC41064698A4314620461F
:109FD000FFF719FC07462246394696A0FBF710FF0B
:109FE000384600F092F89DA0FBF70AFF346816E0AF
:109FF000A4F10C052B46D5E90901CDE900010822A1
:10A0000039469FA0FBF7FCFE687AC00703D0A2A0E8
:10A01000FBF7F6FE02E0A3A0FBF7F2FE2468B442D1
:10A02000E6D1F9F77AFA0146A2A0FBF7E9FE002093
:10A030005DE410B50920FCF753FEBDE81040001D9B
:10A04000C0E7F0B597B005465022A04903A801F03B
:10A05000A1FD9FA429462046FFF7D5FB07462246CF
:10A0600039469DA0FBF7CCFE384600F04EF8A4A080
:10A07000FBF7C6FE2C6803AE11E0A4F10C03187DBB
:10A08000997E132802D856F8200000E01698CDE9F2
:10A09000000108223946A3A0FBF7B2FE2468AC42B7
:10A0A000EBD117B00020F0BD10B50820FCF718FE6A
:10A0B000BDE81040001DC4E770B59FA0FBF7A0FEEF
:10A0C000A2480468A24D0BE00222A2A1206801F080
:10A0D000AEFD20B1D4E900129FA0FBF791FE0C3435
:10A0E00028688442F0D3002070BD0168814201D10C
:10A0F000012070470020704702460020114600E012
:10A10000401C09689142FBD1704710B5044602E03B
:10A1100095A0FBF775FE641E601CF9D110BD000010
:10A120006D656D6865617000252D2A2E7320207085
:10A130006F6F6C2073697A6520206D61782075736C
:10A1400065642073697A6520617661696C61626C0F
:10A15000652073697A650A00202D2D2D2D2D2D2D5A
:10A160002D2D2D202D2D2D2D2D2D2D2D2D2D2D2D2C
:10A170002D202D2D2D2D2D2D2D2D2D2D2D2D2D2D1C
:10A180000A000000252D2A2E2A7320252D3031307B
:10A190006420252D3031336420252D3035640A00AC
:10A1A0006D656D706F6F6C00252D2A2E7320626CAB
:10A1B0006F636B20746F74616C20667265652073C9
:10A1C000757370656E64207468726561640A00005E
:10A1D000202D2D2D2D20202D2D2D2D20202D2D2DF0
:10A1E0002D202D2D2D2D2D2D2D2D2D2D2D2D2D2DAC
:10A1F0000A000000252D2A2E2A73202530346420E1
:10A2000020253034642020253034642025643A0031
:10A21000252D2A2E2A732025303464202025303421
:10A22000642020253034642025640A0074696D653B
:10A2300072000000252D2A2E732020706572696F30
:10A2400064696320202074696D656F757420202017
:10A2500020202020666C61670A000000202D2D2D33
:10A260002D2D2D2D2D2D2D202D2D2D2D2D2D2D2D2B
:10A270002D2D202D2D2D2D2D2D2D2D2D2D2D0A006B
:10A28000252D2A2E2A7320307825303878203078F2
:10A290002530387820000000616374697661746548
:10A2A000640A000064656163746976617465640AB8
:10A2B0000000000063757272656E74207469636BD0
:10A2C0003A3078253038780A0000000040CF000886
:10A2D0006465766963650000252D2A2E7320202091
:10A2E000202020202020747970652020202020202C
:10A2F00020202072656620636F756E740A0000006E
:10A30000202D2D2D2D2D2D2D2D2D2D2D2D2D2D2D8A
:10A310002D2D2D2D2D202D2D2D2D2D2D2D2D2D2D7A
:10A320000A000000252D2A2E2A7320252D32307395
:10A3300020252D38640A00002D2D46756E63746942
:10A340006F6E204C6973743A0A00000050020020BE
:10A35000540200205F5F0000252D313673202D2D23
:10A360002025730A000000002D0000000120704726
:10A3700070B5A5A0FBF744FDAA480468AA4D0CE0FF
:10A380000622AAA1206801F052FC28B9D4E90012E3
:10A39000891DA8A0FBF734FD0C3428688442EFD354
:10A3A000A7A0FBF72DFD002070BD70B51646002359
:10A3B000002400254AE000F8015B5B1C0278202A9B
:10A3C00001D0092A01D18B42F5D30A2C10D39DA0CC
:10A3D000FBF716FD002505E056F82510A1A0FBF7B8
:10A3E0000FFD6D1CA542F7D395A0FBF709FD2FE0EB
:10A3F0008B422DD20278222A03D046F82400641C16
:10A400001BE0401C5B1C46F82400641C08E05C2A2E
:10A4100004D14278222A01D1401C5B1C401C5B1CE9
:10A420000278222A01D08B42F1D38B4210D200F85D
:10A43000015B5B1C0AE0401C5B1C0278202A03D0F5
:10A44000092A01D08B42F6D38B4201D28B42B5D37D
:10A45000204670BD2DE9F0478146884600267148A8
:10A46000046808F10605704F10E006226FA120680D
:10A4700001F0DDFB48B920684246801D494601F0E5
:10A48000D6FB10B92068405D30B10C343868844286
:10A49000EBD33046BDE8F087A668FAE72DE9F04136
:10A4A0008AB005460F4616460024002D05D140F21D
:10A4B00021126D496DA0FBF760FD3EB94FF491721A
:10A4C00069496BA0FBF759FD00E0641C295D202958
:10A4D00003D0092901D0BC42F7D34FF0FF38B4B103
:10A4E00021462846FFF7B6FF044694B12821684666
:10A4F00001F069FB6A4639462846FFF756FF50B11E
:10A500006946A047306000200AB0BDE8F0814046AF
:10A51000FAE74046F8E74046F6E738B5054601E079
:10A520006D1C491E28782028FAD00928F8D031B1AE
:10A530006A462846FFF7B2FF18B12C4604E0002017
:10A5400038BD009838BD641C2078202801D0002830
:10A55000F9D100202070294647A0FBF751FC4FF0AD
:10A56000FF3038BD10B5024601E0521C491C14787A
:10A570001CB10B780BB19C42F7D0101A10BD2DE91D
:10A58000F04781460025002699F80000002804D0F5
:10A5900024480468DFF8908027E0BDE8F0470021F8
:10A5A0000846E5E6062221A1206801F040FBD8B963
:10A5B0002768BF1D484601F01DFB02463946484644
:10A5C00001F035FB80B925B93E46304601F012FB5B
:10A5D000054639463046FFF7C5FFA84200DA054672
:10A5E000394616A0FBF70CFC0C34D8F80000844266
:10A5F000D8D3002E06D02A4631464846BDE8F0475B
:10A60000FBF7D7B946E7000052542D5468726561D4
:10A6100064207368656C6C20636F6D6D616E64732C
:10A620003A0A000050020020540200205F5F636D70
:10A63000645F0000252D313673202D2025730A001C
:10A640000A000000546F6F206D616E79206172679F
:10A65000732021205765206F6E6C79205573653A01
:10A660000A0000002573200090CF0008636D64008D
:10A67000726574700000000025733A20636F6D6D81
:10A68000616E64206E6F7420666F756E642E0A00B2
:10A6900010B5FFF72EF9002010BD0020704710B54F
:10A6A000FCF77FF8002010BD2DE9F04100240127C0
:10A6B00007FA04F52846FBF786FD064666B12946EB
:10A6C00012A0FBF79DFB3046FBF743FE294615A081
:10A6D000FBF796FB641CEBE707FA04F1BDE8F041D9
:10A6E00016A0FBF78DBB1CB505201921CDE9001084
:10A6F0004FF400730022AFF24F0119A0FDF766FC82
:10A7000008B1FDF7EDFB00201CBD0000676574205B
:10A710006D656D6F7279203A256420627974650ADF
:10A720000000000066726565206D656D6F727920AE
:10A730003A256420627974650A00000074727920F9
:10A74000746F206765742025642062797465206DBC
:10A75000656D6F7279206661696C6564210A00001D
:10A7600074687265616431007CB501AC4FF0FF35EF
:10A770002B460622282139480094FAF7C1F818B967
:10A7800037A00199FBF73CFB3DA0FBF739FB4FF4E9
:10A790007A70FDF79BFD2B46052228212F48009457
:10A7A000FAF7AEF818B942A00199FBF729FB48A0C7
:10A7B000FBF726FB7CBD10B549A0FBF721FB082168
:10A7C0002648FAF73BF8C820FDF780FD4AA0FBF7C2
:10A7D00017FB20212148FAF731F8C820FDF776FD54
:10A7E0003FA0FBF70DFB08211C48FAF727F8BDE84E
:10A7F000104047A0FBF704BB7FB5002248A11748D3
:10A80000F9F720FF30B148A0FBF7FAFA4FF0FF301C
:10A8100004B070BD08201149C40105252031CDE9DF
:10A820000205CDE900140023444A45A14648FDF73E
:10A83000F2FA4548FDF754FB434909209431CDE92C
:10A840000205CDE900140023404A41A14248FDF72A
:10A85000E2FA4148FDF744FB0020D9E74C0700200D
:10A86000746872656164313A204F52207265637674
:10A87000206576656E7420307825780A0000000027
:10A88000746872656164313A2064656C6179203165
:10A890007320746F207072657061726520746865D2
:10A8A000207365636F6E64206576656E740A0000C0
:10A8B000746872656164313A20414E442072656368
:10A8C00076206576656E7420307825780A00000061
:10A8D00074687265616431206C656176652E0A006A
:10A8E000746872656164323A2073656E64206576BF
:10A8F000656E74330A000000746872656164323AF0
:10A900002073656E64206576656E74350A000000FC
:10A9100074687265616432206C656176652E0A0028
:10A920006576656E74000000696E697420657665F1
:10A930006E74206661696C65642E0A0069A7000860
:10A9400074687265616431006C0B0020B7A7000861
:10A9500074687265616432000010002010B5294CE3
:10A96000606842F2107190FBF1F201FB12000028C6
:10A9700003D1616824A0FBF743FAFCF728FC606868
:10A98000401C6060BDE81040FCF72CBC2DE9F04194
:10A99000052400261B4D4FF4FA770EE021A0FBF7AB
:10A9A0002FFAFCF714FC6E60FCF71CFC696821A010
:10A9B000FBF726FA3846FDF789FC641E611CEDD1D1
:10A9C00023A0FBF71DFA2748F9F7FCF8BDE8F04192
:10A9D00025A0FBF715BA1CB52248F9F7DBF80520CE
:10A9E0001421CDE900104FF480630022234924A0F4
:10A9F000FDF7ECFA0349086008B1FDF771FA002091
:10AA00001CBD000060020020656E746572206964E0
:10AA10006C6520686F6F6B2025642074696D6573A9
:10AA20002E0A0000656E7465722074687265616438
:10AA3000312E0A00746872656164312064656C614E
:10AA400079203530204F53205469636B2E0A000063
:10AA500064656C6574652069646C6520686F6F6BF4
:10AA60002E0A00005DA900087468726561643120D7
:10AA700066696E6973682E0A000000008DA90008DF
:10AA80007468726561643100054605EB8500184CF9
:10AA90004600FDF791FF216829442160FDF790FFF2
:10AAA000294614A02268FBF7ABF93046FDF70EFCEF
:10AAB000EFE77CB5052414254FF4007633460A22CF
:10AAC000AFF23B01CDE9005413A0FDF77FFA08B1C6
:10AAD000FDF706FA33461422AFF25301CDE90054D4
:10AAE0000FA0FDF773FA08B1FDF7FAF900207CBD5D
:10AAF0006802002070726F746563742074687265F8
:10AB000061645B25645D277320636F756E74657285
:10AB10002069732025640A007468726561643100DD
:10AB2000746872656164320038B5374C4FF0FF3598
:10AB30000DE036A00099FBF763F90098A04203D11D
:10AB40003F48F9F7EDFF38BD6420FDF7BFFB3DA09E
:10AB5000FBF756F92A4669463948FAF7A9F9002859
:10AB6000F5D1E6E710B50024641CE4B2E00705D097
:10AB700025493348491DFAF799F904E0224930483C
:10AB80001131FAF793F9C820FDF7A0FB0A2CEBD39B
:10AB9000BDE810401C492A48FAF788B97FB5002063
:10ABA000274A0090202330322EA12548F9F794FF40
:10ABB00030B12DA0FBF724F94FF0FF3004B070BD89
:10ABC0001F480A264FF48064B0308DE851000525F7
:10ABD00000232B4A2BA1039500F58060FDF71BF99C
:10ABE0002A48FDF77DF92948002394308DE851006B
:10ABF000274A28A1039500F58060FDF70CF9274846
:10AC0000FDF76EF90020D9E76C02002074687265C8
:10AC10006164313A206765742061206D61696C2040
:10AC200066726F6D206D61696C626F782C2074683C
:10AC30006520636F6E74656E743A25730A000000B8
:10AC400094100020746872656164313A20747279DE
:10AC500020746F20726563762061206D61696C0AD3
:10AC6000000000006D627400696E6974206D616996
:10AC70006C626F78206661696C65642E0A00000062
:10AC800029AB0008746872656164310044150020C6
:10AC900065AB00087468726561643200D8190020E1
:10ACA00070B500242F4D661E55F8240050B931466A
:10ACB0002D48FBF7D3FE45F8240018B121462BA000
:10ACC000FBF79EF8641C322CEEDB70BD70B52BA038
:10ACD000FBF796F80024234D002655F8240048B1D0
:10ACE00021462EA0FBF78CF855F82400FBF73CFF1B
:10ACF00045F82460641C322CEFDB70BD7CB500206D
:10AD0000184A002142F82010401C3228FADB50205B
:10AD1000144A00904FF48053C83225A11248FBF723
:10AD200081FD05251920CDE900054FF40076334655
:10AD30000022204920A0FDF749F9214C206008B1EC
:10AD4000FDF7CEF81A20CDE90005334600221D4953
:10AD50001DA0FDF73BF9606008B1FDF7C1F80020C8
:10AD60007CBD00006C1A0020342B0020616C6C6FDD
:10AD700063617465204E6F2E25640A0074687265E5
:10AD80006164322074727920746F2072656C656121
:10AD9000736520626C6F636B0A00000072656C65FE
:10ADA00061736520626C6F636B2025640A0000008C
:10ADB0006D703100A1AC0008746872656164310087
:10ADC00094020020CDAC00087468726561643200A2
:10ADD00038B5002000900024451E2B46012269460C
:10ADE0004148FAF75DFB30B99DF800103FA0FBF732
:10ADF00007F8132C05D0641CE4B23220FDF766FA84
:10AE0000EBE747A0FAF7FCFF3748FAF7B6F938BD89
:10AE100038B5412000900024082C05D0142C13D301
:10AE200045A0FAF7EDFF38BD012269462E48FAF732
:10AE3000CEFA18B14AA0FAF7E3FF13E09DF800102C
:10AE40004CA0FAF7DDFF0DE0012269462648FAF72B
:10AE500052FA10B150A0FAF7D3FF9DF8001052A09B
:10AE6000FAF7CEFF9DF80000401C0090641CE4B28D
:10AE70000520FDF72BFACFE77FB500204FF40061E6
:10AE8000CDE90010184A012334324EA11648FAF7D2
:10AE900039F930B14CA0FAF7B3FF4FF0FF3004B0EE
:10AEA00070BD504819264FF480648DE85100052587
:10AEB00000234D4A4DA1039500F58060FCF7ABFFE0
:10AEC0004C48FDF70DF84B48002394308DE85100B5
:10AED000494A4AA1039500F58060FCF79CFF494868
:10AEE000FCF7FEFF0020DAE76C2B00207468726527
:10AEF0006164313A2072656376206D7367206672F3
:10AF00006F6D206D73672071756575652C20746891
:10AF10006520636F6E74656E743A25630A000000E5
:10AF2000746872656164313A206465746163682095
:10AF30006D71200A000000006D6573736167652004
:10AF400071756575652073746F702073656E642C00
:10AF5000207468726561643220717569740A00003A
:10AF600072745F6D715F757267656E7420455252C1
:10AF70000A000000746872656164323A2073656E7D
:10AF80006420757267656E74206D657373616765A3
:10AF9000202D2025630A000072745F6D715F736558
:10AFA0006E64204552520A00746872656164323AD8
:10AFB0002073656E64206D657373616765202D2055
:10AFC00025630A006D717400696E6974206D657384
:10AFD00073616765207175657565206661696C656B
:10AFE000642E0A00A0330020D1AD00087468726599
:10AFF00061643100A037002011AE000874687265EA
:10B0000061643200343C0020334C4FF0FF35294658
:10B010006068F9F7C2F96078401C60700A20FDF79B
:10B0200055F92078401C20706068F9F75EFAEEE769
:10B0300070B5294C4FF0FF3512E028A0FAF7E0FE7A
:10B0400002E031A0FAF7DCFE6078401C60702078E6
:10B05000401C20706068F9F748FA6078322808D2FE
:10B0600029466068F9F799F9617822789142E8D029
:10B07000E3E770BD7FB500212DA0F9F783F81649ED
:10B08000486018B30820C40105252B49CDE9020505
:10B09000CDE900140023294A29A12B48FCF7BBFE67
:10B0A0002948FCF71DFF284907209431CDE9020506
:10B0B000CDE900140023254A25A12748FCF7ABFE63
:10B0C0002548FCF70DFF002004B070BD23A0FAF75F
:10B0D00097FE4FF0FF30F7E79C0200206E6F742060
:10B0E00070726F746563742E6E756D626572312057
:10B0F0003D2025642C206D756D62657232203D20E7
:10B100002564200A000000006D7574657820707257
:10B110006F74656374202C6E756D62657231203DAD
:10B12000206D756D626572322069732025640A0096
:10B13000646D757465780000C83C002009B0000893
:10B140007468726561643100C840002031B0000845
:10B1500074687265616432005C45002063726561E9
:10B1600074652064796E616D6963206D75746578AE
:10B17000206661696C65642E0A00000010B56420C9
:10B18000FDF7A4F84A4C606890F83510A06890F874
:10B19000350081420DD047A0FAF732FEA06890F842
:10B1A00035104CA0FAF72CFEBDE8104051A0FAF77C
:10B1B00027BE40A0FAF724FEA06890F8351045A0FD
:10B1C000FAF71EFEBDE810404EA0FAF719BE10B502
:10B1D000374C606890F8351036A0FAF711FE32202F
:10B1E000FDF774F84FF0FF31E068F9F7D6F8002862
:10B1F00004D1E068BDE81040F9F777B910BD70B52B
:10B200002B4DA86890F8351032A0FAF7F9FD4FF0F1
:10B21000FF31E868F9F7C1F810B13DA0FAF7F0FD89
:10B22000F8F77BF90446F8F778F9001B3228FAD3CF
:10B23000E868BDE87040F9F758B97CB500213CA03A
:10B24000F8F7A0FF1A4CE06058B305250920CDE9B6
:10B2500000054FF4007633460022374937A0FCF74B
:10B26000B5FE206008B1FCF73BFE0A20CDE90005E1
:10B2700033460022334934A0FCF7A8FE606008B1D1
:10B28000FCF72EFE0B20CDE90005334600223049A5
:10B2900030A0FCF79BFEA06008B1FCF721FE002067
:10B2A0007CBD2EA0FAF7ACFD4FF0FF307CBD000056
:10B2B000A4020020746865207072696F72697479E5
:10B2C000206F6620746872656164322069733A2069
:10B2D00025640A00746865207072696F72697479F8
:10B2E000206F6620746872656164332069733A2048
:10B2F00025640A0074657374206661696C65642E48
:10B300000A00000074657374204F4B2E0A00000081
:10B31000746872656164332074616B652061206DAF
:10B32000757465782C206661696C65642E0A00006E
:10B330006D757465780000007DB1000874687265F1
:10B3400061643100CFB100087468726561643200D5
:10B35000FFB10008746872656164330063726561EF
:10B3600074652064796E616D6963206D75746578AC
:10B37000206661696C65642E0A0000002DE9F041C9
:10B3800000245F4E5F4F4FF0FF3805255D48414672
:10B390003430F8F7C2FD5B4841461430F8F7BDFD84
:10B3A000B068B0FBF5F105FB1102611C47F82210F3
:10B3B000B0FBF5F105FB110057F8201052A0FAF789
:10B3C0001FFDB068401CB0604E481430F8F72AFEEC
:10B3D0004C485430F8F726FE641C1420FCF776FF26
:10B3E0000A2CD3DBBDE8F04151A0FAF709BD2DE9E5
:10B3F000F0410026424D434F4FF0FF3805244148AD
:10B4000041465430F8F789FD3E4841461430F8F77C
:10B4100084FDE868B0FBF4F104FB110157F821103A
:10B420000E44B0FBF4F104FB110157F82120B0FBEE
:10B43000F4F104FB110143A0FAF7E2FCE868401CB8
:10B44000E86030481430F8F7EDFD2E483430F8F756
:10B45000E9FDE8680A2803D03220FCF737FFCEE781
:10B46000314641A0FAF7CCFCBDE8F04145A0FAF71F
:10B47000C7BC2DE9FC41224C0020A060E0602148BF
:10B480000023012244A11430F8F79FFC1D4800233B
:10B49000052243A13430F8F798FC1A4800231A46D5
:10B4A00041A15430F8F791FC05264FF4007700963F
:10B4B0003B460022AFF23B113DA00196FCF786FD12
:10B4C0002060B51F90B1FCF70BFD07203B46002222
:10B4D000AFF2E501CDE9000638A0FCF777FD60602A
:10B4E00048B1FCF7FDFC0020BDE8FC8136A0FAF76E
:10B4F00087FC2846F8E73CA0FAF782FC2846F3E7E9
:10B50000B4020020F04500207468652070726F64FA
:10B51000756365722067656E65726174657320611D
:10B52000206E756D6265723A2025640A0000000085
:10B530007468652070726F647563657220657869E0
:10B5400074210A0074686520636F6E73756D65728F
:10B550005B25645D206765742061206E756D626592
:10B56000723A2025640A000074686520636F6E7368
:10B57000756D65722073756D2069733A2025640AB4
:10B580000000000074686520636F6E73756D6572EE
:10B590002065786974210A006C6F636B00000000FD
:10B5A000656D70747900000066756C6C00000000B9
:10B5B00070726F647563657200000000636F6E7374
:10B5C000756D6572000000006372656174652074BA
:10B5D00068726561642070726F647563657220665D
:10B5E00061696C6564000000637265617465207454
:10B5F000687265616420636F6E73756D6572206635
:10B6000061696C656400000004464FF47A75214658
:10B6100017A0FAF7F5FB2846FCF758FEF7E70A46AD
:10B62000014619A0FAF7ECBB7CB51D48FBF7E2FC1C
:10B630000A201425CDE900504FF4806633460122DC
:10B64000184919A0FCF7C2FC194C206008B1FCF79E
:10B6500047FC0520CDE9005033460222114915A0D0
:10B66000FCF7B4FC606008B1FCF73AFC00207CBD3C
:10B670007468726561642025642069732072756E38
:10B680006E696E670A00000066726F6D3A2025735E
:10B69000202D2D3E2020746F3A202573200A0000B3
:10B6A0001FB6000809B6000874687265616431004D
:10B6B000C4020020746872656164320070B5344D54
:10B6C0000A240DE0401CC0B22870B0FBF4F104FB6A
:10B6D000110028B92FA0FAF793FB6868F8F7A2FCCD
:10B6E00028786428EED970BD70B5294C4FF0FF352D
:10B6F0000EE031A0FAF784FB6068BDE87040F8F70F
:10B70000CDBB6078401CC1B2617035A0FAF778FB00
:10B7100029466068F8F701FCA0600028F1D0E8E74E
:10B720007FB50022114639A0F8F791FB184948600F
:10B73000002827D037A0FAF763FB052519204FF41E
:10B7400080643F49CDE90205CDE9001400233D4A5C
:10B750003DA13F48FCF75FFB3D48FCF7C1FB3C497E
:10B7600018209431CDE90205CDE900140023394AAF
:10B7700039A13B48FCF74FFB3948FCF7B1FB0020EF
:10B7800004B070BD37A0FAF73BFB4FF0FF30F7E78E
:10B79000CC02002074312072656C65617365206194
:10B7A0002064796E616D69632073656D6170686F87
:10B7B00072652E0A0000000074322074616B6520EF
:10B7C000612064796E616D69632073656D61706875
:10B7D0006F72652C206661696C65642E0A0000003A
:10B7E00074322074616B6520612064796E616D69CB
:10B7F000632073656D6170686F72652E206E756D64
:10B80000626572203D2025640A0000006473656D46
:10B810000000000063726561746520646F6E652EC0
:10B820002064796E616D69632073656D6170686F06
:10B8300072652076616C7565203D20302E0A00000F
:10B8400064460020BDB6000874687265616431000A
:10B85000644A0020E9B600087468726561643200C9
:10B86000F84E00206372656174652064796E616DC5
:10B8700069632073656D6170686F726520666169C8
:10B880006C65642E0A00000001461AA0FAF7B8BAE7
:10B8900010B50024AFF20F010A20FBF7B8FD0A2013
:10B8A000FBF7EFFD07E0214619A0FAF7A9FA641C9F
:10B8B0006420FCF70BFD0A2CF5DB10BD1CB5052040
:10B8C0001921CDE900104FF400730022154916A08C
:10B8D000FCF77CFB164C206008B1FCF701FB4FF431
:10B8E0009670FCF7F3FC0A212068FBF7A6FE002007
:10B8F0001CBD000074687265616431207265636507
:10B9000069766564207369676E616C2025640A003E
:10B910007468726561643120636F756E74203A20BB
:10B9200025640A0091B8000874687265616431008A
:10B93000D802002000244FF4FA752146641C1DA093
:10B94000FAF75EFA2846FCF7C1FCF6E710B50024CA
:10B9500021461DA0FAF754FA641C0A2CF8D3BDE85E
:10B9600010401EA0FAF74CBA1FB505241920CDE9E6
:10B9700000044FF4007300221C491DA0FCF726FBB5
:10B980001D49086008B1FCF7ABFA4FF480611B4A0F
:10B990001820CDE90021CDE902040023184A19A19D
:10B9A0001A48FCF738FA1948FCF79AFA04B0002054
:10B9B00010BD00007468726561643120636F756E3C
:10B9C000743A2025640A000074687265616432204C
:10B9D000636F756E743A2025640A0000746872659E
:10B9E00061643220657869740A00000035B9000886
:10B9F0007468726561643100DC0200208C4F0020A5
:10BA00004DB9000874687265616432008C5300207F
:10BA100010B5194C19A02168FAF7F2F92068411CF9
:10BA20002160092807DB6068FCF70CF8BDE81040CE
:10BA30001AA0FAF7E5B910BD20A0FAF7E1B938B5B8
:10BA4000022000900A230022234924A0FBF726FFAE
:10BA5000094C606008B1FBF768FF002002460090C7
:10BA60001E23204920A0FBF719FFA06008B1FBF7B7
:10BA70005CFF002038BD0000E002002070657269A4
:10BA80006F6469632074696D6572206973207469DD
:10BA90006D656F75742025640A0000007065726919
:10BAA0006F6469632074696D6572207761732073B8
:10BAB000746F7070656421200A0000006F6E65204D
:10BAC00073686F742074696D65722069732074697E
:10BAD0006D656F75740A000011BA000874696D65B0
:10BAE0007231000039BA000874696D657232000065
:10BAF00070B5064600240525B4FBF5F305FB13409D
:10BB000038B923463246314612A0FAF779F9C82CE3
:10BB100001D8641CF0E770BD7CB50A201424CDE97F
:10BB200000404FF480652B460122154915A0FCF713
:10BB30004DFA08B1FCF7D4F90520CDE900402B46B9
:10BB400002220F4911A0FCF741FA08B1FCF7C8F92D
:10BB500000207CBD7468726561642025642069736F
:10BB60002072756E6E696E67202C746872656164F0
:10BB700020256420636F756E74203D2025640A00C3
:10BB8000F1BA0008746872656164310074687265A6
:10BB90006164320040EA01039B0703D009E008C951
:10BBA000121F08C0042AFAD203E011F8013B00F882
:10BBB000013B521EF9D27047D2B201E000F8012BCE
:10BBC000491EFBD270470022F6E710B513460A461D
:10BBD00004461946FFF7F0FF204610BD421E12F83A
:10BBE000013F002BFBD111F8013B02F8013B002B78
:10BBF000F9D17047421C10F8011B0029FBD1801AB3
:10BC0000704730B504460020034600E05B1C9342B9
:10BC100003D2E05CCD5C401BF8D030BD034611F888
:10BC2000012B00F8012B002AF9D11846704730B5D6
:10BC300005460020034600E05B1C934205D2EC5C05
:10BC4000C85C201A01D1002CF6D130BD064C074D3E
:10BC500006E0E06840F0010394E8070098471034DC
:10BC6000AC42F6D3F4F768FA60DD000880DD000826
:10BC700070B58C1810F8015B15F0070301D110F8AE
:10BC8000013B2A1106D110F8012B03E010F8016BDB
:10BC900001F8016B5B1EF9D12B0705D40023521E5E
:10BCA0000DD401F8013BFAE710F8013BCB1A921CC6
:10BCB00003E013F8015B01F8015B521EF9D5A142C4
:10BCC000D8D3002070BD02E008C8121F08C1002AA6
:10BCD000FAD170477047002001E001C1121F002A0D
:10BCE000FBD1704753797374656D436C6F636B5F01
:10BCF000436F6E6669670000FFFFFFFF00000000F2
:10BD0000000000000000000001000000B503000872
:10BD1000001801400400000002000000B503000804
:10BD2000001801400800000003000000B5030008EF
:10BD3000001801401000000004000000B5030008D6
:10BD4000001801402000000005000000B5030008B5
:10BD50000018014040000000FFFFFFFF000000004E
:10BD60000000000000000000070000008903000838
:10BD700000100140002000000800000089030008B6
:10BD80000010014000400000090000008903000885
:10BD900000100140008000000A000000CB030008F2
:10BDA000001C0140010000000B000000CB03000854
:10BDB000001C0140020000000C000000CB03000842
:10BDC000001C0140040000000D000000CB0300082F
:10BDD000001C0140080000000E000000CB0300081A
:10BDE000001C0140100000000F000000CB03000801
:10BDF000001C014020000000FFFFFFFF00000000CA
:10BE00000000000000000000FFFFFFFF0000000036
:10BE1000000000000000000012000000CB0300083A
:10BE2000001C01404000000013000000CB0300088C
:10BE3000001C01408000000014000000CB0300083B
:10BE4000001C01400001000015000000CB030008A9
:10BE5000001C01400002000016000000CB03000897
:10BE6000001C014000040000FFFFFFFF0000000075
:10BE70000000000000000000FFFFFFFF00000000C6
:10BE80000000000000000000FFFFFFFF00000000B6
:10BE900000000000000000001A00000089030008F4
:10BEA00000100140010000001B0000008903000891
:10BEB00000100140020000001C000000890300087F
:10BEC00000100140040000001D000000890300086C
:10BED0000010014008000000FFFFFFFF000000000D
:10BEE0000000000000000000FFFFFFFF0000000056
:10BEF0000000000000000000FFFFFFFF0000000046
:10BF00000000000000000000FFFFFFFF0000000035
:10BF10000000000000000000220000005D03000897
:10BF20000008014001000000230000005D0300083C
:10BF30000008014002000000240000005D0300082A
:10BF40000008014004000000250000005D03000817
:10BF50000008014008000000FFFFFFFF0000000094
:10BF60000000000000000000FFFFFFFF00000000D5
:10BF70000000000000000000280000005D03000831
:10BF80000008014010000000290000005D030008C7
:10BF900000080140200000002A0000005D030008A6
:10BFA00000080140400000002B0000005D03000875
:10BFB00000080140800000002C00000089030008F8
:10BFC00000100140100000002D000000890300084F
:10BFD00000100140200000002E0000007303000844
:10BFE000000C0140010000002F0000007303000856
:10BFF000000C014002000000300000007303000844
:10C00000000C01400400000031000000CB030008D8
:10C01000001C01400008000032000000CB030008B3
:10C02000001C014000100000FFFFFFFF00000000A7
:10C030000000000000000000FFFFFFFF0000000004
:10C04000000000000000000035000000CB030008E5
:10C05000001C01400020000036000000CB03000857
:10C06000001C01400040000037000000CB03000826
:10C07000001C01400080000038000000E1030008BF
:10C08000002001400100000039000000E103000829
:10C0900000200140020000003A000000B503000843
:10C0A00000180140800000003B000000B5030008BC
:10C0B00000180140000100003C000000B50300082A
:10C0C0000018014000020000FFFFFFFF0000000019
:10C0D0000000000000000000FFFFFFFF0000000064
:10C0E00000000000000000003F000000B503000851
:10C0F000001801400004000040000000B5030008E3
:10C10000001801400008000041000000B5030008CD
:10C11000001801400010000042000000B5030008B4
:10C12000001801400020000043000000B503000893
:10C13000001801400040000044000000B503000862
:10C140000018014000800000450000007303000853
:10C15000000C0140000400004600000073030008CA
:10C16000000C014000080000FFFFFFFF000000007E
:10C170000000000000000000FFFFFFFF00000000C3
:10C1800000000000000000004900000073030008E8
:10C19000000C0140001000004A000000730300087A
:10C1A000000C0140002000004B0000007303000859
:10C1B000000C0140004000004C0000007303000828
:10C1C000000C0140008000004D0000009F030008AB
:10C1D00000140140000100004E0000009F03000811
:10C1E00000140140000200004F0000009F030008FF
:10C1F0000014014000040000500000009F030008EC
:10C200000014014000080000510000009F030008D6
:10C210000014014000100000520000009F030008BD
:10C220000014014000200000FFFFFFFF000000009D
:10C230000000000000000000FFFFFFFF0000000002
:10C240000000000000000000550000009F030008EF
:10C250000014014000400000560000009F03000849
:10C26000001401400080000057000000E1030008B6
:10C27000002001400400000058000000E103000815
:10C28000002001400800000059000000E103000800
:10C2900000200140100000005A000000E1030008E7
:10C2A00000200140200000005B000000E1030008C6
:10C2B00000200140400000005C000000E103000895
:10C2C00000200140800000005D000000E103000844
:10C2D0000020014000010000FFFFFFFF0000000000
:10C2E0000000000000000000FFFFFFFF0000000052
:10C2F000000000000000000060000000890300084A
:10C3000000100140400000006100000089030008A7
:10C310000010014080000000620000008903000856
:10C3200000100140000100006300000089030008C4
:10C330000010014000020000640000005D030008DE
:10C340000008014000010000650000005D030008D6
:10C350000008014000020000660000005D030008C4
:10C360000008014000040000670000005D030008B1
:10C370000008014000080000680000005D0300089C
:10C380000008014000100000690000005D03000883
:10C390000008014000200000FFFFFFFF0000000038
:10C3A0000000000000000000FFFFFFFF0000000091
:10C3B0000000000000000000FFFFFFFF0000000081
:10C3C00000000000000000006D0000005D03000898
:10C3D00000080140004000006E0000005D030008FE
:10C3E00000080140008000006F0000008903000881
:10C3F00000100140000400007000000089030008E4
:10C4000000100140000800007100000089030008CE
:10C410000010014000100000720000009F0300089F
:10C420000014014001000000730000009F03000899
:10C430000014014002000000740000009F03000887
:10C440000014014004000000750000009F03000874
:10C450000014014008000000760000009F0300085F
:10C460000014014010000000770000009F03000846
:10C470000014014020000000FFFFFFFF000000004B
:10C480000000000000000000FFFFFFFF00000000B0
:10C4900000000000000000007A0000009F03000878
:10C4A00000140140400000007B0000009F030008D2
:10C4B00000140140800000007C000000E10300083F
:10C4C00000200140000200007D000000E1030008A0
:10C4D00000200140000400007E000000E10300088D
:10C4E00000200140000800007F000000E103000878
:10C4F000002001400010000080000000E10300085F
:10C50000002001400020000081000000E10300083D
:10C510000020014000400000FFFFFFFF000000007E
:10C520000000000000000000FFFFFFFF000000000F
:10C53000000000000000000084000000E10300088B
:10C540000020014000800000850000007303000807
:10C55000000C014008000000860000007303000882
:10C56000000C014010000000870000007303000869
:10C57000000C014020000000880000007303000848
:10C58000000C014040000000890000007303000817
:10C59000000C014080000000FFFFFFFF00000000D2
:10C5A00000000000000000008B0000007303000882
:10C5B000000C0140000100008C0000007303000823
:10C5C000000C0140000200008D000000B5030008CF
:10C5D00000180140010000008E000000B5030008B3
:10C5E0000018014002000000FFFFFFFF00000000F4
:10C5F0000000000000000000FFFFFFFF000000003F
:10C60000000000000000000001000600020007001A
:10C61000040008000800090010000A0020001700AC
:10C6200040001700800017000001170000021700EB
:10C63000000428000008280000102800002028001E
:10C6400000402800008028004B0400080F04000868
:10C650002D040008A3040008310500088F05000818
:10C6600000C2010008000100AD07000847080008EB
:10C67000AF080008D70800080000000073746D338D
:10C68000325F636F6E6669677572650073746D33D0
:10C69000325F636F6E74726F6C0073746D33325FF0
:10C6A000707574630073746D33325F676574630013
:10C6B000756172745F697372004D585F55534152D2
:10C6C000545F554152545F496E6974000000000088
:10C6D0000000000001020304060708090000000032
:10C6E0000102030472745F6170706C696361746944
:10C6F0006F6E5F696E69740072745F6465766963FA
:10C70000655F756E72656769737465720072745FD8
:10C710006465766963655F66696E640072745F6400
:10C7200065766963655F64657374726F79007274AE
:10C730005F6465766963655F696E69740072745FD2
:10C740006465766963655F6F70656E0072745F64BF
:10C7500065766963655F636C6F73650072745F64AF
:10C7600065766963655F726561640072745F6465B4
:10C77000766963655F77726974650072745F64657A
:10C78000766963655F636F6E74726F6C0072745F5D
:10C790006465766963655F7365745F72785F696EFF
:10C7A0006469636174650072745F6465766963656A
:10C7B0005F7365745F74785F636F6D706C657465CB
:10C7C0000072745F7468726561645F69646C655F50
:10C7D0006578637574650072745F73656D5F696E0B
:10C7E00069740072745F73656D5F6465746163681A
:10C7F0000072745F73656D5F63726561746500726A
:10C80000745F73656D5F64656C6574650072745FF9
:10C8100073656D5F74616B650072745F73656D5FE6
:10C8200072656C656173650072745F73656D5F63DB
:10C830006F6E74726F6C0072745F6D757465785F83
:10C84000696E69740072745F6D757465785F646594
:10C85000746163680072745F6D757465785F63728C
:10C86000656174650072745F6D757465785F646589
:10C870006C6574650072745F6D757465785F746162
:10C880006B650072745F6D757465785F72656C6559
:10C890006173650072745F6D757465785F636F6E48
:10C8A00074726F6C0072745F6576656E745F696E2A
:10C8B00069740072745F6576656E745F6465746137
:10C8C00063680072745F6576656E745F637265613C
:10C8D00074650072745F6576656E745F64656C651F
:10C8E00074650072745F6576656E745F73656E64FF
:10C8F0000072745F6576656E745F72656376007250
:10C90000745F6576656E745F636F6E74726F6C00D2
:10C9100072745F6D625F696E69740072745F6D62DC
:10C920005F6465746163680072745F6D625F6372F7
:10C93000656174650072745F6D625F64656C6574D7
:10C94000650072745F6D625F73656E645F776169C5
:10C95000740072745F6D625F726563760072745FFB
:10C960006D625F636F6E74726F6C0072745F6D7175
:10C970005F696E69740072745F6D715F6465746184
:10C9800063680072745F6D715F63726561746500E6
:10C9900072745F6D715F64656C6574650072745F5D
:10C9A0006D715F73656E640072745F6D715F757237
:10C9B00067656E740072745F6D715F726563760097
:10C9C00072745F6D715F636F6E74726F6C000000E4
:10C9D0000100020001000300010002000100040048
:10C9E0000100020001000300010002000100050037
:10C9F0000100020001000300010002000100040028
:10CA00000100020001000300010002000100060015
:10CA10000100020001000300010002000100040007
:10CA200001000200010003000100020001000500F6
:10CA300001000200010003000100020001000400E7
:10CA400001000200010003000100020001000700D4
:10CA500001000200010003000100020001000400C7
:10CA600001000200010003000100020001000500B6
:10CA700001000200010003000100020001000400A7
:10CA80000100020001000300010002000100060095
:10CA90000100020001000300010002000100040087
:10CAA0000100020001000300010002000100050076
:10CAB0000100020001000300010002000100040067
:10CAC00001000200010003000100020001003031FA
:10CAD0003233343536373839616263646566003025
:10CAE00031323334353637383941424344454600D4
:10CAF00072745F6672656500706C75675F686F6CF5
:10CB000065730072745F73797374656D5F686561D6
:10CB1000705F696E69740072745F6D616C6C6F63D5
:10CB20000072745F7265616C6C6F630072745F6336
:10CB3000616C6C6F630072745F6D705F696E6974B5
:10CB40000072745F6D705F64657461636800727415
:10CB50005F6D705F6372656174650072745F6D70A4
:10CB60005F64656C6574650072745F6D705F616CA5
:10CB70006C6F630072745F6F626A6563745F696E85
:10CB800069740072745F6F626A6563745F64657470
:10CB90006163680072745F6F626A6563745F616C81
:10CBA0006C6F636174650072745F6F626A65637451
:10CBB0005F64656C6574650072745F6F626A65635B
:10CBC000745F69735F73797374656D6F626A6563AF
:10CBD000740072745F6F626A6563745F6765745F27
:10CBE000747970650072745F6F626A6563745F6602
:10CBF000696E64005F72745F7363686564756C6509
:10CC0000725F737461636B5F636865636B007274FA
:10CC10005F7363686564756C655F696E7365727474
:10CC20005F7468726561640072745F7363686564E1
:10CC3000756C655F72656D6F76655F74687265614E
:10CC4000640072745F7369676E616C5F77616974A9
:10CC50000072745F7468726561645F616C6C6F63AD
:10CC60005F7369670072745F7468726561645F6B9B
:10CC7000696C6C0072745F73797374656D5F73694E
:10CC8000676E616C5F696E69740072745F74696D60
:10CC900065725F696E69740072745F74696D657244
:10CCA0005F6465746163680072745F74696D657256
:10CCB0005F64656C6574650072745F74696D65723C
:10CCC0005F73746172740072745F74696D65725F12
:10CCD00073746F700072745F74696D65725F636FF7
:10CCE0006E74726F6C005F72745F746872656164F9
:10CCF0005F696E69740072745F7468726561645F05
:10CD0000696E69740072745F7468726561645F73E0
:10CD10007461727475700072745F746872656164B6
:10CD20005F6465746163680072745F7468726561E2
:10CD3000645F64656C6574650072745F74687265C5
:10CD400061645F736C6565700072745F74687265AE
:10CD500061645F636F6E74726F6C0072745F74688D
:10CD6000726561645F73757370656E640072745F81
:10CD70007468726561645F726573756D6500727465
:10CD80005F7468726561645F74696D656F75740066
:10CD900072745F7468726561645F66696E64007264
:10CDA000745F68775F6370755F73687574646F77BD
:10CDB0006E005F70696E5F72656164005F70696EBE
:10CDC0005F7772697465005F70696E5F636F6E7420
:10CDD000726F6C0072745F70696E5F61747461630E
:10CDE000685F6972710072745F70696E5F64657408
:10CDF000746163685F6972710072745F70696E5FFD
:10CE00006972715F656E61626C650072745F7069F2
:10CE10006E5F6D6F64650072745F70696E5F7772CC
:10CE20006974650072745F70696E5F726561640039
:10CE30005F73657269616C5F706F6C6C5F727800B4
:10CE40005F73657269616C5F706F6C6C5F747800A2
:10CE50005F73657269616C5F696E745F727800728E
:10CE6000745F73657269616C5F696E697400727476
:10CE70005F73657269616C5F6F70656E0072745F7D
:10CE800073657269616C5F636C6F73650072745F68
:10CE900073657269616C5F726561640072745F735F
:10CEA000657269616C5F77726974650072745F7333
:10CEB000657269616C5F636F6E74726F6C0072741F
:10CEC0005F68775F73657269616C5F7265676973CC
:10CED0007465720072745F68775F73657269616C04
:10CEE0005F6973720066696E73685F676574636813
:10CEF00061720066696E73685F72785F696E640064
:10CF000066696E73685F7365745F6465766963658F
:10CF10000066696E73685F6765745F6465766963F0
:10CF2000650066696E73685F7365745F6563686FDB
:10CF30000066696E73685F6765745F6563686F003C
:10CF40006CD3000828D30008BCD20008D0D2000857
:10CF5000E8D20008B8D2000804D30008F4D20008D0
:10CF6000A8D3000814D30008C4D30008B0D3000825
:10CF7000DCD20008B8D3000848D3000898D30008D2
:10CF800038D300085CD3000880D30008A0D3000881
:10CF90005F6D73685F657865635F636D6400000053
:10CFA00048414C5F5243435F436C6F636B436F6E0A
:10CFB00066696728265243435F436C6B496E697408
:10CFC0005374727563742C20464C4153485F4C4136
:10CFD00054454E43595F3229203D3D2048414C5F26
:10CFE0004F4B000072745F6F626A6563745F6765C0
:10CFF000745F74797065282673656D2D3E7061725B
:10D00000656E742E706172656E7429203D3D2052EC
:10D01000545F4F626A6563745F436C6173735F53FF
:10D02000656D6170686F72650000000072745F6FFB
:10D03000626A6563745F6765745F747970652826DA
:10D040006D712D3E706172656E742E706172656EC9
:10D050007429203D3D2052545F4F626A6563745FBE
:10D06000436C6173735F4D6573736167655175657B
:10D070007565000072745F6F626A6563745F6765EF
:10D08000745F7479706528266576656E742D3E70C0
:10D090006172656E742E706172656E7429203D3DFB
:10D0A0002052545F4F626A6563745F436C617373AF
:10D0B0005F4576656E74000072745F6F626A6563C7
:10D0C000745F6765745F7479706528266D75746523
:10D0D000782D3E706172656E742E706172656E742B
:10D0E00029203D3D2052545F4F626A6563745F435F
:10D0F0006C6173735F4D75746578000072745F6F57
:10D10000626A6563745F6765745F74797065282609
:10D110006D622D3E706172656E742E706172656E07
:10D120007429203D3D2052545F4F626A6563745FED
:10D13000436C6173735F4D61696C426F78000000EE
:10D140002872745F75696E7433325F74292828728F
:10D15000745F75696E74385F74202A296D656D205F
:10D160002B2053495A454F465F5354525543545F01
:10D170004D454D2920252052545F414C49474E5F73
:10D1800053495A45203D3D20300000002872745F0D
:10D1900075696E74385F74202A29726D656D203E42
:10D1A0003D202872745F75696E74385F74202A2977
:10D1B000686561705F707472202626202872745F23
:10D1C00075696E74385F74202A29726D656D203C14
:10D1D000202872745F75696E74385F74202A29681C
:10D1E0006561705F656E64002872745F75696E7446
:10D1F00033325F74296D656D202B2053495A454F9A
:10D20000465F5354525543545F4D454D202B207378
:10D21000697A65203C3D202872745F75696E7433AD
:10D22000325F7429686561705F656E64000000009C
:10D2300072745F6F626A6563745F6765745F747947
:10D240007065282872745F6F626A6563745F742901
:10D2500074687265616429203D3D2052545F4F62BD
:10D260006A6563745F436C6173735F546872656170
:10D2700064000000252D2A2E73207072692020730F
:10D28000746174757320202020202073702020206A
:10D290002020737461636B2073697A65206D6178F7
:10D2A0002075736564206C656674207469636B20F7
:10D2B000206572726F720A00525443004E65747793
:10D2C0006F726B20496E7465726661636500000061
:10D2D0004D544420446576696365000053504920ED
:10D2E000446576696365000043414E204465766974
:10D2F0006365000047726170686963204465766900
:10D3000063650000536F756E6420446576696365DC
:10D310000000000055534220536C6176652044653F
:10D320007669636500000000426C6F636B204465A2
:10D330007669636500000000506F7274616C204470
:10D340006576696365000000504D20507365756413
:10D350006F204465766963650000000054696D655F
:10D36000722044657669636500000000436861725D
:10D37000616374657220446576696365000000002E
:10D380004D697363656C6C616E656F757320446580
:10D390007669636500000000506970650000000058
:10D3A000556E6B6E6F776E00493243204275730085
:10D3B00053504920427573005344494F20427573BE
:10D3C0000000000055534220486F7374204275736B
:10D3D000005F5F636D645F6C65640052542D546838
:10D3E00072656164206669727374206C6564207371
:10D3F000616D706C65006C6973745F6D656D006C58
:10D40000697374206D656D6F7279207573616765DE
:10D4100020696E666F726D6174696F6E0070696EFF
:10D420004D6F646500736574206861726477617222
:10D43000652070696E206D6F64650070696E57724B
:10D440006974650077726974652076616C75652012
:10D45000746F2068617264776172652070696E0014
:10D4600070696E52656164007265616420737461F5
:10D470007475732066726F6D206861726477617273
:10D48000652070696E0068656C6C6F00736179204F
:10D4900068656C6C6F20776F726C64007665727370
:10D4A000696F6E0073686F772052542D54687265EF
:10D4B00061642076657273696F6E20696E666F7243
:10D4C0006D6174696F6E005F5F636D645F76657236
:10D4D00073696F6E0073686F772052542D546872B1
:10D4E0006561642076657273696F6E20696E666F20
:10D4F000726D6174696F6E006C6973745F746872C9
:10D50000656164006C69737420746872656164009D
:10D510005F5F636D645F6C6973745F74687265618B
:10D5200064006C69737420746872656164006C696E
:10D5300073745F73656D006C6973742073656D61DE
:10D5400070686F6E6520696E2073797374656D0005
:10D550005F5F636D645F6C6973745F73656D006CAE
:10D560006973742073656D6170686F726520696E90
:10D570002073797374656D006C6973745F6576658B
:10D580006E74006C697374206576656E7420696EC4
:10D590002073797374656D005F5F636D645F6C69A0
:10D5A00073745F6576656E74006C6973742065765C
:10D5B000656E7420696E2073797374656D006C6993
:10D5C00073745F6D75746578006C697374206D7524
:10D5D00074657820696E2073797374656D005F5F80
:10D5E000636D645F6C6973745F6D75746578006CEE
:10D5F000697374206D7574657820696E2073797312
:10D6000074656D006C6973745F6D61696C626F78CD
:10D61000006C697374206D61696C20626F78206999
:10D620006E2073797374656D005F5F636D645F6C0A
:10D630006973745F6D61696C626F78006C69737493
:10D64000206D61696C20626F7820696E2073797338
:10D6500074656D006C6973745F6D73677175657562
:10D6600065006C697374206D657373616765207103
:10D670007565756520696E2073797374656D005FDB
:10D680005F636D645F6C6973745F6D7367717565FB
:10D690007565006C697374206D65737361676520CF
:10D6A000717565756520696E2073797374656D0099
:10D6B0006C6973745F6D656D68656170006C69732A
:10D6C00074206D656D6F7279206865617020696E78
:10D6D0002073797374656D005F5F636D645F6C695F
:10D6E00073745F6D656D68656170006C697374203B
:10D6F0006D656D6F7279206865617020696E207349
:10D70000797374656D006C6973745F6D656D706FAE
:10D710006F6C006C697374206D656D6F7279207029
:10D720006F6F6C20696E2073797374656D005F5F35
:10D73000636D645F6C6973745F6D656D706F6F6C42
:10D74000006C697374206D656D6F727920706F6FF6
:10D750006C20696E2073797374656D006C697374E5
:10D760005F74696D6572006C6973742074696D65AE
:10D770007220696E2073797374656D005F5F636DED
:10D78000645F6C6973745F74696D6572006C697352
:10D79000742074696D657220696E20737973746585
:10D7A0006D006C6973745F646576696365006C69AC
:10D7B00073742064657669636520696E207379737C
:10D7C00074656D005F5F636D645F6C6973745F6443
:10D7D0006576696365006C69737420646576696356
:10D7E0006520696E2073797374656D006C6973745C
:10D7F000006C69737420616C6C2073796D626F6C5E
:10D8000020696E2073797374656D005F5F636D646A
:10D810005F68656C700052542D54687265616420B5
:10D820007368656C6C2068656C702E005F5F636D5B
:10D83000645F7073004C697374207468726561640E
:10D840007320696E207468652073797374656D2E1A
:10D85000005F5F636D645F74696D65004578656343
:10D8600075746520636F6D6D616E6420776974688F
:10D870002074696D652E005F5F636D645F6672651D
:10D88000650053686F7720746865206D656D6F72F1
:10D890007920757361676520696E207468652073EF
:10D8A000797374656D2E005F5F636D645F64796E7C
:10D8B0006D656D5F73616D706C650064796E6D652B
:10D8C0006D2073616D706C65005F5F636D645F6593
:10D8D00076656E745F73616D706C65006576656EFC
:10D8E000742073616D706C65005F5F636D645F6968
:10D8F000646C655F686F6F6B5F73616D706C650002
:10D9000069646C6520686F6F6B2073616D706C6506
:10D91000005F5F636D645F696E74657272757074C9
:10D920005F73616D706C6500696E7465727275709D
:10D93000742073616D706C65005F5F636D645F6D13
:10D9400061696C626F785F73616D706C65006D61A9
:10D95000696C626F782073616D706C65005F5F63E6
:10D960006D645F6D656D706F6F6C5F73616D706C12
:10D9700065006D656D706F6F6C2073616D706C65A7
:10D98000005F5F636D645F6D7367715F73616D707E
:10D990006C65006D7367712073616D706C65005FFD
:10D9A0005F636D645F6D757465785F73616D706CD6
:10D9B00065006D757465782073616D706C65005FCE
:10D9C0005F636D645F7072695F696E7665727369BB
:10D9D0006F6E007072695F696E76657273696F6EE3
:10D9E0002073616D706C65005F5F636D645F707262
:10D9F0006F64756365725F636F6E73756D657200DA
:10DA000070726F64756365725F636F6E73756D6559
:10DA1000722073616D706C65005F5F636D645F732E
:10DA200063686564756C65725F686F6F6B007363C4
:10DA3000686564756C65725F686F6F6B2073616D8C
:10DA4000706C65005F5F636D645F73656D617068C6
:10DA50006F72655F73616D706C650073656D617089
:10DA6000686F72652073616D706C65005F5F636DD8
:10DA7000645F7369676E616C5F73616D706C650084
:10DA80007369676E616C2073616D706C65005F5FB8
:10DA9000636D645F7468726561645F73616D706CFF
:10DAA00065007468726561642073616D706C6500F7
:10DAB0005F5F636D645F74696D65725F73616D70E4
:10DAC0006C650074696D65722073616D706C6500C2
:10DAD0005F5F636D645F74696D65736C6963655FD7
:10DAE00073616D706C650074696D65736C696365F5
:10DAF0002073616D706C6500813500088535000804
:10DB00006F06000881090008893500083F97000862
:10DB10008D350008D1D30008DBD30008730100085D
:10DB2000F6D30008FFD30008A36700081DD400083F
:10DB300025D40008018C00083BD4000844D4000818
:10DB40002B8C000860D4000868D40008558C0008AD
:10DB500086D400088CD40008F19700089CD40008F3
:10DB6000A4D40008FD970008C7D40008D5D4000845
:10DB7000FD970008F8D4000804D50008F3980008C1
:10DB800010D5000822D50008F39800082ED500080B
:10DB900037D50008AD99000850D500085FD50008BA
:10DBA000AD99000878D5000883D50008399A000897
:10DBB00098D50008A9D50008399A0008BED50008F4
:10DBC000C9D50008A99A0008DED50008EFD50008DD
:10DBD000A99A000804D6000811D60008479B00083F
:10DBE00029D600083CD60008479B000854D60008F8
:10DBF00062D60008C59E00087FD6000893D60008AC
:10DC0000C59E0008B0D60008BDD60008239F0008B6
:10DC1000D8D60008EBD60008239F000806D70008D6
:10DC200013D70008B59F00082ED7000841D7000879
:10DC3000B59F00085CD7000867D7000833A000082C
:10DC40007CD700088DD7000833A00008A2D70008B1
:10DC5000AED70008A9A00008C4D70008D6D700088E
:10DC6000A9A00008ECD70008F1D70008B9A0000867
:10DC70000BD8000816D8000871A300082CD800089B
:10DC800035D8000891A6000851D800085CD80008D3
:10DC90009BA6000877D8000882D800089FA6000835
:10DCA000A7D80008BBD80008E7A60008C9D8000814
:10DCB000DCD80008F9A70008E9D8000800D9000856
:10DCC000D7A9000811D9000828D90008B3AA00086C
:10DCD00039D900084ED900089DAB00085DD900086D
:10DCE00072D90008FDAC000881D9000893D900085A
:10DCF00079AE00089FD90008B2D9000875B00008B5
:10DD0000BFD90008D3D900083BB20008E8D9000801
:10DD100000DA000873B4000819DA00082EDA0008E7
:10DD200029B6000844DA00085BDA000821B70008C9
:10DD30006CDA000880DA0008BDB800088EDA000846
:10DD4000A2DA000869B90008B0DA0008C3DA0008EE
:10DD50003FBA0008D0DA0008E7DA000819BB00086B
:10DD600080DD000800000020EC02000070BC00080C
:10DD700014DE0008EC02002034550000D6BC000878
:10DD8000A3FFFF09B20C11043C3801404225046096
:10DD9000A24A041368012A2004329432011A780C32
:10DDA0002904322032021A880C2904322432031A40
:10DDB000980C29042920299D1AA80C2904323032F4
:10DDC000051AB80C2904323432061AC80C29043258
:10DDD0006432071AD80C2904323832081AE80C29A0
:10DDE00004324032091AF80C2904026B2C156F76A4
:10DDF0006572100C49276D2061206D61696C211ED0
:10DE00007468697320035808616E6F7468657216D0
:04DE100001590000B4
:0400000508000131BD
:00000001FF
